:100000000C941D200C944E200C944E200C944E20E9
:100010000C944E200C944E200C944E200C944E20A8
:100020000C944E200C944E200C944E200C944E2098
:100030000C944E200C946EC70C944E200C944E20C1
:100040000C944E200C94B7E00C944E200C944E204F
:100050000C944E200C944E200C9467FC0C947FB2B0
:100060000C944E200C94E9610C94DF610C944E20AA
:100070000C944E200C944E200C944E200C944E2048
:100080000C944E200C944E200C944E200C944E2038
:100090000C944E200C944E200C944E200C944E2028
:1000A0000C944E200C944E200C944E200C944E2018
:1000B0000C944E200C944E200C944E200C944E2008
:1000C0000C944E200C944E200C944E200C944E20F8
:1000D0000C944E200C944E200C944E200C944E20E8
:1000E0000C944E2066B069B058B05CB062B0A0B05D
:1000F0006DB071B077B07BB07FB085B089B08DB096
:10010000A0B093B097B09BB09BB1A0B1A5B1AFB177
:10011000B9B132B2C3B1CBB1D3B1DDB1E7B1F1B155
:1001200000B20AB232B214B21EB228B2E700E30043
:10013000C900CF00E900CD00F500FD00CB00DF00D5
:100140000901084AD73B3BCE016E84BCBFFDC12FDD
:100150003D6C74319ABD56833DDA3D00C77F11BEB8
:10016000D9E4BB4C3E916BAAAABE000000803F05BB
:10017000A84CCDB2D44EB93836A9020C50B99186EC
:1001800088083CA6AAAA2ABE000000803F000D9461
:10019000B8070D94E61A0D940B1B0D94EF1A0D94ED
:1001A000E91A0D94CA030D940A170D942E190D9493
:1001B000C0010D9462190D9435190D9465190D94B3
:1001C000F51A0D944A190D94011B0D9427190D94DD
:1001D000FE1A0D94EC1A0D9497370D9458190D943E
:1001E0005F190D9468190D9446050D94FB1A0D9432
:1001F00051190D945E1B0D94E6400D94F21A0D9466
:1002000043190D947F060D9482150D9420190D94B9
:100210003C190D94F81A4E414E494E495459494ED5
:1002200046CDCCCC3D0AD7233C17B7D13877CC2B61
:10023000329595E6241FB14F0A000020410000C806
:100240004200401C4620BCBE4CCA1B0E5AAEC59D87
:1002500074434F4D4D554E49434154494F4E004410
:10026000525952554E004552524F525300494E4634
:100270004F004543484F00536C6565702E2E2E008D
:10028000205A3A200020593A200042656420583A0A
:1002900020004D65736820706F696E742063616E15
:1002A0006E6F74206265207265736F6C7665640A88
:1002B00000436C69636B20746F20726573756D65A4
:1002C0002E2E2E004E6F206D6F76652E00456E64CB
:1002D0002066696C65206C6973740A004265676901
:1002E0006E2066696C65206C6973740A00286E6FF5
:1002F0002066696C65290043757272656E742066AC
:10030000696C653A20005344207072696E74696E9E
:1003100067206279746520004E6F7420534420700A
:1003200072696E74696E670A0044656C6574696F02
:100330006E206661696C65642C2046696C653A20A4
:100340000046696C652064656C657465643A0050AC
:1003500072696E742074696D653A200046696C613B
:100360006D656E7420757365643A20005374617412
:10037000733A20002C204C6F6E67657374206A6F8F
:10038000623A2000546F74616C2074696D653A2084
:100390000053746174733A20002C204661696C65C7
:1003A000643A20002C2046696E69736865643A20BF
:1003B000005072696E74733A200053746174733A1A
:1003C00020004520436F6F6C696E672E2E2E00450E
:1003D0002048656174696E672E2E2E006F66660078
:1003E00072026D0266025F02510244454255473A6D
:1003F000004D3131332053006F6B00414E5943554E
:10040000424943204B6F7373656C204F46462E0064
:100410004D4F54494F4E5F4D4F444553005448454E
:10042000524D414C5F50524F54454354494F4E003A
:100430004155544F5245504F52545F53445F5354AB
:100440004154555300454D455247454E43595F5021
:10045000415253455200434153455F4C494748542C
:100460005F4252494748544E45535300544F474703
:100470004C455F4C494748545300534F46545741ED
:1004800052455F504F574552004255494C445F50CA
:10049000455243454E54004C4556454C494E475FE6
:1004A00044415441005A5F50524F42450041555417
:1004B0004F4C4556454C005052494E545F4A4F42AE
:1004C0000050524F4752455353004155544F5245E7
:1004D000504F52545F54454D5000564F4C554D456A
:1004E0005452494300454550524F4D0053455249DF
:1004F000414C5F584F4E5F584F4646004649524D5B
:10050000574152455F4E414D453A4D61726C696E9F
:10051000206275676669782D322E302E7820284744
:1005200069746875622920534F555243455F434FA4
:1005300044455F55524C3A68747470733A2F2F6774
:1005400069746875622E636F6D2F4D61726C696E90
:100550004669726D776172652F4D61726C696E20AC
:1005600050524F544F434F4C5F56455253494F4E94
:100570003A312E30204D414348494E455F54595041
:10058000453A414E594355424943204B6F73736579
:100590006C2045585452554445525F434F554E5474
:1005A0003A3120555549443A636564653261326693
:1005B0002D343161322D343734382D396231322DBA
:1005C0006335356336326633363766660A002F2F59
:1005D00020004D31343520533C696E6465783E20EF
:1005E0006F7574206F662072616E67652028302DEC
:1005F00031290A00205400205200416363656C6574
:10060000726174696F6E3A2050005741524E494EE4
:100610004721204C6F77205A204A65726B206D610C
:1006200079206C65616420746F20756E77616E74DB
:100630006564207061757365732E0A00205A00206E
:100640005900580020204D61783A2000205A00209F
:100650005900580020204D696E3A2000536F66748F
:1006600020656E6473746F70733A200020466C6F5F
:10067000773A200050726F74656374656420506926
:100680006E0A00496E76616C6964206578747275D3
:100690006465720A0020643A0020693A0020703ACA
:1006A0000020643A0020693A0020703A00646973BF
:1006B00000656E0043290A0061626C656420286D44
:1006C000696E2074656D702000436F6C64206578DE
:1006D0007472756465732061726520004D6573687E
:1006E00020706F696E742063616E6E6F7420626536
:1006F000207265736F6C7665640A004D3432312068
:10070000696E636F727265637420706172616D658A
:100710007465722075736167650A00454550524FD4
:100720004D204F4B0A003F5A206F7574206F662092
:1007300072616E676520282D343020746F2032304E
:10074000290A0050726F6265205A204F66667365F1
:10075000743A2000496E76616C6964206578747221
:10076000756465720A007879007A7800797A0020D9
:100770007A0020790020780063002E2020202000BD
:10078000253033692E7800302E25303369002073F0
:10079000643A00456E64204452592D52554E004E25
:1007A0006F20636F6E76657267656E63650049746E
:1007B00065726174696F6E203A202530326900538A
:1007C0006176652077697468204D35303020616E20
:1007D000642F6F7220636F707920746F20436F6E87
:1007E00066696775726174696F6E2E6800253033B3
:1007F000692E7800302E253033690043616C6962C0
:10080000726174696F6E2073643A00726F6C6C6908
:100810006E67206261636B2E0043616C6962726176
:1008200074696F6E204F4B00436F72726563742062
:1008300064656C74612073657474696E6773207786
:10084000697468204D36363520616E64204D363629
:10085000360A0020284452592D52554E290043682B
:1008600065636B696E672E2E2E204143003F284D35
:1008700036363520422965642072616469757320BB
:10088000697320696D706C61757369626C652E0A9D
:1008900000473333204175746F2043616C69627285
:1008A0006174650A003F2856296572626F7365207E
:1008B0006C6576656C20697320696D706C61757309
:1008C00069626C652028302D33292E0A003F2846A6
:1008D000296F72636520697465726174696F6E2037
:1008E000697320696D706C61757369626C6520282D
:1008F000302D3330292E0A003F284329616C69626C
:10090000726174696F6E20707265636973696F6E6E
:1009100020697320696D706C61757369626C652004
:10092000283E3D30292E0A003F2850296F696E74F9
:100930007320697320696D706C61757369626C6591
:100940002028302D3130292E0A006F6B005265733C
:10095000656E643A200053544F505045442E200099
:100960005072696E7465722073746F707065642064
:1009700064756520746F206572726F72732E2046E5
:10098000697820746865206572726F7220616E6488
:1009900020757365204D39393920746F2072657365
:1009A000746172742E202854656D7065726174755F
:1009B00072652069732072657365742E20536574A7
:1009C0002069742061667465722072657374617247
:1009D00074696E67290A004E6F20436865636B7304
:1009E000756D2077697468206C696E65206E756D11
:1009F0006265722C204C617374204C696E653A20DC
:100A0000004E6F20436865636B73756D2077697462
:100A100068206C696E65206E756D6265722C204C65
:100A2000617374204C696E653A2000636865636B7E
:100A300073756D206D69736D617463682C204C61F2
:100A40007374204C696E653A20004C696E65204EC7
:100A5000756D626572206973206E6F74204C6173CE
:100A600074204C696E65204E756D6265722B312C59
:100A7000204C617374204C696E653A20004D313111
:100A800030004D333100534420726561642065723B
:100A9000726F720A00446F6E65207072696E7469BD
:100AA0006E672066696C650A004F4646004F4E002F
:100AB000426564204C6576656C696E67200046610E
:100AC000696C656420746F20656E61626C6520429C
:100AD0006564204C6576656C696E670A00496E76C0
:100AE000616C6964206D6573682E0A002028445289
:100AF0005952554E2900473239204175746F2042B2
:100B00006564204C6576656C696E67003F20284CF3
:100B10002C522C462C4229206F7574206F6620625F
:100B20006F756E64732E0A003F2856296572626FD6
:100B30007365206C6576656C20697320696D706CD7
:100B400061757369626C652028302D34292E0A0086
:100B5000426164205A2076616C75650A004E6F20F0
:100B600062696C696E65617220677269640A00204F
:100B7000200020205261646975733A00547A005451
:100B8000790054780020205261646975733A0045F9
:100B90007A004579004578002E4865696768743A9F
:100BA0000036372602353C3D380F312E303E1213C9
:100BB000281A1C182A08440A2C430809072C00018B
:100BC000627573793A2070617573656420666F721F
:100BD00020696E7075740A00627573793A207061CD
:100BE0007573656420666F7220757365720A0062A2
:100BF0007573793A2070726F63657373696E670AF3
:100C0000004B494C4C206361757365642062792008
:100C10004B494C4C20627574746F6E2F70696E0A6C
:100C2000004B494C4C2063617573656420627920E8
:100C3000746F6F206D75636820696E616374697687
:100C4000652074696D65202D2063757272656E7400
:100C500020636F6D6D616E643A2000506C65617346
:100C600065207265736574005052494E5445522098
:100C700048414C544544004B494C4C45442E2000BF
:100C80005072696E7465722068616C7465642E20A0
:100C90006B696C6C28292063616C6C6564210A00A7
:100CA0004572726F722077726974696E6720746F13
:100CB00020454550524F4D210A006563686F3A0048
:100CC0004572726F723A00486F74656E6420746F7B
:100CD0006F20636F6C640A004C6F6164206D6D005F
:100CE0004C6F6164206D6D00556E6C6F6164206D9A
:100CF0006D00556E6C6F6164206D6D0046696C2EE1
:100D0000204469612E0046696C2E204469612E00E2
:100D10004F6666004F6E004520696E206D6D5E3334
:100D200000416476616E6365642053657474696E16
:100D30006773004D333033205531204525692053EA
:100D4000256900504944204175746F74756E6500C3
:100D5000504944204175746F74756E650050494464
:100D60002D44005049442D44005049442D49005021
:100D700049442D49005049442D50005049442D50BC
:100D800000200220466163740020022046616374E3
:100D9000002002204D6178002002204D6178002063
:100DA00002204D696E002002204D696E004F66667C
:100DB000004F6E004175746F74656D70004164760C
:100DC000616E6365642053657474696E6773005661
:100DD00054726176206D696E005654726176206D92
:100DE000696E00566D696E00566D696E00566D61D4
:100DF00078204500566D6178204500566D61782059
:100E00004300566D6178204300566D6178204200A2
:100E1000566D6178204200566D6178204100566D14
:100E20006178204100416476616E6365642053659A
:100E30007474696E677300436172642072656D6FCC
:100E4000766564004361726420696E7365727465CF
:100E50006400414E594355424943204B6F737365BB
:100E60006C2052656164792E005072696E74696EEF
:100E7000672E2E2E005072696E7420706175736536
:100E80006400A10000006900A20000006300B0003F
:100E900000000900C10000004100C2000000410044
:100EA000C30000004100C40000004100C500000074
:100EB0004100C60000004145C70000004300C800D3
:100EC00000004500C90000004500CD0000004900B9
:100ED000D10000004E00D50000004F00D6000000F9
:100EE0004F00D70000007800DC0000005500DD0056
:100EF00000005900E00000006100E1000000610016
:100F0000E20000006100E30000006100E400000076
:100F10006100E50000006100E60000006165E70097
:100F200000006300E80000006500E90000006500C3
:100F3000EA0000006500EB0000006500EC00000026
:100F40006900ED0000006900EE0000006900EF009C
:100F500000006900F10000006E00F20000006F0068
:100F6000F30000006F00F40000006F00F5000000C7
:100F70006F00F60000006F00F80000006F00F9003D
:100F800000007500FA0000007500FB00000075000D
:100F9000FC0000007500FD0000007900FF0000006B
:100FA0007900040100004100050100006100060114
:100FB000000043000701000063000C010000430033
:100FC0000D01000063000E01000044000F0100004D
:100FD00064001101000064001901000065001F0198
:100FE0000000670030010000490031010000690085
:100FF000410100004C00420100006C004301000070
:101000004E00440100006E00480100006E005901CE
:10101000000072005A01000053005B0100007300E1
:101020005F010000730060010000530061010000D7
:1010300073006501000074006F01000075007C0101
:1010400000007A007D0100005A007E0100007A0055
:10105000920100006600E3020000780084030000B3
:101060002700850300002700860300004100870356
:1010700000002E008803000045008903000048009E
:101080008A03000049008C0300004F008E0300001B
:1010900059008F0300004F00900300006900910386
:1010A000000041009203000042009303000054003E
:1010B00094030000340095030000450096030000EF
:1010C0005A0097030000480098030000300099037D
:1010D000000049009A0300004B009B0300005E00E3
:1010E0009C0300004D009D0300004E009E03000085
:1010F00033009F0300004F00A00300006E00A10317
:1011000000005000A30300004500A40300005400A9
:10111000A50300005900A60300007000A70300000B
:101120005800A80300005000A90300004F00AA03C4
:1011300000004900AB0300005900AC03000061004F
:10114000AD0300006500AE0300006E00AF030000B9
:101150006900B00300007600B10300006100B20333
:1011600000004200B30300007600B40300006400F6
:10117000B50300006500B60300005A00B703000085
:101180006E00B80300003000B90300006900BA0324
:1011900000006B00BB0300004C00BC0300007500A6
:1011A000BD0300007600BE0300006500BF03000021
:1011B0006F00C00300006E00C10300007000C20396
:1011C00000006300C30300006F00C403000074004C
:1011D000C50300007600C60300007000C7030000CE
:1011E0005800C80300005700C90300007700CA0375
:1011F00000006900CB0300007600CC0300006F0004
:10120000CD0300007600CE0300007700010400004B
:1012100045001004000041001104000062001204A7
:1012200000004200130400005400140400005100A8
:10123000150400004500160400002A0017040000F1
:101240004500180400004E00190400004E001A0466
:1012500000004B001B04000054001C0400004D0063
:101260001D04000048001E0400004F001F04000081
:101270006E002004000050002104000043002204FE
:1012800000005400230400005900240400006F00F3
:101290002504000058002604000055002704000023
:1012A00079002804000057002904000057002A0490
:1012B000000062002B040000627C2C04000062002D
:1012C0002D04000065002E0400007C4F2F04000058
:1012D000397C300400006100310400003600320423
:1012E000000042003304000072003404000061007A
:1012F000350400006500360400002A0037040000B1
:1013000065003804000075003904000075003A04D7
:1013100000006B003B0400006E003C0400006D0008
:101320003D04000048003E0400006F003F04000040
:101330006E0040040000700041040000630042049D
:101340000000740043040000790044040000717040
:1013500045040000780046040000750047040000C2
:1013600079004804000077004904000077004A042F
:10137000000062004B040000627C4C04000062002C
:101380004D04000065004E0400007C6F4F04000017
:101390006700510400006500222000002E001E217D
:1013A0000000507822210000544D902100003C2D77
:1013B000922100002D3EB02100000300BB2100005F
:1013C00004003C2200007E00482200007E3D602296
:1013D0000000213D612200003D00642200003C3DF0
:1013E000652200003E3DF12300000700A030000010
:1013F0003D0021F301000200C2F401000500A2003B
:101400000000EC00B0000000DF00E4000000E1009C
:10141000F6000000EF00F7000000FD00FC000000F7
:10142000F500E3020000EB0087030000A5008F0336
:101430000000F40098030000F2009E030000E300A7
:10144000A3030000F600A9030000F400AC030000B1
:10145000E000AD030000E300B1030000E000B203D0
:101460000000E200B5030000E300B8030000F20052
:10147000BC030000E400BE030000E300C003000062
:10148000F700C1030000E600C3030000E50090215F
:1014900000007F00922100007E001A220000E80078
:1014A0001E220000F30088250000FF00023000002B
:1014B000A1000C300000A2000D300000A3009B3002
:1014C0000000DE009C300000DF00A03000003D0086
:1014D000A1300000A700A2300000B100A33000003E
:1014E000A800A4300000B200A5300000A900A6307A
:1014F0000000B300A7300000AA00A8300000B4002C
:10150000A9300000AB00AA300000B500AB300000ED
:10151000B600AC300000B6DEAD300000B700AE3033
:101520000000B7DEAF300000B800B0300000B8DE19
:10153000B1300000B900B2300000B9DEB3300000B5
:10154000BA00B4300000BADEB5300000BB00B630DF
:101550000000BBDEB7300000BC00B8300000BCDECD
:10156000B9300000BD00BA300000BDDEBB30000065
:10157000BE00BC300000BEDEBD300000BF00BE308B
:101580000000BFDEBF300000C000C0300000C0DE81
:10159000C1300000C100C2300000C1DEC330000015
:1015A000AF00C4300000C200C5300000C2DEC6304B
:1015B0000000C300C7300000C3DEC8300000C40014
:1015C000C9300000C4DECA300000C500CB300000C6
:1015D000C600CC300000C700CD300000C800CE30BF
:1015E0000000C900CF300000CA00D0300000CADEC1
:1015F000D1300000CADFD2300000CB00D330000071
:10160000CBDED4300000CBDFD5300000CC00D630AC
:101610000000CCDED7300000CCDFD8300000CD0099
:10162000D9300000CDDEDA300000CDDFDB30000045
:10163000CE00DC300000CEDEDD300000CEDFDE305C
:101640000000CF00DF300000D000E0300000D1000B
:10165000E1300000D200E2300000D300E3300000AF
:10166000AC00E4300000D400E5300000AD00E6300E
:101670000000D500E7300000AE00E8300000D600E2
:10168000E9300000D700EA300000D800EB3000005D
:10169000D900EC300000DA00ED300000DB00EF3064
:1016A0000000DC00F2300000A600F3300000DD0096
:1016B000F4300000B3DEF7300000DCDEFA3000006A
:1016C000A6DEFB300000A500FC300000B000FD30BD
:1016D0000000A400074E0000FB0086510000FC0043
:1016E00043530000FA0064FF0000A40065FF0000FF
:1016F000A50066FF0000A60067FF0000A70068FFC6
:101700000000A80069FF0000A9006AFF0000AA000D
:101710006BFF0000AB006CFF0000AC006DFF000031
:10172000AD006EFF0000AE006FFF0000AF0070FF65
:101730000000B00071FF0000B10072FF0000B200B5
:1017400073FF0000B30074FF0000B40075FF0000D9
:10175000B50076FF0000B60077FF0000B70078FF05
:101760000000B80079FF0000B9007AFF0000BA005D
:101770007BFF0000BB007CFF0000BC007DFF000081
:10178000BD007EFF0000BE007FFF0000BF0080FFA5
:101790000000C00081FF0000C10082FF0000C20005
:1017A00083FF0000C30084FF0000C40085FF000029
:1017B000C50086FF0000C60087FF0000C70088FF45
:1017C0000000C80089FF0000C9008AFF0000CA00AD
:1017D0008BFF0000CB008CFF0000CC008DFF0000D1
:1017E000CD008EFF0000CE008FFF0000CF0090FFE5
:1017F0000000D00091FF0000D10092FF0000D20055
:1018000093FF0000D30094FF0000D40095FF000078
:10181000D50096FF0000D60097FF0000D70098FF84
:101820000000D80099FF0000D9009AFF0000DA00FC
:101830009BFF0000DB009CFF0000DC009DFF000020
:10184000DD009EFF0000DE009FFF0000DF00E5FFDF
:1018500000005C00001C1F11111F00000006191879
:1018600003130C00040E1F041C000000000E1315CF
:10187000110E00001C10181705060500040A0A0ABC
:101880000A11110E0C12120C00000000001F15119D
:10189000151F00002D2D2D2D2D2D007C4D61726CFE
:1018A000696E7C002D2D2D2D2D2D000000000001D6
:1018B0000204040000001C1C0C04040402010000CB
:1018C000000000040810000000000024F4D4305090
:1018D000C38E20C2A24017828B7011127A910D81A3
:1018E0006CD90AA861E108C7586607615143061E12
:1018F0004B5D05C145A7041A411104093D980371C8
:101900003931034036DB0265339102D43054028012
:101910002E1D02632CEE01752AC501B028A001100E
:101920002781018F2564012B244B01E0223401AC77
:10193000211F018D200D01801FFC00841EED0097EA
:101940001DDF00B81CD200E61BC600201BBC0064D3
:101950001AB200B219A8000A19A0006A189900D199
:1019600017910040178B00B516840031167E00B326
:101970001579003A157300C7146F0058146A00EE09
:101980001366008813630025135E00C7125B006CAA
:1019900012570015125400C111510070114F00214F
:1019A000114B00D61049008D10470046104400022C
:1019B000104200C00F4000800F3E00420F3C000666
:1019C0000F3B00CB0E3800930E37005C0E3500271E
:1019D0000E3400F30D3200C10D3100900D30006067
:1019E0000D2E00320D2D00050D2C00D90C2B00AE54
:1019F0000C2900850C29005C0C2700350C27000EF3
:101A00000C2600E80B2400C40B2400A00B23007D4F
:101A10000B23005A0B2100390B2100180B2000F872
:101A20000A1F00D90A1E00BB0A1E009D0A1D008065
:101A30000A1D00630A1C00470A1B002C0A1B001128
:101A40000A1A00F7091A00DD091900C4091900ABC8
:101A5000091900920917007B091800630917004C47
:101A600009160036091600200916000A091500F5A6
:101A7000081500E0081400CC081400B8081400A4ED
:101A8000081400900813007D0812006B081300581A
:101A90000812004608120034081100230811001231
:101AA00008110001081100F0071000E0071000D035
:101AB000071000C0071000B0070F00A10710009129
:101AC000070E0083070F0074070F0065070E00570D
:101AD000070E0049070E003B070D002E070E0020E1
:101AE000070D0013070D0006070D00F9060C00EDA9
:101AF000060D00E0060C00D4060C00C8060C00BC65
:101B0000060C00B0060C00A4060B0099060C008D14
:101B1000060B0082060B0077060B006C060B0061BB
:101B2000060A0057060B004C060A0042060A003857
:101B3000060A002E060A0024060A001A060A0010E9
:101B400006090007060A00FD050900F4050900EB77
:101B5000050900E2050900D9050900D0050900C7FB
:101B6000050900BE050900B5050800AD050800A57A
:101B70000509009C050800940508008C05080084F0
:101B80000508007C050800740508006C0507006561
:101B90000508005D050700560508004E05070047CB
:101BA0000507004005080038050700310507002A31
:101BB000050700230507001C050600160507000F92
:101BC0000507000805060002050700FB040600F5EE
:101BD000040700EE040600E8040600E2040700DB48
:101BE000040600D5040600CF040600C9040600C39D
:101BF000040600BD040600B7040600B1040500ACED
:101C0000040600A6040600A00405009B0406009537
:101C1000040500900406008A040500850405008080
:101C20000406007A04050075040500700405006BC5
:101C300004050066040500610405005C0405005706
:101C4000040500520405004D040500480405004346
:101C50000405003E0404003A040500350405003084
:101C60000404002C04050027040400230405001EBE
:101C70000404001A04040016040500110404000DF5
:101C8000040400090405000404040000040400FC2A
:101C9000030400F8030400F4030400F0030400EC60
:101CA000030400E8030400E4030400E0030400DC90
:101CB000030400D8030400D4030400D0030400CCC0
:101CC000030400C8030300C503030024F404D9205F
:101CD0001BC40C5C0E9804C4095F0265077101F413
:101CE00005F900FB04B30048048700C103690058EC
:101CF00003550003034500BE023A0084023100533D
:101D0000022A002902250004022000E4011C00C868
:101D1000011900AF0117009801140084011300712C
:101D20000110006101100051010E0043010D003649
:101D3000010B002B010B0020010B00150109000C09
:101D400001090003010800FB000800F3000800EB94
:101D5000000700E4000600DE000600D8000600D2FE
:101D6000000600CC000500C7000500C2000500BD4C
:101D7000000400B9000400B5000400B1000400AD87
:101D8000000400A9000400A5000300A20003009FB6
:101D90000004009B000300980003009500020093DC
:101DA000000300900003008D0002008B00030088F8
:101DB0000002008600020084000300810002007F10
:101DC0000002007D0002007B000200790002007723
:101DD0000001007600020074000200720001007130
:101DE0000002006F0002006D0001006C0002006A3A
:101DF0000001006900020067000100660001006543
:101E00000001006400020062000100610001006046
:101E10000001005F0002005D0001005C0001005B4A
:101E20000001005A0001005900010058000100574C
:101E3000000100560001005500010054000100534C
:101E40000000005300010052000100510001005049
:101E50000001004F0001004E0000004E0001004D47
:101E60000001004C0001004B0000004B0001004A43
:101E7000000100490001004800000048000100473F
:101E8000000100460000004600010045000000453A
:101E90000001004400010043000000430001004233
:101EA000000000420001004100000041000100402C
:101EB0000001003F0000003F0001003E0000003E26
:101EC0000001003D0000003D0001003C0000003C1E
:101ED0000000003C0001003B0000003B0001003A14
:101EE0000000003A0001003900000039000100380C
:101EF0000000003800000038000100370000003703
:101F000000010036000000360000003600010035F8
:101F100000000035000000350001003400000034EE
:101F200000000034000100330000003300000033E3
:101F300000010032000000320000003200010031D8
:101F400000000031000000310001003000000030CE
:101F5000000000300001002F0000002F0000002FC3
:101F60000000002F0001002E0000002E0000002EB7
:101F70000001002D0000002D0000002D0000002DAC
:101F80000001002C0000002C0000002C0000002CA0
:101F90000001002B0000002B0000002B0000002B94
:101FA0000001002A0000002A0000002A0000002A88
:101FB000000100290000002900000029000000297C
:101FC000000000290001002800000028000000286F
:101FD0000000002800000028000100270000002762
:101FE0000000002700000027000000270001002655
:101FF0000000002600000026000000260000002649
:10200000000100250000002500000025000000253B
:10201000000000250000002500010024000000242D
:102020000000002400000024000000240001002320
:102030000000002300000023000000230000002314
:102040000000002300000023000100220000002205
:1020500000000022000000220000002200000022F8
:1020600000010021000000210000002100000021EB
:1020700000000021000000210000002100010020DC
:1020800000000020000000200000002000000020D0
:102090000000002000000020000000200001001FC0
:1020A0000000001F0000001F0000001F0000001FB4
:1020B0000000001F0000001F0001001E0000001EA5
:1020C0000000001E0000001E000000393000003338
:1020D00025000087190000B00F0000DB080000BDDC
:1020E000040000740200003F0100004C6F61642096
:1020F00073657474696E677300526573746F72658B
:10210000206661696C736166650053746F72652047
:1021100073657474696E6773005072656865617485
:102120002041425320636F6E66005072656865619E
:102130007420504C4120636F6E660044656C74617E
:102140002043616C6962726174696F6E00416476EC
:10215000616E6365642053657474696E6773004DC6
:1021600061696E00486F6D696E672058595A004763
:102170003238004469616720526F640044696167C6
:1021800020526F6400547A00547A005479005479D4
:10219000005478005478005261646975730052618C
:1021A0006469757300457A00457A00457900457980
:1021B000004578004578004865696768740048659F
:1021C000696768740044656C74612043616C69627E
:1021D000726174696F6E0043616C696272617465EB
:1021E000205A0043616C6962726174652059004332
:1021F000616C6962726174652058004175746F206A
:10220000686F6D650044656C746120536574746912
:102210006E6773004C6F61642073657474696E67D8
:10222000730043616C6962726174652043656E740A
:1022300065720053746F72652073657474696E679C
:1022400073004175746F2043616C696272617469D7
:102250006F6E00473333004D61696E00290A00201C
:1022600062797465733B20637263200053657474F4
:10227000696E67732053746F72656420280045454A
:1022800050524F4D206461746173697A65206572A4
:10229000726F722E0A00290A002062797465733BFE
:1022A0002063726320002073746F7265642073650D
:1022B0007474696E6773207265747269657665649B
:1022C000202800202863616C63756C617465642943
:1022D000210A0020213D2000454550524F4D20430A
:1022E0005243206D69736D61746368202D202873DB
:1022F000746F7265642920002053697A653A200062
:10230000496E6465783A2000204D61726C696E3DBB
:10231000563634290A0028454550524F4D3D004558
:102320004550524F4D2076657273696F6E206D690E
:10233000736D6174636820004D6F76696E672E2E31
:102340002E004578747275646572004175746F2053
:10235000686F6D6500473238004D6F7665205A0012
:1023600046726565205859004D6F76652059004DBD
:102370006F76652058004F6666004F6E00536F669B
:102380007420456E6473746F7073004D6F74696F61
:102390006E0044697361626C65207374657070656A
:1023A0007273004D383400426564204C6576656C6C
:1023B000696E67004175746F20686F6D6500473204
:1023C00038004D6F76652061786973004D61696EE4
:1023D0000043616E6E6F7420656E74657220737554
:1023E000626469723A2000052E2E004D61696E000C
:1023F0005072656865617420504C4120456E6400E0
:102400005072656865617420504C41005072656877
:1024100065617420504C41204265640054656D70C4
:1024200065726174757265005072656865617420CB
:1024300041425320456E64005072656865617420A6
:1024400041425320426564005072656865617420A2
:102450004142530054656D70657261747572650018
:10246000507265686561742041425300507265681E
:1024700065617420504C4100436F6F6C646F776EE0
:102480000046616E20737065656420320046616E9F
:1024900020737065656420320046616E207370653C
:1024A000656420310046616E20737065656420317B
:1024B0000042656400426564004E6F7A7A6C650084
:1024C0004E6F7A7A6C65004D61696E004261627987
:1024D00073746570205A004261627973746570206C
:1024E0005A00466C6F7700466C6F770046616E202D
:1024F000737065656420320046616E207370656597
:102500006420320046616E2073706565642031007E
:1025100046616E2073706565642031004265640019
:10252000426564004E6F7A7A6C65004E6F7A7A6C01
:1025300065005370656564005370656564004D61A6
:10254000696E004D61782054656D703A20313230EB
:10255000004D696E2054656D703A20350054426517
:10256000643A4154432031303447542D32004D6198
:10257000782054656D703A20323735004D696E20F1
:1025800054656D703A20350054303A204154432050
:1025900031303447542D32005053553A2047656E40
:1025A000657269630050726F746F636F6C3A2031AB
:1025B0002E3000426175643A2032353030303000C0
:1025C000416E7963756269632052414D50532031E9
:1025D0002E340042696C696E656172204C657665C7
:1025E0006C696E67004578747275646572733A2021
:1025F0003100687474703A2F2F6D61726C696E6669
:10260000772E6F726700414E594355424943204B24
:102610006F7373656C00323031382D30312D3230AC
:10262000006275676669782D322E302E78004D6114
:10263000726C696E005072696E74657220537461B9
:10264000747300546865726D6973746F72730042BD
:102650006F61726420496E666F005072696E7465B6
:102660007220496E666F004D61696E005072696E2E
:10267000742061626F727465640053746F702070AF
:1026800072696E74004D61696E004D323520503BA9
:10269000200A204D3234004D3234005072696E747D
:1026A0002066726F6D2053440041626F7574205034
:1026B00072696E746572004368616E676520666951
:1026C0006C616D656E7400436F6E666967757261EB
:1026D00074696F6E0054656D7065726174757265B2
:1026E000004D6F74696F6E00526573756D65207073
:1026F00072696E74004E6F205344206361726400EF
:1027000054756E650053746F70207072696E74003A
:102710005061757365207072696E7400496E666FE2
:102720002073637265656E004D6F76652058004DAD
:102730006F76652059004D6F7665205A0045787494
:102740007275646572007C3C3E5E2B3D3F2F5B5D85
:102750003B2C2A225C0043616E6E6F74206F7065A3
:102760006E20737562646972200053442063617245
:1027700064206F6B0A006F70656E526F6F74206615
:1027800061696C65640A00766F6C756D652E696EA3
:102790006974206661696C65640A00534420696E3F
:1027A0006974206661696C0A004D3234004D323321
:1027B0002025730057726974696E6720746F2066F4
:1027C000696C653A20006F70656E206661696C65A2
:1027D000642C2046696C653A20006F70656E206637
:1027E00061696C65642C2046696C653A2000466915
:1027F0006C652073656C65637465640A00205369B9
:102800007A653A200046696C65206F70656E656474
:102810003A2000667265736800646F696E67002015
:1028200066696C653A20004E6F772000454E442063
:10283000535542524F5554494E450A002220706F5D
:1028400073002220706172656E743A220053554203
:10285000524F5554494E452043414C4C20746172AF
:102860006765743A2200747279696E6720746F200C
:1028700063616C6C207375622D67636F646520669D
:10288000696C6573207769746820746F6F206D615F
:102890006E79206C6576656C732E204D4158206CE6
:1028A0006576656C2069733A310A000000210024C6
:1028B0000027002A002D0030003300010100000431
:1028C0000107010A0100002200250028002B002E2C
:1028D000003100340002010000050108010B010075
:1028E0000020002300260029002C002F00320000C9
:1028F000010000030106010901050505050705089A
:10290000080808020202020A0A0808040404040172
:102910000101010101010103030303030303030494
:102920000707070C0C0C0C0C0C0C0C020202020624
:10293000060606060606060B0B0B0B0B0B0B0B0114
:1029400002102020080810204010204080020102C0
:102950000108040201010204081020408080402088
:1029600010080402018004020180402010080402C3
:102970000108040201010204081020408001020441
:10298000081020408000000A0B02090C0D0E0807F9
:10299000030401000000000000000000000000002F
:1029A0000000000000000000000000000000000027
:1029B00000121110000000000000000000000000E4
:1029C000000000000000000000000020746F6F2075
:1029D0006C6F6E6720657874727573696F6E2070A6
:1029E000726576656E7465640A0020636F6C64209E
:1029F000657874727573696F6E2070726576656E36
:102A00007465640A000257656C636F6D6520746FAE
:102A100020414E5943554249430057656C636F6DE1
:102A20006520746F20414E59435542494300576514
:102A30006C636F6D6520746F20414E594355424958
:102A400043006275676669782D322E302E780062F9
:102A500075676669782D322E302E7800627567664C
:102A600069782D322E302E78000057656C636F6DBB
:102A70006520746F20414E594355424943005765C4
:102A80006C636F6D6520746F20414E594355424908
:102A9000430057656C636F6D6520746F20414E591C
:102AA000435542494300206275676669782D322E8E
:102AB000302E78002020506C616E6E657242756613
:102AC00066657242797465733A20002046726565C6
:102AD000204D656D6F72793A2000436F6D70696C9F
:102AE00065643A204A616E20323620323031390A2C
:102AF00000207C20417574686F723A2040627261D8
:102B00006E6473746165747465722C2040677262C0
:102B1000640A00323031382D30312D323000204CF3
:102B200061737420557064617465643A2000627545
:102B3000676669782D322E302E780A004D61726CEE
:102B4000696E0020536F66747761726520526573F9
:102B500065740A00205761746368646F672052656A
:102B60007365740A002042726F776E206F7574204F
:102B700052657365740A002045787465726E616CE5
:102B80002052657365740A00506F77657255700A3C
:102B90000073746172740A006175746F25632E6727
:102BA000006572726F722077726974696E67207443
:102BB0006F2066696C650A00446F6E6520736176EC
:102BC000696E672066696C652E0A004D32390045D2
:102BD0006E6473746F7073202563202563202563F2
:102BE00020256300205A3A0020593A0020583A0024
:102BF000656E6473746F7073206869743A200000A6
:102C000000E8420000E8420000A0430000E8C200E3
:102C100000E8C20000000020746F6F206C6F6E67C8
:102C200020657874727573696F6E20707265766551
:102C30006E7465640A0020636F6C6420657874723A
:102C40007573696F6E2070726576656E7465640A5F
:102C5000000000C8420000C8420000C84200000056
:102C6000005761726E696E673A20486F6D696E67D2
:102C70002042756D702044697669736F72203C2024
:102C8000310A000A0A0A0000A0400000A04000002B
:102C9000A04000006843000068430000A043010119
:102CA00001000000010000000100008000555555A2
:102CB000000000400033333300AAAA2A00499224BE
:102CC0000000002000C7711C0099991900D1451718
:102CD00000555515003BB113002449120011111184
:102CE00000000010000F0F0F00E3380E0043790DB5
:102CF00000CCCC0C00C3300C00E8A20B0064210B0C
:102D000000AAAA0A00703D0A009DD80900427B096A
:102D10000092240900DCD3080088880800104208CB
:102D20000000000800F0C107008787070075500702
:102D300000711C07003EEB0600A1BC06006990066E
:102D40000066660600703E06006118060017F4056E
:102D50000074D105005BB00500B2900500627205F9
:102D6000005555050078390500B81E050005050514
:102D7000004EEC040087D40400A1BD040090A70419
:102D80000049920400C17D0400EE690400C75604A6
:102D900000444404005C3204000821040041100493
:102DA00000000004003FF00300F8E0030026D20317
:102DB00000C3C30300CCB503003AA803000A9B0379
:102DC00000388E0300C08103009F750300D06903A3
:102DD00000505E03001D53030034480300913D037F
:102DE000003333030016290300381F03009715032F
:102DF00000300C0300030303000BFA020049F10248
:102E000000BAE802005CE002002DD802002DD002DA
:102E10000059C80200B0C0020031B90200DAB102A4
:102E200000AAAA0200A0A30200BC9C0200FA95021C
:102E3000005C8F0200DF88020082820200457C0273
:102E4000002776020027700200436A02007C6402B9
:102E500000D05E02003F590200C85302002364659F
:102E600066696E652044454641554C545F000062DA
:102E70006564004B6420004B6920004B70200050BB
:102E80004944204175746F74756E652066696E697A
:102E900073686564212050757420746865206C61C6
:102EA0007374204B702C204B6920616E64204B643E
:102EB00020636F6E7374616E74732066726F6D2021
:102EC00062656C6F7720696E746F20436F6E666900
:102ED0006775726174696F6E2E680A0050494420EC
:102EE0004175746F74756E65206661696C656421E7
:102EF0002074696D656F75740A004531205448452A
:102F0000524D414C2052554E415741590042454483
:102F100020544845524D414C2052554E415741593D
:102F200000546865726D616C2052756E61776179CD
:102F30000045312048656174696E67206661696C7F
:102F40006564004265642068656174696E67206627
:102F500061696C65640048656174696E67206661CB
:102F6000696C656400504944204175746F74756ED6
:102F700065206661696C6564212054656D706572B9
:102F8000617475726520746F6F20686967680A00E4
:102F9000204B643A2000204B693A2000204B703AC5
:102FA00020000A20436C61737369632050494420F8
:102FB0000A002054753A2000204B753A2000206DFD
:102FC00061783A2000206D696E3A200020643A2032
:102FD0000020626961733A200050494420417574B1
:102FE0006F74756E652073746172740A0050494481
:102FF000204175746F74756E65206661696C6564D7
:10300000212054656D706572617475726520746FEE
:103010006F20686967680A00504944204175746FE1
:1030200074756E65206661696C6564212042616417
:10303000206578747275646572206E756D62657254
:103040000A0025753A2530327500253032753A254B
:10305000303275002D2D2D005344002020202020DB
:1030600020002020202000FFFDFCFAF8F6F4F2F00A
:10307000EEECEAE9E7E5E3E1E0DEDCDAD9D7D5D446
:10308000D2D0CFCDCBCAC8C7C5C3C2C0BFBDBCBAE2
:10309000B9B7B6B4B3B2B0AFADACAAA9A8A6A5A44F
:1030A000A2A1A09E9D9C9A99989795949392908F97
:1030B0008E8D8B8A8988878684838281807F7E7DBE
:1030C0007B7A797877767574737271706F6E6D6CC8
:1030D0006B6A696867666564636261605F5E5D5CB8
:1030E0005B5A5958585756555453525150504F4E99
:1030F0004D4C4B4A4A494847464645444342424163
:10310000403F3E3E3D3C3B3B3A393838373635351B
:10311000343332323130302F2E2E2D2C2B2B2A29C6
:103120002928272726252524232322212120201F63
:103130001E1E1D1C1C1B1B1A1919181817161615F4
:103140001514131312121111100F0F0E0E0D0D0C7A
:103150000C0B0A0A090908080707060605050404F6
:103160000303020201000053746F77205A2D50723E
:103170006F6265004465706C6F79205A2D50726FD4
:1031800062650050726F62696E67206661696C6586
:10319000640A0050726F62696E67206661696C65CF
:1031A00064004D6F766520302E316D6D004D6F7669
:1031B0006520316D6D004D6F76652031306D6D008D
:1031C0004D6F7665206178697300486F74656E6431
:1031D00020746F6F20636F6C64004578747275643F
:1031E0006572004D6F7665205A004D6F76652059E7
:1031F000004D6F76652058004368616E67652066F4
:10320000696C616D656E7400556E6C6F61642066EB
:10321000696C616D656E74004C6F61642066696CE9
:10322000616D656E740050726568656174204375E8
:1032300073746F6D0050726568656174204142530C
:10324000005072656865617420504C410050726591
:103250006865617420437573746F6D004261636BC0
:1032600000486F6D6520257325732573206669728C
:103270007374002066697273740A005A005900580A
:1032800000486F6D652000496E7365727420666931
:103290006C616D656E7420616E642070726573730D
:1032A00020627574746F6E20286F72204D31303833
:1032B000290A00556E6B6E6F776E20636F6D6D61BE
:1032C0006E643A20220050726573732062757474C4
:1032D0006F6E20746F20726573756D650A00496E9C
:1032E000736572742066696C616D656E7420616EC1
:1032F0006420707265737320627574746F6E0A0057
:10330000507265737320627574746F6E20746F20D1
:1033100068656174206E6F7A7A6C650A004D36308C
:10332000303A20546F6F20636F6C6400486F74658F
:103330006E6420746F6F20636F6C640A0042696C66
:10334000696E656172204C6576656C696E672047B1
:103350007269643A0A0020496E76616C696420657E
:10336000787472756465722000202D20496E766134
:103370006C6964206578747275646572206E756D11
:1033800062657220210A001000C90210012C014060
:1033900001220170011801B0010E01F00104015079
:1033A00002FA00B002F0003003E600D003DC009027
:1033B00004D2007005C800A006BE000008B400B02A
:1033C00009AA00D00BA000600E960060118C0000CE
:1033D00015820020197800C01D6E00A0226400B084
:1033E000275A00902C500000314600E0343C001079
:1033F000383200903A2800603C1E00A03D14008046
:103400003E0A00203F0000453120544845524D41BE
:103410004C2052554E415741590042454420544892
:1034200045524D414C2052554E4157415900546828
:1034300065726D616C2052756E61776179004531FE
:10344000204572723A204D415854454D5000457206
:10345000723A204D415854454D5020424544004D4C
:10346000415854454D5020747269676765726564B0
:10347000004531204572723A204D494E54454D5019
:10348000004572723A204D494E54454D50204245F8
:1034900044004D494E54454D50207472696767652C
:1034A000726564004D383420582059205A20450058
:1034B000202F002042403A0020403A0020573A0096
:1034C000496E697469616C697A6520454550524F4F
:1034D0004D00416476616E63656420536574746960
:1034E0006E677300496E697469616C697A6520451D
:1034F0004550524F4D0046696C616D656E740054C5
:10350000656D706572617475726500537465707372
:103510002F6D6D004A65726B00416363656C657267
:103520006174696F6E0056656C6F636974790050E1
:10353000726F6265205A204F666673657400507220
:103540006F6265205A204F666673657400436F6E24
:1035500066696775726174696F6E0053746F726526
:103560002073657474696E6773004C6F61642073B7
:10357000657474696E67730050726F6265205A20BB
:103580004F66667365740050726F6265205A204FF3
:103590006666736574004F6666004F6E0042656430
:1035A000204C6576656C696E67004C6576656C20AD
:1035B000626564004732380A4732390047323900C1
:1035C0004175746F20686F6D6500473238004D6F2C
:1035D00074696F6E0053746F7265207365747469DB
:1035E0006E67730042656400426564004E6F7A7ACC
:1035F0006C65004E6F7A7A6C650046616E20737060
:103600006565640046616E20737065656400436F94
:103610006E66696775726174696F6E00416D61787D
:10362000204500416D6178204500416D617820435F
:1036300000416D6178204300416D61782042004176
:103640006D6178204200416D6178204100416D61DB
:1036500078204100412D74726176656C00412D74B3
:10366000726176656C00412D7265747261637400DD
:10367000412D7265747261637400416363656C000F
:10368000416363656C00416476616E6365642053D9
:10369000657474696E67730056652D6A65726B0098
:1036A00056652D6A65726B0056632D6A65726B00F4
:1036B00056632D6A65726B0056622D6A65726B00E7
:1036C00056622D6A65726B0056612D6A65726B00D9
:1036D00056612D6A65726B00416476616E63656444
:1036E0002053657474696E677300457374657073F5
:1036F0002F6D6D004573746570732F6D6D0043738E
:10370000746570732F6D6D004373746570732F6DE6
:103710006D004273746570732F6D6D004273746534
:1037200070732F6D6D004173746570732F6D6D0034
:103730004173746570732F6D6D00416476616E63C3
:1037400065642053657474696E6773004361703AF1
:103750000047322F47332062616420706172616DCF
:1037600065746572730A002569730025696D2025EB
:103770006973002569682025696D20256973002516
:103780006964202569682025696D202569730025F5
:10379000697920256964202569682025696D2025BF
:1037A00069730020573A0042656420636F6F6C694B
:1037B0006E672E2E2E004265642068656174696E06
:1037C000672E2E2E004D37303220542564004D36A2
:1037D000303020423020542564004D373032203BB9
:1037E0002564004D3730312054256400556E6C6FD0
:1037F00061642066696C616D656E7400556E6C6FF6
:1038000061642066696C616D656E74004D3730329D
:10381000004D373031004C6F61642066696C616D1A
:10382000656E74004D363030204230004368616E62
:1038300067652066696C616D656E74004D61696EC7
:10384000005075726765206D6F726500436F6E740E
:10385000696E756500524553554D45204F5054498A
:103860004F4E533A005052494E5420504155534503
:103870004400554E4C4F41442046494C414D454E25
:1038800054004C4F41442046494C414D454E540054
:1038900020204E6F7A7A6C653A20002000746F20E9
:1038A00073746172740066696C616D656E74206317
:1038B00068616E6765005761697420666F720066A3
:1038C000696C616D656E7420756E6C6F6164005714
:1038D00061697420666F7200506C65617365207752
:1038E0006169742E2E2E004E6F7A7A6C65206865A1
:1038F0006174696E6700746F2068656174206E6F13
:103900007A7A6C6500507265737320627574746F97
:103910006E00746F20636F6E74696E756500616E02
:103920006420707265737320627574746F6E0049E1
:103930006E736572742066696C616D656E74006685
:10394000696C616D656E74206C6F616400576169AC
:103950007420666F7200746F20726573756D6520D8
:103960007072696E7400507265737320627574743E
:103970006F6E00746F20726573756D652E2E2E004C
:103980005761697420666F72207072696E74006688
:10399000696C616D656E7420707572676500436C4B
:1039A00069636B20746F2066696E697368000045F7
:1039B0007874727564656420746F74616C3A200069
:1039C000256C642E25696D00004C6F6E67657374FD
:1039D000206A6F622074696D653A200000546F742C
:1039E000616C207072696E742074696D653A200094
:1039F000436F6D706C657465643A20005072696E37
:103A00007420436F756E743A2000000000000000BF
:103A100000000000A043486F6D696E672066616911
:103A20006C6564006F70656E00545249474745529B
:103A30004544003A20007A5F6D6178007A5F6D69D5
:103A40006E00795F6D617800785F6D617800526516
:103A5000706F7274696E6720656E6473746F702026
:103A60007374617475730A0020433A0020423A006F
:103A700020436F756E7420413A0020453A00205A69
:103A80003A0020593A00583A006F70656E2066611E
:103A9000696C65642C2046696C653A200046696E45
:103AA0006973686564210A00206F662000205A004F
:103AB000205900205800476F696E6720746F3A00E4
:103AC0002C200050756C6C696E6720706F696E7485
:103AD00020746F77617264732063656E7465723AE7
:103AE00000436C6F636B776973650A00436F756E93
:103AF0007465722D0020446972656374696F6E3A53
:103B00002000202020616E676C653A2000537461AC
:103B10007274696E67207261646975733A2000502F
:103B20006F736974696F6E696E6720746865207061
:103B3000726F62652E2E2E0A003F4E756D626572A1
:103B4000206F66206C65677320696E206D6F7665E7
:103B50006D656E74206E6F7420706C617573696230
:103B60006C652028302D3135292E0A003F20285839
:103B70002C5929206F7574206F6620626F756E64F2
:103B8000732E0A003F53616D706C652073697A650E
:103B9000206E6F7420706C61757369626C6520288B
:103BA000342D3530292E0A004D3438205A2D5072CC
:103BB0006F6265205265706561746162696C6974D9
:103BC0007920546573740A003F2856296572626F24
:103BD0007365206C6576656C20697320696D706C07
:103BE00061757369626C652028302D34292E0A00B6
:103BF00048617264636F6465642044656661756CD6
:103C0000742053657474696E6773204C6F616465CA
:103C1000640A00B80B0000B80B0000B80B0000B835
:103C20000B00000000C8420000C8420000C842006B
:103C300000C8420000A0420000A0420000A04200D4
:103C400000C0423A0A0020204D3630332000205573
:103C5000004C0046696C616D656E74206C6F616428
:103C60002F756E6C6F6164206C656E677468733A53
:103C70000A0020204D383531205A005A2D50726FDD
:103C80006265204F66667365740020440020490019
:103C900020204D33303420500020440020490020A3
:103CA000204D3330312050005049442073657474E6
:103CB000696E67733A0A00204600204200204800DF
:103CC00020204D3134352053004D61746572696197
:103CD0006C2068656174757020706172616D6574C7
:103CE0006572733A0A00205A0020590020580020BB
:103CF000420020530020480020520020204D36363C
:103D000035204C0044656C74612073657474696E71
:103D100067733A204C3C646961676F6E616C5F72D7
:103D20006F643E20523C7261646975733E20483C6A
:103D30006865696768743E20533C7365676D656E9E
:103D400074735F7065725F733E20423C63616C699F
:103D500062726174696F6E207261646975733E206E
:103D600058595A3C746F77657220616E676C652094
:103D7000636F7272656374696F6E733E0A00205AD6
:103D80000020590020204D363636205800456E64FC
:103D900073746F702061646A7573746D656E743AC4
:103DA0000A00204A002020473239205720490020AD
:103DB000204D3432302053004175746F20426564C9
:103DC000204C6576656C696E673A0A0020450020D4
:103DD0005A00205900205800205400205300202071
:103DE0004D32303520420020453C6D61785F655F83
:103DF0006A65726B3E0020583C6D61785F785F6A3F
:103E000065726B3E20593C6D61785F795F6A6572BF
:103E10006B3E205A3C6D61785F7A5F6A65726B3EDB
:103E200000416476616E6365643A20423C6D696E60
:103E30005F7365676D656E745F74696D655F7573DB
:103E40003E20533C6D696E5F6665656472617465A2
:103E50003E20543C6D696E5F74726176656C5F667E
:103E6000656564726174653E002054002052002034
:103E7000204D323034205000416363656C657261BF
:103E800074696F6E2028756E6974732F7332293AC6
:103E900020503C7072696E745F616363656C3E2094
:103EA000523C726574726163745F616363656C3EFA
:103EB00020543C74726176656C5F616363656C3E2F
:103EC0000A00204500205A0020590020204D3230A1
:103ED000312058004D6178696D756D2041636365CF
:103EE0006C65726174696F6E2028756E6974732FCA
:103EF0007332293A0A00204500205A002059002038
:103F0000204D3230332058004D6178696D756D2039
:103F10006665656472617465732028756E69747373
:103F20002F73293A0A00204500205A00205900200A
:103F3000204D3932205800537465707320706572BB
:103F400020756E69743A0A0020204D3230302044CA
:103F5000300A0020204D3230302044002044697364
:103F600061626C65640A0046696C616D656E7420FF
:103F700073657474696E67733A0020204D3134396B
:103F80002043203B20556E69747320696E20436581
:103F90006C736975730A0020286D6D290020204715
:103FA0003231202020203B20556E69747320696EC9
:103FB000206D6D002CFFFFFFFFFFFF0001010101DD
:103FC00001016265640A002C2073797374656D20A9
:103FD00073746F7070656421204865617465725FE9
:103FE00049443A20004265642068656174696E67DF
:103FF000206661696C65640048656174696E67205C
:104000006661696C65640045312048656174696E5C
:1040100067206661696C65640048656174696E67F4
:10402000206661696C656400656E717565756569AA
:104030006E6720220000FB00EB0011241FBECFEFB3
:10404000D1E2DEBFCDBF00E00CBF13E0A0E0B2E0E4
:10405000E4E7FDE902E00BBF02C007900D92A63D28
:10406000B107D9F726E1A6EDB3E001C01D92AB364A
:10407000B207E1F710E2CCE1D0E200E006C0219700
:104080000109802FFE010F941E4ECB31D10780E035
:104090000807A9F70F94B1370D94A94E0C940000AE
:1040A0002F923F924F925F926F927F928F929F9248
:1040B000AF92BF92CF92DF92EF92FF920F931F9336
:1040C000CF93DF93CDB7DEB7A3970FB6F894DEBFDB
:1040D0000FBECDBF0091810E20E6029F800111240A
:1040E0000F5F124F80918B0C80FF05C00E944860CB
:1040F000C8010E94C06110920504109204048FE36D
:104100008093060410920304109202041092FD039F
:104110001092FE031092FF0310920004C8018C015C
:10412000DC012C9101962032D1F32E34D9F4119672
:104130008C9190ED980F9A3020F08D3211F08B32E7
:1041400089F4F80132969F012F5F3F4F80818053A1
:104150008A3010F4F901F7CF8F013196D8018C9194
:104160008032D1F31093840F0093830F7801BFEF57
:10417000EB1AFB0AF80170806AE270E0C7010F9445
:10418000664E009731F0FC01319780818032E1F377
:104190001182FDE47F1631F024E5721619F037E440
:1041A0007312F0C0F70180814FEFE41AF40A8032F5
:1041B000C9F380538A3008F0E5C07092060480E0AD
:1041C00090E06AE03196DF0111972C91022E000CED
:1041D000330B20533109689FA001699F500D1124B2
:1041E000C901840F951F208120532A3058F39093E2
:1041F0000304809302049F01D9012F5F3F4F4C912C
:104200004032D1F3EDE47E121AC08E31910591F067
:104210003CF48731910571F08C31910581F40AC02D
:104220008537910564F08737910524F0803AF3E0F3
:104230009F0729F4B0930504A0930404A3C0C12CE4
:10424000D12C760140E050E0812C912C54018394D4
:10425000FD0131966C9161110DC05093050440939E
:104260000404C092FD03D092FE03E092FF03F0929B
:10427000000488C06132E9F42DE472121AC0803261
:104280009105B9F4C092FD03D092FE03E092FF03C2
:10429000F0920004F0930504E093040463E270E0FC
:1042A000CF010F94664E009709F46CC0DC011C929C
:1042B00069C061546A3108F042C09F01F901708100
:1042C0002F5F3F4F7032D1F320ED270F2A30E8F0F7
:1042D0007E3211F421810CC07D3211F07B3259F411
:1042E000218130ED320F3A3080F02E3221F42281DC
:1042F00020532A3050F04115510511F00C9415331C
:10430000AF01415051090C9415339F01A62FB0E025
:104310001401250104C0220C331C441C551C6A9551
:10432000D2F7C228D328E428F5282115310511F049
:10433000201B01C020E0AA52BC4F2C9304C04115A1
:10434000510509F4AD01208121542A3110F4DF0117
:104350007FCF9F01F901D9016D916623C1F370ED03
:10436000760F7A3010F49D01F5CF73ED760F723031
:10437000D0F36B32C1F3F9012F5F3F4F60816032A0
:10438000D1F3E5CF41E04093810F809106048D3455
:1043900009F443C2843511F40C94F332873411F0DC
:1043A0000C940E3320910204309103042C3131051A
:1043B00009F4B1C094F42430310534F422303105CD
:1043C000DCF537FF2DC025C22430310509F443C088
:1043D0002B31310509F47EC01CC22A32310509F4A3
:1043E00085C174F42E31310509F4AEC00CF498C0C7
:1043F0002132310509F00DC20E9479380C94103336
:104400002B35310509F4FEC02C35310509F4FEC009
:104410002A35310509F0FDC1109201040C941033C6
:1044200080915F02882311F40C9410330E9408EFEE
:104430000E943FCF0C94103380915F02882311F4C7
:104440000C94103381E02230310509F080E00F94A4
:10445000400D0C94103380E50E94B4EF882329F0BE
:104460000F9472156B017C0103C0C12CD12C760115
:1044700083E50E94B4EF882361F00E9488EE20E07B
:1044800030E04AE754E40F94EE460F941E4C6B0163
:104490007C010E94D1C88091860F811105C060E027
:1044A00087E792E00E94F3720E9473B2C60ED71E95
:1044B000E81EF91E0E9473B2DC01CB018C199D0924
:1044C000AE09BF09B7FD02C00C94103380E00E9412
:1044D0007462F0CF0E94EDE981110C9410331982BF
:1044E0001A821B821C821D821E821F82188680E017
:1044F00090E0A0EAB1E489879A87AB87BC8760E047
:1045000070E080E50F945F15BE016F5F7F4F0E94E2
:10451000A09B0C94103380E00E9461520C941033E5
:104520000E94EDE981110C94103380917D0688235F
:1045300011F40C94193360E08FE40E944D52811104
:104540000C9410330C94193320E030E0A9016091F1
:104550006D0670916E0680916F06909170060F94B3
:10456000D54AAB01BC0188E50E9468DB6C8F7D8F6A
:104570008E8F9F8F20E030E0A901609171067091CD
:10458000720680917306909174060F94D54AAB0120
:10459000BC0189E50E9468DB6B017C0169837A8339
:1045A0008B839C836C8D7D8D8E8D9F8D9B01AC014B
:1045B0000F94EE464B015C01A7019601C701B601BD
:1045C0000F94EE469B01AC01C501B4010F94D54A8E
:1045D0006B017C0120E030E442E556E40F9489460B
:1045E000181614F40C94103320E034E64FE156E42E
:1045F000C701B6010F948946181614F40C941033B1
:104600000C941C33409301040C94103384E6282E40
:1046100082E0382E93EEE92E9EE0F92E2DE6C22E92
:1046200026E0D22E00E010E0F10181911F010E94EE
:10463000B4EF882309F446C00E9488EE2B013C01A8
:10464000133049F0D7012D913D914D915C910F941C
:10465000D44A2B013C01F6012081318142815381F2
:10466000C301B2010F94D44A4B015C012DEB37E337
:1046700046E855EB0F94494D87FD0AC02DEB37E313
:1046800046E855E3C501B4010F9489461816D4F4E1
:10469000133051F44092790650927A0660927B066C
:1046A00070927C0601E00EC0A5019401D7016D91C6
:1046B0007D918D919C910F94D54AF7016083718310
:1046C000828393831F5FF4E0EF0EF11C24E0C20E9F
:1046D000D11C143009F0A8CF002321F089E796E01F
:1046E0000E9450E80F94161F0C94103380915F02C3
:1046F000882311F40C94103389E40E94B4EFE82E5F
:10470000882321F00E94A352F82E01C0F12C8AE4E4
:104710000E94B4EF082F882321F00E94A352182F83
:1047200001C010E0EE2019F038E03F1520F0002322
:1047300041F0193030F082E992E00E9404600C945C
:1047400010330E94BB50EE20F1F02091981430916C
:1047500099144F2D4203B001439F700D1124809195
:10476000B1059091B205680F791F072E000C880BD8
:10477000990B0F948F4660938D0E70938E0E8093DD
:104780008F0E9093900E0023E9F020919A143091AF
:104790009B141203B001139F700D11248091B30577
:1047A0009091B405680F791F072E000C880B990BA8
:1047B0000F948F466093910E7093920E8093930E98
:1047C0009093940E60E080E50E944D5240E050E0EE
:1047D000BA0186E40E9468DB6B017C0120E030E0D6
:1047E000A9010F94494D181684F420E030E040E709
:1047F00052E4C701B6010F94B14B60934702709326
:1048000048028093490290934A020E943FCF0C9441
:1048100010330E94EFE80C941033809102049091C1
:1048200003048737910511F40C942B2C0CF0E4C091
:104830008D34910509F449C40CF068C08A319105A2
:1048400009F4E9C29CF58431910509F46FC27CF446
:104850008131910509F45BC22CF4029708F4DFC1A1
:104860000C94F032429709F48CC60C94F0328731E4
:10487000910509F485C28CF48531910509F47CC257
:10488000469711F00C94F0320E9450B38091951429
:10489000877F809395140C9410338831910509F427
:1048A00082C2499709F4ACC20C94F0328F31910561
:1048B00009F4C0C384F48C31910509F40DC30CF4E0
:1048C000B8C28D31910511F40C9410334E9709F450
:1048D0000DC30C94F0328033910509F4EEC34CF40F
:1048E0008032910509F460C38A9709F4C3C30C941C
:1048F000F0328B34910509F4E4C38C34910511F046
:104900000C94F0320E948B9B0C9410338B369105E3
:1049100009F407C6BCF58435910509F432C6CCF418
:104920008135910509F414C634F48E34910509F4E7
:10493000D0C30C94F0328235910509F41EC683353C
:10494000910511F00C94F03281E08093F8030C94FF
:1049500010338836910509F471C454F485359105F6
:1049600009F442C68C35910509F459C60C94F0320D
:104970008936910509F482C58A36910509F4B9C5CD
:104980000C94F0328037910509F433C584F48D36E8
:10499000910509F477C40CF426C58E36910509F407
:1049A000CEC48F36910509F4DDC40C94F032833700
:1049B000910509F4C1C67CF48137910509F41DC540
:1049C0008237910511F00C94F0320E94D1C80F94F7
:1049D000161F0C9410338537910509F407C78637E5
:1049E000910511F00C94F03200910404109105042B
:1049F00083E0F12C40E008C78033A1E09A0711F46E
:104A00000C940C300CF079C08C3C910511F40C9492
:104A1000272D8CF58139910509F42FC784F4893746
:104A2000910509F423C70CF419C78D37910509F4D2
:104A30008BC58C38910509F403C50C94F032883C81
:104A4000910509F475C76CF48B39910509F429C5F2
:104A50008E3B910511F00C94F0320F949E0A0C9449
:104A60001033893C910509F4B0C78B3C910509F4DA
:104A7000CFC70C94F032823E910511F40C94202F94
:104A8000CCF4833D910511F40C94072E3CF48D3C3D
:104A9000910511F40C94582D0C94F0328C3D910535
:104AA00011F40C94BD2E8D3D910511F40C94CA2E79
:104AB0000C94F0328D32E1E09E0711F40C948C2FAF
:104AC0006CF4823221E0920711F40C946C2F8C323A
:104AD000914011F40C94772F0C94F0328E3241E017
:104AE000940711F40C947F308F32914011F00C94A4
:104AF000F0320E947FDB0C941033883FB1E09B07BB
:104B000011F40C944F310CF049C0843AF1E09F0746
:104B100011F40C94D130FCF4813931E0930711F495
:104B20000C94C3304CF48039914011F00C94F03265
:104B30000E94D1C80C9410338239B1E09B0711F464
:104B40000C94C9308A39914011F00C94F0320E94D3
:104B50009F650C941033853FF1E09F0711F40C948E
:104B60003D317CF4853A31E0930711F40C94D43054
:104B7000843F914011F00C94F0320E943C870C94D9
:104B80001033863FA1E09A0711F40C944031873F1F
:104B9000914011F40C9443310C94F0328A39E2E0E4
:104BA0009E0711F40C94E32DD4F4883522E092078B
:104BB00011F40C94A4313CF48C30924011F40C9418
:104BC0005F310C94F0328B35A2E09A0711F40C940B
:104BD000A7318939924009F47BC70C94F0328335B0
:104BE000E3E09E0711F40C9467316CF48D3B22E0F6
:104BF000920711F40C9420328E3B924011F40C94E5
:104C000023320C94F032803A43E0940709F402C254
:104C1000873E934011F40C94E2320C94F032A09051
:104C20000404B090050480E50E94B4EF882359F095
:104C30000F9472156B017C0111E0672B682B692BB7
:104C400031F410E004C010E0C12CD12C760183E5D2
:104C50000E94B4EF882311F40C94A0330E9488EED4
:104C600020E030E04AE754E40F94EE460F941E4CE7
:104C70006B017C0111110BC0672B682B692B39F478
:104C8000A114B10421F0F5018081811102C010E06E
:104C900001C011E00E94D1C8112329F061E0C501D3
:104CA0000E942F7305C060E081EB92E00E94F372D6
:104CB00083E08093810F81E08093800FC114D10441
:104CC000E104F104B1F00E9473B2C60ED71EE81ED3
:104CD000F91E0E9473B2DC01CB018C199D09AE094B
:104CE000BF09B7FF0EC08091800F81110C94A533CE
:104CF00008C08091800F882321F080E00E947462B8
:104D0000F8CF0E9457731092800F0C94103360E01C
:104D100084EC92E00E94F3725F988A988091080177
:104D200081708093060112980C9410338CED92E000
:104D30000E9404601092610682EF92E10E9467AACD
:104D40008BE1E2EFF2E1DE01119601900D928A957E
:104D5000E1F740E050E0BE016F5F7F4F80E090E000
:104D60000E94D2B4CE0101960E9475AD8DEC92E006
:104D70000E9404600C9410330E94C4B30C9410334E
:104D80008091040490910504FC012081222329F0E4
:104D9000203209F410823196F8CF40E061E00E94A1
:104DA0006DB60C9410338091F3058823E9F080E010
:104DB00090E0A6E1B3E488A399A3AAA3BBA31C8EA9
:104DC0001D8E1E8E1F8E19821A821B821C8220E06D
:104DD000AE01405E5F4FBE01645E7F4FCE01019623
:104DE0000E94B3F50C9410330F94320D882321F0F8
:104DF0000E9460B30E949FE50E9457730C94103389
:104E00008091951482FF03C08B7F809395140F943B
:104E10009C140C9410338091951483FD02C00C9463
:104E2000103383E50E94B4EF81110C94AA330C94E3
:104E3000103383E40E94BFEE882319F187EF92E0DC
:104E40000E94046080919C12882391F0BE016F5FE4
:104E50007F4F89E992E10E9409AD8E010F5F1F4FDC
:104E6000D8018D918D01882339F00E94F35FF8CF2E
:104E70008DEE92E00E9404608AE00E94F35F0C9441
:104E800010338091951482FF21C086E093E00E9448
:104E90000460609191147091921480919314909198
:104EA00094144AE00E949D608FE20E94F35F60913B
:104EB0008D1470918E1480918F14909190144AE00B
:104EC0000E949D600E94BC610C94103388E193E0C5
:104ED0000E9404600C94103340E060E08091040470
:104EE000909105040E946DB60C9410338091951436
:104EF00083FD02C00C9410330E94D8E86091040432
:104F0000709105048091951483FD02C00C941033B8
:104F1000CE014C960F94FC258C01009711F40C9453
:104F200010336C8D7D8D19821C8222E0AC01CE0184
:104F300001960E9460AF811102C0F12C14C0CE0115
:104F400001960F946A258823C1F361E0CE01019692
:104F50000E94EEAC009789F325EEFC0120831C82B1
:104F60000E9492A7F82ECE0101960E9475ADB8015D
:104F7000FF2089F081E493E00E9412608AE00E94A1
:104F8000F35F109291141092921410929314109255
:104F900094140C94103389E293E00E9412608EE224
:104FA0000E94F35F0C9410338091951482FD0E944F
:104FB000D1C88091951483FD02C00C94103360E039
:104FC00080E50E944D52182F482F61E08091040423
:104FD000909105040E946DB683E50E94B4EF88238A
:104FE00081F00E9467EEAB01BC0140939114509395
:104FF0009214609393147093941489E992E10E943F
:10500000D1A90E9460B311110C9410330E949FE546
:105010000C94103320910404309105049091951460
:1050200092609093951440E060E0C9010E946DB6D3
:105030000C9410330E943C9B6C8F7D8F8E8F9F8FC2
:10504000BE016F5F7F4FCE014C960F94560C60E00F
:10505000CE0101960E942F730E944860BE016F5FCF
:105060007F4F8FE493E00E9412608AE00E94F35F1A
:105070000C94103383E50E94B4EF882311F40C9450
:1050800010330E9477EEF82E6DE070E080E50E940C
:10509000A7528C0197FF02C00C941033E82E60E0F9
:1050A00089E40E944D5281110C94BB33802F0F94E0
:1050B00049378111E2C60C94BB330F9407280C9436
:1050C00010330E949FE50C9410330E94FBE50C9472
:1050D000103360E070E083E50E94A7528E349105A2
:1050E00021F40E946BE60C9410338AEB93E00E944B
:1050F000046081EB93E00E9404606091EC0C70917D
:10510000ED0C80E090E04AE00E949D6084EA93E02C
:105110000E9404606091EE0C7091EF0C80E090E0D2
:105120004AE00E949D6089E993E00E9404606091DA
:10513000EC0C7091ED0C8091EE0C9091EF0C681BD3
:10514000790B8091DE0E815021E030E0823010F04A
:1051500020E030E0621B730B80E090E04AE00E94A8
:105160009D608AE00E94F35F81E993E00E94046001
:105170008091F00C9091F10CA091F20CB091F30C95
:105180008C8F9D8FAE8FBF8FBE016F5F7F4FCE0123
:105190004C960F94560C84E893E00E9404608E01B4
:1051A0000F5F1F4F7801D7018D917D01882319F082
:1051B0000E94F35FF8CF8091F40C9091F50CA091D0
:1051C000F60CB091F70C8C8F9D8FAE8FBF8FBE0108
:1051D0006F5F7F4FCE014C960F94560C84E793E09F
:1051E0000E940460F80181918F01882319F00E94C8
:1051F000F35FF8CF8AE00E94F35F8CE693E00E94B1
:1052000004608CE593E00E94046020E030E04AE70F
:1052100054E46091F80C7091F90C8091FA0C909123
:10522000FB0C0F94B14B42E00E943C618DE60E9462
:10523000F35F8AE00E94F35F0C94103380918B0C33
:1052400083FF02C00C9410330E94C0EF87FF02C09E
:105250000C94103383E50E94B4EF882379F00E9408
:1052600088EE0F94194C8B01CB010E9452FE06353B
:10527000110524F40E94FBE50E9457730F94AA3D88
:105280000C94103380918B0C83FF02C00C9410336C
:105290000E94C0EFF82E87FF02C00C94103383E504
:1052A0000E94B4EF082F811106C082E50E94B4EF7E
:1052B000182F8823C1F10E9488EE0F94194CCB015E
:1052C0000E9452FE0E9488EE20E030E04AEA52E45A
:1052D0000F948946181614F40C94D4330E94FBE5FD
:1052E0000E9457736091060F7091070F072E000CF4
:1052F000880B990B0F948F464B015C014090C506BB
:105300005090C6066090C7067090C806A30192012F
:105310000F94494D181614F40C94E733002311F43C
:105320000C94D83311E00F94AA3D112311F40C947E
:105330001033602F8F2D0E9439F90C9410338EE4B6
:105340000E94B4EF882311F40C9410330E9467EE8E
:105350006093890470938A0480938B0490938C04E7
:105360000C94103383E50E94BFEE882331F060E097
:1053700083E50E94AF5080938B0C0E9448608AEEB8
:1053800093E00E94046080918B0C882349F100EE29
:10539000E02E03E0F02E00E010E020E080918B0C86
:1053A00090E0002E02C0959587950A94E2F780FF61
:1053B0000EC0DD24D394D20E222319F08CE20E9479
:1053C000F35FF701859194910E9404602D2D0F5F8A
:1053D0001F4FF2E0EF0EF11C05301105F9F64CCD30
:1053E0008CED93E047CD1092800F109219020C942F
:1053F000103380E090E00E94306283E50E94B4EFB9
:10540000882371F00E9477EE8093000290E0CD97A0
:1054100014F40C9410338CE3809300020C9410333A
:105420000E9448604091000250E060E070E081EF2F
:1054300093E00E9408618AE00E94F35F0C941033AD
:1054400080918B0C83FF02C00C94103383E50E9483
:10545000B4EF882311F40C9410330E9488EE0F945B
:10546000194C6936710514F069E670E07093FA0E14
:105470006093F90E0E94B4FD0C9410330E94C0EFAB
:10548000182F87FD0AC088EF93E00E940460812FE7
:105490000E94C8F88AE00E94F35F1092810F0C947A
:1054A000153583E50E94B4EF882311F40C94103372
:1054B0000E9477EE182F90E0CD970CF01CE310932C
:1054C000F4030E9473B26B017C01212F30E0A8EE3F
:1054D000B3E00F94C54AC60ED71EE81EF91EC0924F
:1054E000F003D092F103E092F203F092F3030C94F4
:1054F000103360E080E50E94AF5081110C941033AE
:105500006FEF70E083E50F945F158F3F910519F001
:1055100010F08FEF90E08093B2068093F70E0C941A
:10552000103360E080E50E94AF50823010F00C94A0
:10553000103390E0FC01EE54F94F1082FC01E95069
:10554000F14F10820C9410330F949C140C94103370
:105550000E9462FE0E94FBE50E949CCA0E94D065E8
:1055600068EE73E080E090E00E94925F60E08BEF75
:1055700093E00E94F3720C9410331092F8030C9491
:10558000103383E50E94B4EF8823A1F00E9488EED7
:1055900020E030E04AE754E40F94EE460F941E4CAE
:1055A00060930102709302028093030290930402BD
:1055B0000C94103388E50E94BFEE81110C94EA33FD
:1055C00089E50E94BFEE81110C94EA338AE50E94BE
:1055D000BFEE81110C94EA3385E40E94BFEE811185
:1055E0000C94EA330C941A3483E50E94BFEE8823AE
:1055F00011F40C9410330E9488EE20E030E04AE76A
:1056000054E40F94EE460F941E4C6093F90370938C
:10561000FA038093FB039093FC030C9410330E94D5
:10562000C0EF87FF01C0FCC7B4E6CB2EB2E0DB2E93
:105630001CE8E12E1CE0F12E10E0D6018D916D01E9
:105640000E94BFEE882309F46DC0133009F063C0D7
:105650000E9488EE4B015C0120E030E040EA51E41A
:105660000F94894687FF4EC0A50194016091AC0C50
:105670007091AD0C8091AE0C9091AF0C0F94B14B2A
:105680002B013C019B01AC0160919606709197063D
:1056900080919806909199060F94EE466093960635
:1056A000709397068093980690939906A3019201B0
:1056B0006091BC0C7091BD0C8091BE0C9091BF0CA0
:1056C0000F94EE466093BC0C7093BD0C8093BE0C9F
:1056D0009093BF0C6091A6067091A7068091A806D2
:1056E0009091A9060F948D46A30192010F94EE4666
:1056F0000F941E4C6093A6067093A7068093A8068D
:105700009093A9068092AC0C9092AD0CA092AE0C36
:10571000B092AF0C07C00E9488EEF701648B758BC6
:10572000868B978B1F5FF4E0EF0EF11C143009F0AD
:1057300084CF0E942DE874C78CEF94E00E9404602F
:1057400060E08CEE94E00F944E1261E085EE94E000
:105750000F944E1261E08AED94E00F944E1261E0D6
:105760008AEC94E00F944E1260E081EC94E00F9488
:105770004E1261E087EB94E00F944E1261E08DEAE7
:1057800094E00F944E1261E085EA94E00F944E127B
:1057900061E087E994E00F944E1260E089E894E0BC
:1057A0000F944E1260E08AE794E00F944E1260E08E
:1057B0008CE694E00F944E1260E086E594E00F943E
:1057C0004E1260E085E494E00F944E1260E080E3B6
:1057D00094E00F944E1261E08DE194E00F944E122C
:1057E00060E080E194E00F944E121AC760E080916F
:1057F0000404909105040E942F7312C7D8019C9154
:10580000292F2B7F213419F08150C1F717C0119631
:105810002C912133C9F7913421F0953421F441E0E2
:1058200002C0FF24F39498012E5F3F4F89012F5F40
:105830003F4FF80190819032C9F3E6CF41110E94A9
:105840004860FF2021F08EEC95E00E940460C801C2
:105850000E94C061E5C60F94EE20E2C681E080930D
:10586000FD0C8093FC0C0F940C21DAC61092FD0CF9
:105870001092FC0C0F940C21D3C660E070E083E51D
:105880000E94A7528C011127023011053CF00E94A2
:10589000236082ED95E00E940460C2C688E40E9405
:1058A000B4EF8823A9F00E94A3528A3A91053CF0F4
:1058B0008530F1E09F072CF084E091E002C08AEA95
:1058C00090E0F801EE0FFF1FEF5FF04F91838083B0
:1058D00086E40E94B4EF882381F00E94A35297FDD2
:1058E00007C08F3F910529F024F08FEF90E001C0B1
:1058F00080E0F801EC55FB4E808382E40E94B4EF17
:10590000882309F48DC60E94A3528530910534F096
:105910008A3691052CF089E690E002C085E090E09F
:10592000F801EE0FFF1FEA55FB4E9183808378C686
:105930000E94C0EF182F87FD73C684E40E94BFEE5B
:10594000882309F43FC00E9488EE6B017C0101E0CE
:1059500020E030E0A9010F948946811101C000E0E8
:105960000093AF0E20E030E0A901C701B6010F940B
:105970008946882339F10E9488EE24E01202F00162
:105980001124EC54F14F608371838283938320E070
:1059900030E0A9016091B40E7091B50E8091B60E01
:1059A0009091B70E0F94894681110CC080E090E071
:1059B000A0EEBFE38093B40E9093B50EA093B60E05
:1059C000B093B70E0E940DC82BC60E94C0EF87FD92
:1059D00027C664E6E62E62E0F62E0CE81CE0D7014E
:1059E0008D917D010E94BFEE882349F00E9488EED0
:1059F0000F941E4CF80160837183828393830C5F44
:105A00001F4FFCE00C391F0751F70E94E6E708C65C
:105A10000E94C0EF87FD04C654E6E52E52E0F52E45
:105A20000CE81CE0D7018D917D010E94BFEE882318
:105A300039F00E9488EEF80164A375A386A397A3AA
:105A40000C5F1F4FFCE00C391F0761F7E9C580911F
:105A5000FE0387FDF2C68091FF038E7009F0EDC64C
:105A60004091C00C5091C10C6091C20C7091C30C5C
:105A70008AEF95E00E94AD614091C40C5091C50C35
:105A80006091C60C7091C70C87EF95E00E94AD61E4
:105A90004091C80C5091C90C6091CA0C7091CB0C0C
:105AA00084EF95E00E94AD618AE00E94F35FB8C583
:105AB0008091FD03827109F006C78091FF038C7805
:105AC00009F001C780910004837009F0FCC6A8C5E5
:105AD00088E40E94BFEE882351F00E9488EE609314
:105AE000850E7093860E8093870E9093880E8CE4BB
:105AF0000E94BFEE882351F00E9488EE6093491007
:105B000070934A1080934B1090934C1082E50E9442
:105B1000BFEE882351F00E9488EE60934D10709381
:105B20004E1080934F109093501083E50E94BFEE6B
:105B3000882351F00E9488EE6093890E70938A0E3C
:105B400080938B0E90938C0E82E40E94BFEE88238C
:105B500051F00E9488EE6093AA147093AB14809366
:105B6000AC149093AD1488E50E94BFEE882351F0E9
:105B70000E9488EE609351107093521080935310DE
:105B80009093541089E50E94BFEE882351F00E9443
:105B900088EE609355107093561080935710909331
:105BA00058108AE50E94BFEE882351F00E9488EECB
:105BB0006093591070935A1080935B1090935C100F
:105BC0000F9437232DC544E6E42E42E0F42E03EA79
:105BD0001EE0D7018D917D010E94BFEE882381F0E8
:105BE0000E9488EE4B015C0120E030E0A9010F9497
:105BF000894618162CF0F80180829182A282B38225
:105C00000C5F1F4FFEE00F3A1F0719F709C50E94EE
:105C100048608CE596E00E94046083E50E94BFEE38
:105C2000882321F00E94C55080931A0280911A02A5
:105C3000882319F08DEA9AE002C089EA9AE00E946E
:105C4000046084E596E00E9404602091E30E3091A8
:105C5000E40E4091E50E5091E60E6091290270919C
:105C60002A0280912B0290912C020F94D54AAB010D
:105C7000BC0182E596E00E94AD612091E70E309173
:105C8000E80E4091E90E5091EA0E60912D0270915C
:105C90002E0280912F02909130020F94D54AAB01D1
:105CA000BC018FE496E00E94AD612091EB0E309133
:105CB000EC0E4091ED0E5091EE0E6091310270911C
:105CC000320280913302909134020F94D54AAB0195
:105CD000BC018CE496E00E94AD6184E496E00E94F1
:105CE00004602091E30E3091E40E4091E50E509156
:105CF000E60E60911D0270911E0280911F0290912C
:105D000020020F94D54AAB01BC0182E496E00E94C8
:105D1000AD612091E70E3091E80E4091E90E50916F
:105D2000EA0E6091210270912202809123029091EB
:105D300024020F94D54AAB01BC018FE396E00E9488
:105D4000AD612091EB0E3091EC0E4091ED0E509133
:105D5000EE0E6091250270912602809127029091AB
:105D600028020F94D54AAB01BC018CE396E00E9457
:105D7000AD618AE00E94F35F53C483E50E94B4EFF3
:105D8000882309F44DC40E94A35290931C0280936F
:105D90001B0246C40E94C0EFF82E87FD41C483E574
:105DA0000E94B4EF0F2D0F2C000C110B882369F10A
:105DB0000E94A352F801EE0FFF1FEB5CFD4F918391
:105DC0008083000F111F000F111F9801245F3D4FAA
:105DD0007901BC01990F880B990B0F948F462AE02B
:105DE00037ED43E25CE30F94EE46F801E055F14FE6
:105DF00020813181428153810F94EE46D7016D930A
:105E00007D938D939C9313970BC40E94486085E407
:105E10000E94F35F80E38F0D0E94F35F000F111F5C
:105E2000F801EB5CFD4F608171818CE696E00E9489
:105E3000316185E20E94F35F8AE00E94F35FF0C364
:105E400080E50E94BFEE882309F4EAC360E070E0B9
:105E500080E50E94A752F82E6FEF7FEF83E50E9446
:105E6000A7528C010196039708F0DAC3F7FCD8C358
:105E70008F2D0F944937882339F00E94236084E7DF
:105E800096E00E940460CCC30E94D1C860E08F2DD0
:105E90000E9438B10F3FBFEF1B0731F001301105F1
:105EA00071F000E010E00DC08F2D0F946E3731E0DF
:105EB00020E0892B09F030E0032F122F02C001E00F
:105EC00010E08F2D0F946E378017910709F4A8C347
:105ED00080E00E947462F5CF8AE50E94B4EF8111E0
:105EE00069C583E50E94B4EF811164C599C364E07C
:105EF00071E083E50F945F158C0168EE73E080E537
:105F00000F945F158938E3E19E0710F088E893E16C
:105F1000B8010E94EC9F84C360E085E40E94AF500A
:105F2000811173C080E50E94BFEE882351F00E946A
:105F300088EE60931D1670931E1680931F16909323
:105F4000201689E40E94BFEE882381F00E9488EE2B
:105F50002CEA35EC47E25EE30F94EE46609321169F
:105F600070932216809323169093241684E40E9443
:105F7000BFEE882381F00E9488EE2CEA35EC47E2E0
:105F80005EE30F94B14B60932516709326168093B1
:105F90002716909328160E94486040911D16509134
:105FA0001E1660911F16709120168DE996E00E94D2
:105FB000AD612CEA35EC47E25EE360912116709109
:105FC000221680912316909124160F94B14BAB01A9
:105FD000BC0189E996E00E94AD612CEA35EC47E20C
:105FE0005EE3609125167091261680912716909198
:105FF00028160F94EE46AB01BC0185E996E00E949D
:10600000AD618AE00E94F35F0BC30E94236083E8C6
:1060100096E00E94046004C380E50E94BFEE8823DE
:1060200051F00E9488EE60931116709312168093BF
:1060300013169093141689E40E94BFEE882381F012
:106040000E9488EE2CEA35EC47E25EE30F94EE46C0
:106050006093151670931616809317169093181662
:1060600084E40E94BFEE882381F00E9488EE2CEA2F
:1060700035EC47E25EE30F94B14B609319167093D1
:106080001A1680931B1690931C160E94486040912C
:10609000111650911216609113167091141689EA18
:1060A00096E00E94AD612CEA35EC47E25EE3609138
:1060B00015167091161680911716909118160F9458
:1060C000B14BAB01BC0185EA96E00E94AD612CEAC0
:1060D00035EC47E25EE36091191670911A168091D3
:1060E0001B1690911C160F94EE46AB01BC0181EA81
:1060F00096E00E94AD618AE00E94F35F91C283E561
:106100000E94BFEE182F882371F00E9488EE0F9432
:10611000194C709311026093100221E0672B09F073
:1061200020E02093C40680E50E94BFEE882359F04A
:106130002091100230911102232B11F00E94C550C2
:106140008093C4066DC211116BC20E94486089EC35
:1061500096E00E9404608091C406882319F081EBC8
:1061600096E002C08DEA96E00E9404606091100201
:106170007091110288EB96E00E94316184EB96E009
:106180000E9404604DC281E00E941FE20F94161F1E
:1061900047C280E00E941FE20E94D7E10F94161FC1
:1061A0003FC20E94D5503CC26FEF7FEF89E40E944E
:1061B000A752182F6FEF7FEF8AE40E94A752082F93
:1061C0008AE50E94BFEEF82E811105C081E50E948C
:1061D000BFEED82E01C0D12C17FD06C007FD04C0AC
:1061E000F11009C0D11007C00E9423608BEF96E028
:1061F0000E94046015C2193010F4093038F00E9472
:1062000023608CED96E00E9404600AC2E12E110F1B
:10621000FF08002E000C110B0E9488EEDD2099F083
:1062200029E02E9DF0012F9DF00D1124E00FF11FAC
:10623000EE0FFF1FEE0FFF1FE255FB4E2081318155
:106240004281538103C020E030E0A901A9E0AE9D66
:10625000F001AF9DF00D11240E0F1F1F000F111F35
:10626000000F111F02551B4E0F94D54AD8016D9394
:106270007D938D939C931397D3C10F94A22ED0C17D
:106280000F94F82CCDC183E50E94BFEE882321F046
:106290000E94C55091E089270F94AF2EC1C1409351
:1062A00097140E944B8B10929714882309F4B8C15D
:1062B0000E9448608BE197E00E940460B1C1809128
:1062C000951482FFADC1806280939514A9C18AE5BF
:1062D0000E94B4EF882331F10E9488EE6B017C01AB
:1062E00020E030E040E252EC0F94494D87FD13C0AE
:1062F00020E030E040EA51E4C701B6010F9489463E
:1063000018164CF0C092EF0ED092F00EE092F10E03
:10631000F092F20E85C10E94236086E297E00E940F
:1063200004607EC10E9448604091EF0E5091F00ED3
:106330006091F10E7091F20E83E497E00E94AD61DE
:106340008AE00E94F35F6CC10F94931369C10E94AD
:10635000C0EF082F87FD64C185E50E94BFEE88234A
:10636000A1F1E02E002E000CFF080E9488EE4B01E8
:106370005C0120E030E0A9010F94494D87FF04C083
:10638000B7FAB094B7F8B094C70133E0880F991FFB
:106390003A95E1F7FC01E456FB4E7F018082918241
:1063A000A282B38220E030E84BE354E4C501B4019B
:1063B0000F94494D18164CF480E090E8ABE3B4E438
:1063C000F70180839183A283B3838CE40E94BFEEA4
:1063D000882309F425C1002E000C110B0E9488EEC1
:1063E0006B017C0120E030E0A9010F94494D87FF4B
:1063F00004C0F7FAF094F7F8F09423E0000F111FAF
:106400002A95E1F704561B4ED8011496CD92DD92E1
:10641000ED92FC92179720E030E84BE354E4C7017B
:10642000B6010F94494D18160CF0FAC080E090E8C0
:10643000ABE3B4E4F80184839583A683B783F0C00B
:106440000F946812EDC00E94C0EF182F87FDE8C0BE
:106450008AE50E94B4EF882349F040E050E0BA0199
:106460008AE50E9468DB4B015C0106C0812C912CFF
:1064700090EAA92E91E4B92E412F63E082E00F94B7
:10648000D21A20E030E0A901C501B4010F94494DB2
:1064900018167CF580E090E0A8ECB2E489839A833A
:1064A000AB83BC83209175063091760640917706C8
:1064B00050917806C501B4010F94D54A6B017C0157
:1064C00020E030E040EA53E40F94894687FD06C09F
:1064D000C12CD12C80EAE82E83E4F82ECC8EDD8E00
:1064E000EE8EFF8EBE016F5F7F4FCE014C960E94F5
:1064F000CCD485E50E94BFEE882329F00E9488EE67
:106500006B017C010AC028E01202F0011124E4565C
:10651000FB4EC080D180E280F38020E030E0A90112
:10652000C701B6010F94494D87FF04C0F7FAF094F4
:10653000F7F8F094F7FAF094F7F8F094C982DA8259
:10654000EB82FC8243E061E0CE0101960E9486F678
:1065500020E030E0A901C501B4010F94494D18169F
:106560005CF580E090E0A8ECB2E489839A83AB8389
:10657000BC83A501940160917506709176068091A7
:106580007706909178060F94D44A6B017C0120E045
:1065900030E0A9010F94494D18161CF0C12CD12CE4
:1065A0007601CC8EDD8EEE8EFF8EBE016F5F7F4F4B
:1065B000CE014C960E94CCD440E060E088E00F947D
:1065C000D21A2EC081E080935F021092C90F60E062
:1065D00083E50E944D52811123C00E94CA5720C0FA
:1065E0000E94EFE81DC000910204109103040023F3
:1065F000B9F00E94486084E50E94F35FB8017727F4
:10660000072E000C880B990B0E94176180E20E94F4
:10661000F35F84E597E00E94046002C00E94EFE807
:106620001092810F0E94BA5700C220E030E00C9413
:1066300086210E94B552F4CF80E00E9487F40E9428
:1066400020CF61E085E40E944D52182F01E021E047
:10665000482FBE016F5F7F4FCE014C960E9406E32C
:106660006B017C019B01AC010F94CF4D81115FC088
:106670008C8C9D8CAE8CBF8C20E030E0A901C501D4
:10668000B4010F94894687FF05C027E137EB41E548
:1066900058EB04C027E137EB41E558E3C501B401ED
:1066A0000F94D54AAB01BC018AE892E00E94AD612B
:1066B00089809A80AB80BC8020E030E0A901C501D0
:1066C000B4010F94894687FF05C027E137EB41E508
:1066D00058EB04C027E137EB41E558E3C501B401AD
:1066E0000F94D54AAB01BC0185E892E00E94AD61F0
:1066F00020E030E0A901C701B6010F94894687FF69
:1067000005C027E137EB41E558EB04C027E137EB43
:1067100041E558E3C701B6010F94D54AAB01BC016E
:1067200080E892E00E94AD618AE00E94F35F0E94DF
:106730000FD3113011F40E94D7E10F94161F70CFC0
:1067400011110C9447260C94402680E00E9474623C
:106750000C9469260E9467EEAB01BC014093911432
:1067600050939214609393147093941489E992E176
:106770000E94D1A955CF61E0802F0E9438B16F2DC2
:10678000802F0E94F7B06F2D70E0802F0E9474B1AF
:1067900037E0E31203C0F092B30642CF49E0E412BF
:1067A0003FCFF092B2063CCF0E949FE50C94722935
:1067B000A3019201C501B4010F94494D18163CF094
:1067C00082EC93E060E00E94F3720C9492298FECCB
:1067D00093E0F8CF0E94D1C888E50E94BFEE8823DD
:1067E00031F05F9A8091FE0C8E7F8093FE0C89E5DC
:1067F0000E94BFEE882331F08A9A8091FE0C8D7F33
:106800008093FE0C8AE50E94BFEE882359F08091A8
:10681000080180958170809306018091FE0C8B7F2A
:106820008093FE0C85E40E94BFEE882309F4F8CE25
:10683000129AF6CE0E949CCAF3CE83E50E94B4EF72
:10684000882391F00E9488EE6093C00C7093C10C75
:106850008093C20C9093C30C6093C80C7093C90CC6
:106860008093CA0C9093CB0C80E50E94B4EF8823F0
:1068700051F00E9488EE6093C00C7093C10C80931D
:10688000C20C9093C30C82E50E94B4EF882351F0B0
:106890000E9488EE6093C40C7093C50C8093C60C64
:1068A0009093C70C84E50E94B4EF882309F4B8CE16
:1068B0000E9488EE6093C80C7093C90C8093CA0C38
:1068C0009093CB0CADCE82E40E94BFEE882351F0B2
:1068D0000F94721560939C0C70939D0C80939E0C8A
:1068E00090939F0C83E50E94BFEE882351F00E9495
:1068F00088EE6093CC0C7093CD0C8093CE0C90936B
:10690000CF0C84E50E94BFEE882351F00E9488EEF0
:106910006093D00C7093D10C8093D20C9093D30CD5
:1069200088E50E94BFEE882351F00E9488EE6093B4
:106930008A0670938B0680938C0690938D0689E56A
:106940000E94BFEE882351F00E9488EE60938E066D
:1069500070938F0680939006909391068AE50E942B
:10696000BFEE8823B1F00E9488EE60939206709388
:10697000930680939406909395062DEC3CEC4CEC9A
:106980005DE30F948946181624F08AE096E00E9491
:10699000046085E40E94BFEE882309F441CE0E9482
:1069A00088EE60939606709397068093980690936E
:1069B000990636CE0E9488EE20E030E040E050ECB0
:1069C0000F94894687FD12C00E9488EE20E030E0D7
:1069D00040E050E40F94494D18161CF00E9488EED8
:1069E00009C060E070E080E090E404C060E070E026
:1069F00080E090EC2091A80C3091A90C4091AA0C59
:106A00005091AB0C0F94EE460F94194C2091FE0C54
:106A100022FF06CE20911B1030911C10620F731FB5
:106A200070931C1060931B10FBCDA3960FB6F894C7
:106A3000DEBF0FBECDBFDF91CF911F910F91FF90B1
:106A4000EF90DF90CF90BF90AF909F908F907F900E
:106A50006F905F904F903F902F9008952F923F92AC
:106A60004F925F926F927F928F929F92AF92BF925E
:106A7000CF92DF92EF92FF920F931F93CF93DF930A
:106A8000CDB7DEB7C85BD1090FB6F894DEBF0FBE35
:106A9000CDBF1C016B01CB54DF4F288339834A8360
:106AA0005B83C55BD040DC018D919D910D90BC91C5
:106AB000A02DCF54DF4F88839983AA83BB83C15B0A
:106AC000D040BE016F5F7F4FC1010E94474FCB5442
:106AD000DF4F288139814A815B81C55BD04060915D
:106AE0004D1070914E1080914F10909150100F9456
:106AF000D54A60934D1070934E1080934F10909331
:106B00005010C355DF4F0883CD5AD040C255DF4FD8
:106B10001883CE5AD040E1E5F0E1C155DF4FF9834B
:106B2000E883CF5AD0408F01C355DF4FE880F9800A
:106B3000CD5AD040D7012D913D914D915D917D0170
:106B4000F80160817181828193810F94D54AD801C7
:106B50006D937D938D939D938D01EDE5F0E1EA17A3
:106B6000FB0741F70F943723BE016B5A7F4FC101DA
:106B70000E94474F56018E010F5F1F4F9E012B5AF7
:106B80003F4F490133E0C755DF4F3883C95AD040E2
:106B9000D5014D905D906D907D905D016801E12C77
:106BA000F12CF401EE0DFF1D2081318142815381D2
:106BB000C301B2010F94D54A9B01AC01F60160817B
:106BC0007181828193810F94D44AD6016D937D9314
:106BD0008D939C931397BCE0CB0ED11CECE0EE0E92
:106BE000F11CF4E5EF16F104E1F6C755DF4F2881FB
:106BF000C95AD0402150C755DF4F2883C95AD040C9
:106C00000C5F1F4F34E0830E911C2111C1CF2091E6
:106C10004D1030914E1040914F1050915010609196
:106C2000AA147091AB148091AC149091AD140F9490
:106C3000B14B6B017C0120E030E0A9010F94EE46DE
:106C400020E030E040E450E40F94B14B2BEA3AEA04
:106C50004AEA5EE30F94D54A4B015C0129813A81EF
:106C60004B815C810F94EE462B013C012D813E81CE
:106C70004F815885C501B4010F94EE469B01AC01CC
:106C8000C301B2010F94D54A2B013C0129853A85F5
:106C90004B855C85C501B4010F94EE469B01AC01A8
:106CA000C301B2010F94D54AD1016D937D938D93A9
:106CB0009C931397A7019601C701B6010F94D54A7B
:106CC00020E030E040E450E40F94B14B2BEA3AEA84
:106CD0004AEA5EE30F94D54AC755DF4F688379834C
:106CE0008A839B83C95AD040C701B601905820E0DF
:106CF00030E040E450E40F94B14B2BEA3AEA4AEA20
:106D00005EE30F94D54A4B015C012D853E854F858E
:106D10005889C755DF4F688179818A819B81C95A1B
:106D2000D0400F94EE462B013C0129893A894B89CA
:106D30005C89C501B4010F94EE469B01AC01C3010F
:106D4000B2010F94D54A2B013C012D893E894F8910
:106D5000588DC501B4010F94EE469B01AC01C301EF
:106D6000B2010F94D54AF1016483758386839783BA
:106D70002DA13EA14FA158A5C501B4010F94EE4627
:106D80002B013C0129A53AA54BA55CA5C755DF4FB2
:106D9000688179818A819B81C95AD0400F94EE46DF
:106DA0009B01AC01C301B2010F94D54A2B013C01F8
:106DB0002DA53EA54FA558A9C501B4010F94EE46D7
:106DC0009B01AC01C301B2010F94D54AD1011C96BD
:106DD0006D937D938D939C931F9721962CAD3DAD24
:106DE0004EAD5FAD2197C501B4010F94EE462B0166
:106DF0003C0125962CAD3DAD4EAD5FAD2597C5014F
:106E0000B4010F94EE469B01AC01C301B2010F9493
:106E1000D54A4B015C0129962CAD3DAD4EAD5FAD21
:106E20002997C755DF4F688179818A819B81C95A2B
:106E3000D0400F94EE469B01AC01C501B4010F9404
:106E4000D54AF101648B758B868B978B20E030E0FF
:106E500040E050ECC701B6010F94EE4620E030E070
:106E600040E450E40F94B14B2BEA3AEA4AEA5EE37D
:106E70000F94D54A4B015C0120E030E040E450E43F
:106E8000C701B6010F94B14B2BEA3AEA4AEA5EE336
:106E90000F94D54A6B017C0129A93AA94BA95CA999
:106EA000C501B4010F94EE462B013C012DA93EA96A
:106EB0004FA958ADC701B6010F94EE469B01AC0136
:106EC000C301B2010F94D54A2B013C0129AD3AAD63
:106ED0004BAD5CADC701B6010F94EE469B01AC0112
:106EE000C301B2010F94D54AD10150966D937D93A1
:106EF0008D939C9353972D962CAD3DAD4EAD5FADCC
:106F00002D97C701B6010F94EE462B013C01619607
:106F10002CAD3DAD4EAD5FAD6197C501B4010F9491
:106F2000EE469B01AC01C301B2010F94D54A2B017F
:106F30003C0165962CAD3DAD4EAD5FAD6597C7018B
:106F4000B6010F94EE469B01AC01C301B2010F9450
:106F5000D54AF101608F718F828F938F298D3A8D81
:106F60004B8D5C8DC701B6010F94EE462B013C01A1
:106F70002D8D3E8D4F8D58A1C701B6010F94EE4661
:106F80009B01AC01C301B2010F94D54A6B017C0196
:106F900029A13AA14BA15CA1C501B4010F94EE4611
:106FA0009B01AC01C701B6010F94D54AD1011896D7
:106FB0006D937D938D939C931B9781010C5F1F4F65
:106FC0007101BCE1EB0EF11CCF54DF4F28813981F8
:106FD0004A815B81C15BD040F10160817181828116
:106FE00093810F94D44A9B01AC01D8016D917D919E
:106FF0008D919C910F94D44AF80161937193819380
:1070000091938F01EE16FF06F9F6CF54DF4F88817A
:107010009981AA81BB81C15BD040F10180839183BA
:10702000A283B383CB54DF4F288139814A815B81AE
:10703000C55BD04060914D1070914E1080914F1003
:10704000909150100F94D44A60934D1070934E104D
:1070500080934F1090935010C355DF4FA881B98192
:10706000CD5AD0402D913D914D915D91C355DF4F4B
:10707000B983A883CD5AD040C155DF4FE881F9814B
:10708000CF5AD04060817181828193810F94D44A1C
:10709000C155DF4FA881B981CF5AD0406D937D9300
:1070A0008D939D93C155DF4FB983A883CF5AD040AC
:1070B000EDE5F0E1EA17FB0779F60F943723C854A2
:1070C000DF4F0FB6F894DEBF0FBECDBFDF91CF917B
:1070D0001F910F91FF90EF90DF90CF90BF90AF90F6
:1070E0009F908F907F906F905F904F903F902F90E8
:1070F00008952F923F924F925F926F927F928F925C
:107100009F92AF92BF92CF92DF92EF92FF920F9336
:107110001F93CF93DF93CDB7DEB7C350D1400FB6E7
:10712000F894DEBF0FBECDBF64E070E080E50E9442
:10713000A752AE968FAFAE978B3018F088E299E0E9
:10714000CEC184E50E94BFEEC756DF4F8883C95980
:10715000D04040E050E0BA0183E40E9468DBCC54A8
:10716000DF4F688379838A839B83C45BD04020E0B0
:1071700030E0A9010F94894687FF03C088EF98E0AB
:10718000AEC160E070E086E40E94A752C254DF4FB7
:107190008883CE5BD0408F3118F08DEC98E09FC192
:1071A00061E086E50E94AF50C656DF4F8883CA591A
:1071B000D040843018F085EA98E091C181E0C7564C
:1071C000DF4F2881C959D0402827CD54DF4F28836D
:1071D000C35BD04085E40E94BFEE082FAE968FAD12
:1071E000AE97813011F40C94104F91E0C755DF4FEA
:1071F0009883C95AD0408F3F11F40C94DE4EC75586
:10720000DF4F1882C95AD0408230C9F4C756DF4FC9
:10721000A881C959D040A1110C94EB4EC655DF4F3F
:107220001882CA5AD040CD54DF4FB881C35BD040DA
:10723000C855DF4FB883C85AD04010E01BC0AE9687
:10724000BFADAE97B33014F40C94DE4E91E0C85548
:10725000DF4F9883C85AD04010E0A1E0C655DF4FF9
:10726000A883CA5AD040AE96EFADAE97EF3F11F467
:107270000C94214F21E0C854DF4F2883C85BD040D5
:10728000AE968FADAE97882311F40C94214FAE9635
:107290009FADAE97933014F40C94264FCD54DF4F2E
:1072A000A881C35BD040C955DF4FA883C75AD040DF
:1072B000C656DF4FB881CA59D040C556DF4F188235
:1072C000CB59D040B11110C0C456DF4F1882CC59F1
:1072D000D040C356DF4F1882CD59D040C256DF4F41
:1072E0001882CE59D04012C0E0ECC456DF4FE8837C
:1072F000CC59D040F9E7C356DF4FF883CD59D04081
:1073000024E4C256DF4F2883CE59D0408091A30E8B
:107310009091A40EA091A50EB091A60EC452DF4F7D
:1073200088839983AA83BB83CC5DD0408091A70ECC
:107330009091A80EA091A90EB091AA0ECC52DF4F49
:1073400088839983AA83BB83C45DD0408091AB0EB0
:107350009091AC0EA091AD0EB091AE0EC453DF4F24
:1073600088839983AA83BB83CC5CD04080914D10E5
:1073700090914E10A0914F10B0915010C054DF4F1B
:1073800088839983AA83BB83C05CD0408091850E9B
:107390009091860EA091870EB091880ECC53DF4F4E
:1073A00088839983AA83BB83C45CD04080915110A9
:1073B00090915210A0915310B0915410C853DF4FC8
:1073C00088839983AA83BB83C85CD0408091551081
:1073D00090915610A0915710B0915810C852DF4F9D
:1073E00088839983AA83BB83C85DD040809159105C
:1073F00090915A10A0915B10B0915C10C053DF4F78
:1074000088839983AA83BB83C05DD04081E998E0DB
:107410000E940460C755DF4F9881C95AD04091112E
:107420006BC0AE96AFADAE97AA2309F465C080904D
:10743000AA149090AB14A090AC14B090AD14F2EDDF
:107440002F2E312CB101032C000C880B990B0F94BB
:107450008F462BED3FE049E450E40F94EE4620E0E8
:1074600030E044E353E40F94B14B6B017C010F9483
:10747000844D9B01AC01C501B4010F94EE462B0174
:107480003C01C701B6010F94AE4B9B01AC01C50195
:10749000B4010F94EE469B01AC010F94EE46E296C8
:1074A0006CAF7DAF8EAF9FAFE297A3019201C30196
:1074B000B2010F94EE469B01AC01E2966CAD7DAD3E
:1074C0008EAD9FADE2970F94D54A20E030E442E5BF
:1074D00056E40F948946181634F48DE698E00E941D
:1074E00004600C942D4FBCE32B0E311CEAE32E16E6
:1074F000E2E03E0609F0A6CF8EE598E00E94046027
:10750000C656DF4FF881CA59D040F11104C083E557
:1075100098E00E9404608AE00E94F35F60E08EE5DC
:1075200098E00E94F372C955DF4F6881C75AD04076
:10753000C854DF4F8881C85BD0400E941950AE9676
:107540002FADAE97222341F081E0C755DF4FF88081
:10755000C95AD040F82601C0F12C0E94D1C80E941F
:1075600020CFF1100E94CCF4AE968FADAE97882359
:1075700059F081E08093FD0C0F940C210F9426218B
:107580008091FC0C8093FD0C002339F091E0C354F2
:10759000DF4F9883CD5BD04006C0A2E0C354DF4FDD
:1075A000A883CD5BD040AE96BFADAE97B8303CF06F
:1075B000E2E0C154DF4FE883CF5BD04005C0C15447
:1075C000DF4F1882CF5BD040112339F0F2E0C05278
:1075D000DF4FF883C05ED04006C021E0C052DF4FCD
:1075E0002883C05ED040AE968FADAE97823039F41E
:1075F00092E0CF51DF4F9883C15ED04006C0A1E03A
:10760000CF51DF4FA883C15ED040C556DF4FB88150
:10761000CB59D040C156DF4FB883CF59D040C45664
:10762000DF4FE881CC59D040C056DF4FE883C05AC5
:10763000D040C356DF4FF881CD59D040CF55DF4FF2
:10764000F883C15AD040C256DF4F2881CE59D0406E
:10765000CE55DF4F2883C25AD040EB2EFE2E0F2F7F
:10766000122FCC56DF4F1882C459D040CE014D9610
:10767000AB969FAF8EAFAB97DE01D996AD96BFAFFD
:10768000AEAFAD97C154DF4FE881CF5BD0400E2E37
:10769000000CFF0BC250DF4FF983E883CE5FD04070
:1076A0004C971C01AE968FADAE97082E000C990B2F
:1076B000AA0BBB0BC050DF4F88839983AA83BB837F
:1076C000C050D1408CE1AB96AEADBFADAB971D9233
:1076D0008A95E9F720E030EC49E754E4B701C801A6
:1076E0000F948946882399F19701A801C556DF4F69
:1076F0006881CB59D040C456DF4F7881CC59D040F7
:10770000C356DF4F8881CD59D040C256DF4F988194
:10771000CE59D0400F94D54A20E030E040E05FE3FE
:107720000F94EE46CB56DF4F6883C559D040CA56FA
:10773000DF4F7883C659D040C956DF4F8883C75979
:10774000D040C856DF4F9883C859D04028C0C5568E
:10775000DF4FB881CB59D040CB56DF4FB883C559E6
:10776000D040C456DF4FE881CC59D040CA56DF4FD5
:10777000E883C659D040C356DF4FF881CD59D04079
:10778000C956DF4FF883C759D040C256DF4F288112
:10779000CE59D040C856DF4F2883C859D040CC5668
:1077A000DF4F8881C459D0408F5FCC56DF4F88832C
:1077B000C459D040AE969FADAE97913061F0A1E034
:1077C000AF96AFAFAF979F3F51F0AF961FAEAF9759
:1077D000923029F406C0B1E0AF96BFAFAF9710E08A
:1077E00005C0C756DF4F1881C959D040FE017D96AC
:1077F0001192119211921192AD968EAD9FADAD97EF
:10780000E817F907A9F7AE969FADAE97911111C091
:10781000ACEAAF96AFAFAF97B5ECE396BFAFE397E7
:10782000E7E2E796EFAFE797F7E3E896FFAFE89771
:1078300023C4AE962FADAE97233099F4AE968FAD9C
:10784000AE978550833008F448C0C12CD12C70EA23
:10785000E72E70E4F72E812C912CA12CE0E4BE2EB3
:1078600059C0AE968FADAE97863041F3AE96AFADB0
:10787000AE97A93009F43EC019821A821B821C827D
:1078800019AE1AAE1BAE1CAE00E020E0C354DF4FB1
:107890004881CD5BD040B101CE01C9960E9406E37C
:1078A0002D8D3E8D4F8D58A10F94D54A6D8F7E8FB3
:1078B0008F8F98A39B01AC010F94CF4D81110C9435
:1078C000D84EAE96BFADAE97B3300CF4D0C0AE96E6
:1078D0009FADAE97983074F4B1CFC12CD12C50EC41
:1078E000E52E50E4F52E812C912C60E8A62E6FE356
:1078F000B62E10C03BEAC32E3AEAD32E3AECE32E62
:1079000030E4F32E4BEA842E4AEA942E4AE2A42E67
:107910004FE3B42E22E739EF4FE75FE3C701B6012B
:107920000F94494D18160CF080C020E030E040E87C
:107930005FE3C701B6010F94D44A20E030E040E78E
:1079400052E40F94EE4620E030E042E553E40F9419
:10795000D54A2BED3FE049E450E40F94EE4620E099
:1079600030E044E353E40F94B14B2B013C012DEC88
:107970003CEC4CEC5DE36091AA147091AB148091E7
:10798000AC149091AD140F94EE46E6966CAF7DAFBB
:107990008EAF9FAFE697C301B2010F94844D9B0158
:1079A000AC01E6966CAD7DAD8EAD9FADE6970F94C4
:1079B000EE4669837A838B839C83C301B2010F9463
:1079C000AE4B9B01AC01E6966CAD7DAD8EAD9FAD2F
:1079D000E6970F94EE4669AF7AAF8BAF9CAF00E0AD
:1079E00020E0C354DF4F4881CD5BD040B101CE01D0
:1079F000C9960E9406E32D8D3E8D4F8D58A10F94A0
:107A0000D54A6D8F7E8F8F8F98A39B01AC010F9409
:107A1000CF4D81110C94D84EA5019401C701B60138
:107A20000F94D44A6B017C0175CFCD8CDE8CEF8C2A
:107A3000F8A0AE96EFADAE97E53069F0C050DF4FDD
:107A4000688179818A819B81C050D1400F948F4693
:107A50009B01AC0104C020E030E040EE50E4C701DF
:107A6000B6010F94B14B6D8F7E8F8F8F98A3AF9619
:107A7000FFADAF97F11194C2111102C061E001C0D6
:107A800062E0AE962FADAE972A3009F1293069F148
:107A90002830E1F1273009F44AC0263009F458C0F3
:107AA000253009F463C0AF961FAEAF97E3961FAEC3
:107AB000E397243009F46BC0233009F470C0E796D3
:107AC0001FAEE79780E4E8968FAFE89770C099E81B
:107AD000AF969FAFAF97A8E8E396AFAFE397B8E84C
:107AE000E796BFAFE797EDE356C0FBEAAF96FFAF6F
:107AF000AF972AEAE3962FAFE3978AEAE7968FAF2C
:107B0000E7979DE3E8969FAFE89751C0A9E3AF964A
:107B1000AFAFAF97BEE8E396BFAFE397E3EEE7966C
:107B2000EFAFE797FDE3E896FFAFE89740C025E2A7
:107B3000AF962FAFAF9789E4E3968FAFE39792E1CB
:107B4000E7969FAFE797AEE3E896AFAFE8972FC011
:107B5000BDECAF96BFAFAF97ECECE396EFAFE3971A
:107B6000FCE4E796FFAFE7972EE31EC08BEAAF96E3
:107B70008FAFAF979AEAE3969FAFE397AAEAE796AB
:107B8000AFAFE797BEE3E896BFAFE89710C0E796C0
:107B90001FAEE797EFE3E896EFAFE89708C0F0E88D
:107BA000E796FFAFE7972FE3E8962FAFE897062E0B
:107BB000000C770B880B990B0F948F464B015C01DF
:107BC00081E0E9968FAFE9972EE23FEF4FED50E469
:107BD000C501B4010F94894687FF97C120E030E0CA
:107BE00040E85FE3C501B4010F94D44A20E030E0DF
:107BF00040E752E40F94EE4620E030E042E553E4E3
:107C00000F94D54A2BED3FE049E450E40F94EE4643
:107C100020E030E044E353E40F94B14B6B017C016E
:107C200020E030E040E85FE3C501B4010F94644C0C
:107C3000C058DF4F688379838A839B83C058D040C4
:107C4000C701B6010F94844DC857DF4F688379830D
:107C50008A839B83C858D040C701B6010F94AE4BAE
:107C6000C457DF4F688379838A839B83CC58D04085
:107C7000ED961FAEED97E9969FADE997992391F0A8
:107C8000C250DF4F68817981CE5FD040ED96AFADB5
:107C9000ED976A1B7109A7FD7395072E000C880BE1
:107CA000990B08C0ED96BFADED976B2FBB0F770B0F
:107CB000880B990B0F948F462DEC3CEC4CEC5DE35C
:107CC0000F94EE469B01AC0160E070E080E89FE31A
:107CD0000F94D44A2091AA143091AB144091AC1463
:107CE0005091AD140F94EE466B017C01C857DF4FE5
:107CF000288139814A815B81C858D0400F94EE4673
:107D000069837A838B839C83C457DF4F28813981B1
:107D10004A815B81CC58D040C701B6010F94EE4632
:107D200069AF7AAF8BAF9CAF00E020E0C354DF4F68
:107D30004881CD5BD040B101CE01C9960E9406E3D7
:107D40006B017C019B01AC010F94CF4D81110C9410
:107D5000D84EC058DF4F288139814A815B81C05895
:107D6000D040C501B4010F94D44A2B013C0120E05E
:107D700030E040EC50E40F94D54A20E030E040E899
:107D80005FE30F94D44A0F94544D862F66E00F940E
:107D9000EB4D0DE110E00C0F1D1FE4E09E9F000D68
:107DA000111D11240C5F1F4F20E030E044EB52E422
:107DB000C058DF4F688179818A819B81C058D0404B
:107DC0000F94EE462BED3FE049E450E40F94EE466D
:107DD00020E030E044E353E40F94B14BCC57DF4F45
:107DE000688379838A839B83C458D0400F94AE4BB9
:107DF0009B01AC010F94EE46A70196010F94EE464D
:107E00009B01AC01D8016D917D918D919C910F9456
:107E1000D54AF8016083718382839383C301B201E1
:107E20000F94544D862F66E00F94EB4D0DE110E05A
:107E30000C0F1D1FF4E09F9F000D111D11240C5FFE
:107E40001F4FCC57DF4F688179818A819B81C4584D
:107E5000D0400F94844D9B01AC010F94EE46A701D6
:107E600096010F94EE469B01AC01D8016D917D9176
:107E70008D919C910F94D54AF80160837183828320
:107E80009383ED96FFADED97FF5FED96FFAFED9716
:107E9000C154DF4F2881CF5BD0402F170CF0EBCEC1
:107EA000E9968FADE99791E08927E9968FAFE99739
:107EB000AE96AFADAE97A8309CF020E030E040E445
:107EC00050E4AF966FADAF97E3967FADE397E7963B
:107ED0008FADE797E8969FADE8970F94EE460CC0FC
:107EE000AF966FADAF97E3967FADE397E7968FAD13
:107EF000E797E8969FADE8979B01AC01C501B401F7
:107F00000F94D54A4B015C015FCEAE96BFADAE97E4
:107F1000B430C4F419821A821B821C8219AE1AAEC4
:107F20001BAE1CAE29961CAE1DAE1EAE1FAE299711
:107F3000A101BE01675C7F4FCE018B5B9F4F0E940A
:107F4000ABD42EC0AF962FADAF97E3963FADE3977E
:107F5000E7964FADE797E8965FADE89760E070E091
:107F600080E89FE30F94B14B6B017C018E010F5DA4
:107F70001F4FA7019601F801608171818281938171
:107F80000F94B14BD8016D937D938D939D938D018B
:107F9000AD96EEADFFADAD97EA17FB0751F7BACF3F
:107FA000C755DF4F2881C95AD040211131CC6D8D82
:107FB0007E8D8F8D98A19B01AC010F94EE466B01D5
:107FC0007C01C052DF4FB880C05ED04001E010E0BD
:107FD000EDE1F0E0EC0FFD1F24E0B29EE00DF11D9D
:107FE000112460817181828193819B01AC010F9486
:107FF000EE469B01AC01C701B6010F94D54A6B0157
:108000007C010F5F1F4FCF51DF4F8881C15ED04091
:10801000B80E96E09B15E0F6B801110F880B990B8E
:108020000F948F469B01AC01C701B6010F94B14B71
:108030000F948E4D20E030E04AE754E40F94EE4672
:108040000F94544D0F948F4620E030E04AE754E4FB
:108050000F94B14B2CEA35EC47E257E30F94D54A25
:10806000AF966FAFAF97E3967FAFE397E7968FAF8B
:10807000E797E8969FAFE897AF962FADAF97E39657
:108080003FADE397E7964FADE797E8965FADE8978A
:10809000CB56DF4F6881C559D040CA56DF4F788133
:1080A000C659D040C956DF4F8881C759D040C856FD
:1080B000DF4F9881C859D0400F94494D181674F07D
:1080C000C254DF4FA881CE5BD040CC56DF4FB88181
:1080D000C459D040AB1714F40C94284AAF962FAD76
:1080E000AF97E3963FADE397E7964FADE797E896F6
:1080F0005FADE897CC54DF4F688179818A819B819D
:10810000C45BD0400F94894687FD02C00C94284A76
:10811000AF962FADAF97E3963FADE397E7964FADA0
:10812000E797E8965FADE897C156DF4F6881CF5972
:10813000D040C056DF4F7881C05AD040CF55DF4F76
:108140008881C15AD040CE55DF4F9881C25AD04065
:108150000F94494D18160CF080C08091A30E909199
:10816000A40EA091A50EB091A60EC452DF4F888335
:108170009983AA83BB83CC5DD0408091A70E909158
:10818000A80EA091A90EB091AA0ECC52DF4F888301
:108190009983AA83BB83C45DD0408091AB0E90913C
:1081A000AC0EA091AD0EB091AE0EC453DF4F8883DC
:1081B0009983AA83BB83CC5CD04080914D10909171
:1081C0004E10A0914F10B0915010C054DF4F8883D3
:1081D0009983AA83BB83C05CD0408091850E909127
:1081E000860EA091870EB091880ECC53DF4F888306
:1081F0009983AA83BB83C45CD04080915110909135
:108200005210A0915310B0915410C853DF4F88837F
:108210009983AA83BB83C85CD0408091551090910C
:108220005610A0915710B0915810C852DF4F888354
:108230009983AA83BB83C85DD040809159109091E7
:108240005A10A0915B10B0915C10C053DF4F88832F
:108250009983AA83BB83C05DD040FE01E35AFF4FE0
:108260008CE0DF01282F1D922A95E9F73C97DF016A
:108270001D928A95E9F74090AA145090AB14609033
:10828000AC147090AD14AE96BFADAE97B83084F01C
:1082900026E636E646E65FE3C301B2010F94EE46FA
:1082A0006093AA147093AB148093AC149093AD14A4
:1082B00020914D1030914E1040914F105091501020
:1082C0006091AA147091AB148091AC149091AD148C
:1082D0000F94B14B2BEA3AEA4AE25FE30F94B14BB9
:1082E0009B01AC0160E070E080E89FE30F94B14B2C
:1082F000C458DF4F688379838A839B83CC57D040EF
:108300008CE1E82EF1012E2D11922A95E9F75E01FC
:1083100085E4A80EB11C9CE0F92ED501EF2D1D922D
:10832000EA95E9F7AD96AEADBFADAD97EF2D1D92D5
:10833000EA95E9F78E01075C1F4F2AE037ED43E22B
:108340005CE3B501C1010E942E352D853E854F8528
:1083500058896D817E818F8198850F94D54A2D89AA
:108360003E894F89588D0F94D54A29893A894B897E
:108370005C890F94D54A298D3A8D4B8D5C8D0F9475
:10838000D54A29853A854B855C850F94D54A905806
:1083900020E030E040EC50E40F94B14B9B01AC0185
:1083A0006AE077ED83E29CE30F94B14B20E030E08C
:1083B00040E450E40F94B14BC155DF4F688379839B
:1083C0008A839B83CF5AD040D1011D92EA94E9F76A
:1083D000F5012F2D11922A95E9F7AD96AEADBFADFF
:1083E000AD971D92FA94E9F7EA961FAF0EAFEA97A0
:1083F000610125E0F22EC555DF4F188219821A82DD
:108400001B82CB5AD040C058DF4FA882C058D04002
:10841000EB2C19AE1AAE1BAE1CAE21961CAE1DAED7
:108420001EAE1FAE219725961CAE1DAE1EAE1FAE12
:108430002597EA96EEADFFADEA978AE097EDA3E2C5
:10844000BCE381939193A193B193EA96FFAFEEAF12
:10845000EA978E01075C1F4F20E030E0A901C05869
:10846000DF4F6881C058D0407E2DC1010E942E355B
:108470008F2D66E00F94EB4DF10124E0929FE00D0B
:10848000F11D112420E030E040EC50E4648175815E
:10849000868197810F94B14BC555DF4F2881398173
:1084A0004A815B81CB5AD0400F94D54A4B015C0185
:1084B00020E030E040EC50E4D60118966D917D91BB
:1084C0008D919C911B970F94B14B9B01AC01C50101
:1084D000B4010F94D44AC555DF4F688379838A83EA
:1084E0009B83CB5AD040F394F394B8E0CB0ED11CCD
:1084F000EBE0FE128ECF4092AA145092AB14609221
:10850000AC147092AD14AE96FFADAE97F13029F079
:10851000F23031F1F111C5C235C720E030E040E85A
:1085200050E46D8D7E8D8F8D98A10F94EE4620E0E6
:1085300030E040E85EE30F94EE46A1966CAF7DAF6D
:108540008EAF9FAFA197A5966CAF7DAF8EAF9FAF5B
:10855000A597A9966CAF7DAF8EAF9FAFA99712C7B5
:108560008D8D9E8DAF8DB8A1EC968CAF9DAFAEAFCB
:10857000BFAFEC97CD54DF4F9881C35BD0409923B8
:1085800009F434C189A19AA1ABA1BCA1C058DF4FA5
:1085900088839983AA83BB83C058D04020E030E011
:1085A00040E850E4BC01CD010F94EE4620E030E0FD
:1085B00040E85EE30F94EE46CC57DF4F6883798343
:1085C0008A839B83C458D040C9A4DAA4EBA4FCA43A
:1085D000A7019601C701B6010F94D54A20E030E00B
:1085E00040E85EE30F94EE46C857DF4F6883798317
:1085F0008A839B83C858D04089A89AA8ABA8BCA8F6
:10860000A5019401C501B4010F94D54A20E030E0E2
:1086100040E85EE30F94EE46C457DF4F68837983EA
:108620008A839B83CC58D04020E030E040E850E47F
:10863000EC966CAD7DAD8EAD9FADEC970F94EE4694
:1086400020E030E040E85EE30F94EE462B013C0171
:10865000C857DF4F288139814A815B81C858D04093
:10866000CC57DF4F688179818A819B81C458D04083
:108670000F94D44AC457DF4F288139814A815B81E6
:10868000CC58D0400F94D44AC458DF4F2881398148
:108690004A815B81CC57D0400F94EE46A3019201F2
:1086A0000F94D54AA1966CAF7DAF8EAF9FAFA197C7
:1086B00020E030E040E850E4C701B6010F94EE46F8
:1086C00020E030E040E85EE30F94EE46C057DF4F15
:1086D000688379838A839B83C059D040C058DF4F19
:1086E000288139814A815B81C058D040CA01B901D3
:1086F0000F94D54A20E030E040E85EE30F94EE4668
:108700006B017C019B01AC01C057DF4F688179810F
:108710008A819B81C059D0400F94D44AC457DF4FFF
:10872000288139814A815B81CC58D0400F94D44A4A
:10873000C458DF4F288139814A815B81CC57D040B2
:108740000F94EE46A30192010F94D54AA5966CAF03
:108750007DAF8EAF9FAFA59720E030E040E850E4BA
:10876000C501B4010F94EE4620E030E040E85EE33E
:108770000F94EE464B015C01C701B6019058C857F3
:10878000DF4F288139814A815B81C858D0400F94DE
:10879000D44AA50194010F94D54AC458DF4F2881CB
:1087A00039814A815B81CC57D0400F94EE46A301BA
:1087B00092010F94D54AA9966CAF7DAF8EAF9FAF53
:1087C000A997C057DF4F288139814A815B81C05901
:1087D000D040CC57DF4F688179818A819B81C45812
:1087E000D0400F94D54AA501940132C18DA99EA90C
:1087F000AFA9B8ADC058DF4F88839983AA83BB83E4
:10880000C058D0409C01AD01BC01CD010F94D54AA8
:1088100020E030E040E85EE30F94EE46CC57DF4FB7
:10882000688379838A839B83C458D0408DA49EA497
:10883000AFA4B8A820E030E040E850E4C501B4019E
:108840000F94EE4620E030E040E85EE30F94EE4601
:10885000C857DF4F688379838A839B83C858D04089
:10886000CDA0DEA0EFA0F8A4A7019601C701B60134
:108870000F94D54A20E030E040E85EE30F94EE46E6
:10888000C457DF4F688379838A839B83CC58D04059
:1088900020E030E040E850E4EC966CAD7DAD8EAD6C
:1088A0009FADEC970F94EE4620E030E040E85EE3A9
:1088B0000F94EE462B013C01C857DF4F28813981C8
:1088C0004A815B81C858D040CC57DF4F688179819D
:1088D0008A819B81C458D0400F94D44AC457DF4F3B
:1088E000288139814A815B81CC58D0400F94D54A88
:1088F000C458DF4F288139814A815B81CC57D040F1
:108900000F94EE46A30192010F94D54AA1966CAF45
:108910007DAF8EAF9FAFA197A5019401C501B401B2
:108920000F94D54A20E030E040E85EE30F94EE4635
:10893000C057DF4F688379838A839B83C059D040B7
:1089400020E030E040E850E4C058DF4F6881798192
:108950008A819B81C058D0400F94EE4620E030E0E1
:1089600040E85EE30F94EE464B015C019B01AC01D5
:10897000C057DF4F688179818A819B81C059D0407F
:108980000F94D44AC457DF4F288139814A815B81D3
:10899000CC58D0400F94D54AC458DF4F2881398134
:1089A0004A815B81CC57D0400F94EE46A3019201DF
:1089B0000F94D54AA5966CAF7DAF8EAF9FAFA597AC
:1089C00020E030E040E850E4C701B6010F94EE46E5
:1089D00020E030E040E85EE30F94EE466B017C015E
:1089E000C057DF4F288139814A815B81C059D0400F
:1089F000CC57DF4F688179818A819B81C458D040F0
:108A00000F94D54AA70196010F94D44AC458DF4F5A
:108A1000288139814A815B81CC57D0400F94EE4642
:108A2000A30192010F94D54AA9966CAF7DAF8EAF8A
:108A30009FAFA997A5019401C857DF4F688179813D
:108A40008A819B81C858D0400F94D54AA7019601CE
:108A50000F94D54A6B017C0120E030E040E451E402
:108A6000EC966CAD7DAD8EAD9FADEC970F94EE4660
:108A700020E030E040E85EE30F94EE469B01AC015D
:108A8000C701B6010F94D44AC155DF4F28813981FF
:108A90004A815B81CF5AD0400F94EE464B015C0176
:108AA00088C489A19AA1ABA1BCA1EC968CAF9DAF63
:108AB000AEAFBFAFEC979C01AD01BC01CD010F94EF
:108AC000D54A20E030E040E85EE30F94EE46C7541C
:108AD000DF4F688379838A839B83C95BD04089A5F4
:108AE0009AA5ABA5BCA5C058DF4F88839983AA83FC
:108AF000BB83C058D04020E030E040E85EE3BC01DA
:108B0000CD010F94EE46CE51DF4F688379838A837F
:108B10009B83C25ED04089A99AA9ABA9BCA9CC57B6
:108B2000DF4F88839983AA83BB83C458D04020E059
:108B300030E040E85EE3BC01CD010F94EE464B010E
:108B40005C018DA59EA5AFA5B8A9C857DF4F888346
:108B50009983AA83BB83C858D0409C01AD01BC0156
:108B6000CD010F94D54A20E030E040E85EE30F9459
:108B7000EE46CA51DF4F688379838A839B83C65E42
:108B8000D0408DA99EA9AFA9B8ADC457DF4F888347
:108B90009983AA83BB83CC58D04020E030E040E8E2
:108BA0005EE3BC01CD010F94EE46C651DF4F6883F2
:108BB00079838A839B83CA5ED0408DA19EA1AFA199
:108BC000B8A5C057DF4F88839983AA83BB83C05958
:108BD000D04020E030E040E85EE3BC01CD010F94DE
:108BE000EE466B017C018D8D9E8DAF8DB8A1CD556C
:108BF000DF4F88839983AA83BB83C35AD04020E088
:108C000030E040E850E4BC01CD010F94EE4620E096
:108C100030E040E85EE30F94EE462B013C01CE517C
:108C2000DF4F288139814A815B81C25ED040C754C1
:108C3000DF4F688179818A819B81C95BD0400F9425
:108C4000D44AA50194010F94D44ACA51DF4F288118
:108C500039814A815B81C65ED0400F94D44AC651A7
:108C6000DF4F288139814A815B81CA5ED0400F94F1
:108C7000D54AA70196010F94D54AC458DF4F2881E1
:108C800039814A815B81CC57D0400F94EE46A301D5
:108C900092010F94D54AA1966CAF7DAF8EAF9FAF76
:108CA000A197C058DF4F288139814A815B81C05824
:108CB000D040CA01B9010F94D54A20E030E040E825
:108CC0005EE30F94EE46C251DF4F688379838A8357
:108CD0009B83CE5ED04020E030E040E85EE3EC963F
:108CE0006CAD7DAD8EAD9FADEC970F94EE46CE5042
:108CF000DF4F688379838A839B83C25FD04020E003
:108D000030E040E85EE3C857DF4F688179818A81AF
:108D10009B81C858D0400F94EE46CA50DF4F6883FD
:108D200079838A839B83C65FD040C457DF4F2881F5
:108D300039814A815B81CC58D040CA01B9010F9476
:108D4000D54A20E030E040E85EE30F94EE46C6509E
:108D5000DF4F688379838A839B83CA5FD040CE507C
:108D6000DF4F288139814A815B81C25FD040C25187
:108D7000DF4F688179818A819B81CE5ED0400F94DC
:108D8000D44AA50194010F94D44ACA50DF4F2881D8
:108D900039814A815B81C65FD0400F94D54AC65065
:108DA000DF4F288139814A815B81CA5FD0400F94AF
:108DB000D44AA70196010F94D54AC458DF4F2881A1
:108DC00039814A815B81CC57D0400F94EE46A30194
:108DD00092010F94D54AA5966CAF7DAF8EAF9FAF31
:108DE000A597CC57DF4F288139814A815B81C458D0
:108DF000D040CA01B9010F94D54A20E030E040E8E4
:108E00005EE30F94EE464B015C01C057DF4F2881B3
:108E100039814A815B81C059D040CA01B9010F94A0
:108E2000D54A20E030E040E85EE30F94EE466B0167
:108E30007C01CE50DF4F688179818A819B81C25F3E
:108E4000D0409058CE51DF4F288139814A815B81D3
:108E5000C25ED0400F94D44AA50194010F94D54A24
:108E6000CA50DF4F288139814A815B81C65FD0407B
:108E70000F94D54AC651DF4F288139814A815B81E1
:108E8000CA5ED0400F94D54AA70196010F94D44AE8
:108E9000C458DF4F288139814A815B81CC57D0404B
:108EA0000F94EE46A30192010F94D54AA9966CAF98
:108EB0007DAF8EAF9FAFA997C251DF4F2881398117
:108EC0004A815B81CE5ED040C754DF4F6881798193
:108ED0008A819B81C95BD0400F94D54AA50194013A
:108EE0000F94D54ACA51DF4F288139814A815B816D
:108EF000C65ED0400F94D54AC650DF4F28813981D5
:108F00004A815B81CA5FD0400F94D54AA701960180
:108F10000F94D54A6B017C0120E030E040E451E43D
:108F2000CD55DF4F688179818A819B81C35AD040BA
:108F30000F94EE4620E030E040E85EE30F94EE460A
:108F40009B01AC01C701B6010F94D44AC155DF4F54
:108F5000288139814A815B81CF5AD0400F94EE46F7
:108F60004B015C01CD54DF4F9881C35BD040992306
:108F700009F41FC2C555DF4F288139814A815B81C1
:108F8000CB5AD0406AE077ED83E29CE30F94B14B7B
:108F900020E030E040E450E40F94B14BC458DF4F80
:108FA000688379838A839B83CC57D04020E030E06C
:108FB00040E850E4C058DF4F688179818A819B8105
:108FC000C058D0400F94EE4620E030E040E85EE329
:108FD0000F94EE46C555DF4F688379838A839B8360
:108FE000CB5AD04020E030E040E850E4CC57DF4F8F
:108FF000688179818A819B81C458D0400F94EE4664
:1090000020E030E040E85EE30F94EE462B013C01A7
:1090100020E030E040E850E4C457DF4F68817981B8
:109020008A819B81CC58D0400F94EE4620E030E0FE
:1090300040E85EE30F94EE46C155DF4F68837983C5
:109040008A839B83CF5AD04020E030E040E850E450
:10905000C057DF4F688179818A819B81C059D04098
:109060000F94EE4620E030E040E85EE30F94EE46D9
:10907000C754DF4F688379838A839B83C95BD04061
:1090800020E030E0A901CD55DF4F688179818A81E8
:109090009B81C35AD0400F94EE4620E030E040E878
:1090A0005EE30F94EE46CD55DF4F688379838A8364
:1090B0009B83C35AD04020E030E0A901EC966CAD10
:1090C0007DAD8EAD9FADEC970F94EE4620E030E085
:1090D00040E85EE30F94EE46C555DF4F28813981A5
:1090E0004A815B81CB5AD0400F94D44AA3019201AC
:1090F0000F94D54A6B017C0120E030E0A901C857EC
:10910000DF4F688179818A819B81C858D0400F9454
:10911000EE4620E030E040E85EE30F94EE469B012F
:10912000AC01C701B6010F94D54AC155DF4F288164
:1091300039814A815B81CF5AD0400F94D44AC754B9
:10914000DF4F288139814A815B81C95BD0400F9410
:10915000D54ACD55DF4F288139814A815B81C35A79
:10916000D0400F94D54AC458DF4F288139814A81B5
:109170005B81CC57D0400F94EE4665966CAF7DAFC7
:109180008EAF9FAF659720E030E040E850E4EC966A
:109190006CAD7DAD8EAD9FADEC970F94EE4620E0AB
:1091A00030E040E85EE30F94EE46EC966CAF7DAFA6
:1091B0008EAF9FAFEC9720E030E040E850E4C85716
:1091C000DF4F688179818A819B81C858D0400F9494
:1091D000EE4620E030E040E85EE30F94EE466B019F
:1091E0007C0120E030E0A901C058DF4F688179811F
:1091F0008A819B81C058D0400F94EE4620E030E039
:1092000040E85EE30F94EE46EC962CAD3DAD4EADDE
:109210005FADEC970F94D54AA30192010F94D44A05
:10922000A70196010F94D54A2B013C0120E030E0C4
:10923000A901C457DF4F688179818A819B81CC580D
:10924000D0400F94EE4620E030E040E85EE30F941B
:10925000EE469B01AC01C301B2010F94D54AC7543D
:10926000DF4F288139814A815B81C95BD0400F94EF
:10927000D44ACD55DF4F288139814A815B81C35A59
:10928000D0400F94D54AC458DF4F288139814A8194
:109290005B81CC57D0400F94EE4669966CAF7DAFA2
:1092A0008EAF9FAF699720E030E0A901CC57DF4F28
:1092B000688179818A819B81C458D0400F94EE46A1
:1092C00020E030E040E85EE30F94EE462B013C01E5
:1092D000EC962CAD3DAD4EAD5FADEC97C555DF4F77
:1092E000688179818A819B81CB5AD0400F94D44A7E
:1092F0009B01AC01C301B2010F94D54AA7019601AD
:109300000F94D44AC155DF4F288139814A815B814E
:10931000CF5AD0400F94D54A6B017C0120E030E059
:10932000A901C057DF4F688179818A819B81C0592B
:10933000D0400F94EE4620E030E040E85EE30F942A
:10934000EE469B01AC01C701B6010F94D54ACD553D
:10935000DF4F288139814A815B81C35AD0400F9405
:10936000D54AC458DF4F288139814A815B81CC5767
:10937000D0400F94EE466D966CAF7DAF8EAF9FAF31
:109380006D9717C0812C912C5401CB56DF4F18825A
:10939000C559D040CA56DF4F1882C659D040C95669
:1093A000DF4F1882C759D040C856DF4F1882C859BE
:1093B000D0407E01ADE5EA0EF11C03EA1EE0F701A4
:1093C00021913191419151917F01D8016D917D9110
:1093D0008D919C910F94D54AF8016193719381937B
:1093E00091938F01FEE00F3A1F0749F7A501940101
:1093F00060914D1070914E1080914F1090915010CF
:109400000F94D54A60934D1070934E1080934F1077
:10941000909350107E0121E5E20EF11C01E510E170
:10942000D7012D913D914D915D917D01F8016081B4
:109430007181828193810F94D54AD8016D937D9378
:109440008D939D938D01B0E10D351B0749F7A5C0A4
:10945000AF962FADAF97E3963FADE397E7964FAD4D
:10946000E797E8965FADE897CB56DF4F6881C5591F
:10947000D040CA56DF4F7881C659D040C956DF4F19
:109480008881C759D040C856DF4F9881C859D0400D
:109490000F94894618160CF480C0C452DF4F88819F
:1094A0009981AA81BB81CC5DD0408093A30E90931B
:1094B000A40EA093A50EB093A60ECC52DF4F8881C8
:1094C0009981AA81BB81C45DD0408093A70E9093FF
:1094D000A80EA093A90EB093AA0EC453DF4F8881A3
:1094E0009981AA81BB81CC5CD0408093AB0E9093D4
:1094F000AC0EA093AD0EB093AE0EC054DF4F88817A
:109500009981AA81BB81C05CD04080934D1090931B
:109510004E10A0934F10B0935010CC53DF4F888162
:109520009981AA81BB81C45CD0408093850E9093C1
:10953000860EA093870EB093880EC853DF4F8881A4
:109540009981AA81BB81C85CD040809351109093CF
:109550005210A0935310B0935410C852DF4F88811B
:109560009981AA81BB81C85DD040809355109093AA
:109570005610A0935710B0935810C053DF4F8881F6
:109580009981AA81BB81C05DD0408093591090938E
:109590005A10A0935B10B0935C10C656DF4F9881B1
:1095A000CA59D040911148C00F943723AF962FADC0
:1095B000AF97E3963FADE397E7964FADE797E89611
:1095C0005FADE897C156DF4F6881CF59D040C05694
:1095D000DF4F7881C05AD040CF55DF4F8881C15AC4
:1095E000D040CE55DF4F9881C25AD0400F94494D9C
:1095F00018160CF0BEC0AF96AFADAF97C156DF4F97
:10960000A883CF59D040E396BFADE397C056DF4F54
:10961000B883C05AD040E796EFADE797CF55DF4FFC
:10962000E883C15AD040E896FFADE897CE55DF4FAA
:10963000F883C25AD0409DC0C955DF4F2881C75A10
:10964000D040211123C06090AB0E7090AC0E809082
:10965000AD0E9090AE0EA090A70EB090A80E009107
:10966000A90E1091AA0EC090A30ED090A40EE09067
:10967000A50EF090A60E9501A801B301C4010F94A8
:10968000894687FD42C0530184013FC020E030E09D
:10969000A9016091511070915210809153109091D6
:1096A00054100F94D54A2091551030915610409186
:1096B0005710509158100F94D54A2091591030915D
:1096C0005A1040915B1050915C100F94D54A20E0E5
:1096D00030E040E450E40F94B14B6B017C0101E5B4
:1096E00010E1A7019601D8016D917D918D919C911A
:1096F0000F94D44AF80161937193819391938F01F0
:10970000F0E10D351F0769F79ECF9501A801B6015D
:10971000C7010F94494D181614F0650178019601A0
:10972000A7016091850E7091860E8091870E9091B1
:10973000880E0F94D44A6093850E7093860E8093A2
:10974000870E9093880E03EA1EE09601A701D801C8
:109750006D917D918D919C910F94D44AF801619304
:109760007193819391938F01FEE00F3A1F0769F780
:109770001BCFC656DF4F2881CA59D040233009F08D
:1097800051C08AE797E00E940460BE01635E7F4F8C
:1097900088E797E025D4C855DF4F8881C85AD04064
:1097A000882319F1BE016F5D7F4F85E797E018D4DC
:1097B000BE01675D7F4F82E797E012D4BE016F5C08
:1097C0007F4F8FE697E00CD4C655DF4F9881CA5A79
:1097D000D040992319F18AE00E94F35F8EE20E9443
:1097E000F35F8DE00E94FA5F07C0C655DF4FA88186
:1097F000CA5AD040AA2391F0BE01635D7F4F8CE628
:1098000097E0EED3BE016B5C7F4F89E697E0E8D32B
:10981000BE016B5D7F4F86E697E0E2D38AE00E944F
:10982000F35F08C0C656DF4FB881CA59D040BB238A
:1098300009F4AEC1AF962FADAF97E3963FADE39776
:10984000E7964FADE797E8965FADE897CB56DF4FC9
:109850006881C559D040CA56DF4F7881C659D0407B
:10986000C956DF4F8881C759D040C856DF4F98810D
:10987000C859D0400F94894618166CF0C254DF4F77
:10988000E881CE5BD040CC56DF4FF881C459D04040
:10989000EF17CCF046C0AF962FADAF97E3963FAD34
:1098A000E397E7964FADE797E8965FADE897CC541E
:1098B000DF4F688179818A819B81C45BD0400F949E
:1098C000494D87FD01C189E198E00E94046080E272
:1098D0000E94FA5FAF962FADAF97E3963FADE39747
:1098E000E7964FADE797E8965FADE897CB56DF4F29
:1098F0006881C559D040CA56DF4F7881C659D040DB
:10990000C956DF4F8881C759D040C856DF4F98816C
:10991000C859D0400F948946181614F508E113E091
:1099200030C0AF962FADAF97E3963FADE397E79684
:109930004FADE797E8965FADE897CC54DF4F68816D
:1099400079818A819B81C45BD0400F94494D87FD0A
:10995000BBC089E198E00E94046080E20E94FA5F47
:10996000C755DF4F2881C95AD0402111D7CFAE96B5
:109970008FADAE97882391F28BE098E00E9404604F
:109980001FC0D8018D918D01882319F00E94F35FCB
:10999000F8CF43E0C156DF4F6881CF59D040C05661
:1099A000DF4F7881C05AD040CF55DF4F8881C15AF0
:1099B000D040CE55DF4F9881C25AD0400E943C61C2
:1099C0008AE00E94F35F6BEF77E0C1010F94D2450C
:1099D00020E030E040E85FE3C156DF4F6881CF59B7
:1099E000D040C056DF4F7881C05AD040CF55DF4FAE
:1099F0008881C15AD040CE55DF4F9881C25AD0409D
:109A00000F94894687FF21C020E030E04AE754E404
:109A1000C156DF4F6881CF59D040C056DF4F7881A3
:109A2000C05AD040CF55DF4F8881C15AD040CE5563
:109A3000DF4F9881C25AD0400F94EE460F94544D98
:109A40007F936F9384EF97E01AC0C156DF4F688110
:109A5000CF59D040C056DF4F7881C05AD040CF5543
:109A6000DF4F8881C15AD040CE55DF4F9881C25A0E
:109A7000D0400F94544D7F936F938DEE97E09F935A
:109A80008F93CE0140969F938F930F9423460F9010
:109A90000F900F900F900F900F9060E0C1010E9407
:109AA0002F73C955DF4F6881C75AD040C854DF4F64
:109AB0008881C85BD040BDD28FEB97E00E940460E4
:109AC0008AE00E94F35FE3C0CC56DF4FB881C459EF
:109AD000D040BF31C4F48B2F0B2E000C990B9F93F9
:109AE000BF938EEA97E09F938F933F922F920F94AC
:109AF00023460F900F900F900F900F900F908E01B4
:109B00000F5F1F4F06C06FE977E0C1010F94D24588
:109B1000F6CFF80181918F01882319F00E94F35F3D
:109B2000F8CF80E20E94FA5F08E113E0D8018D913E
:109B30008D01882319F00E94F35FF8CF43E0AF96C0
:109B40006FADAF97E3967FADE397E7968FADE7975D
:109B5000E8969FADE8970E943C618AE00E94F35F1F
:109B600060E0C1010E942F73C656DF4FB881CA5909
:109B7000D040B23008F48BC0C955DF4F6881C75A56
:109B8000D040C854DF4F8881C85BD04052D27FC0DC
:109B900083E997E00E94046083E20E94FA5F08E193
:109BA00013E0F80181918F01882319F00E94F35F7F
:109BB000F8CF43E0AF966FADAF97E3967FADE397F5
:109BC000E7968FADE797E8969FADE8970E943C61D6
:109BD0008AE00E94F35F63E977E0C1010F94D24508
:109BE0006EE877E0CE010C960F94D24520E030E08D
:109BF00040E85FE3AF966FADAF97E3967FADE39735
:109C0000E7968FADE797E8969FADE8970F94894662
:109C100087FF19C020E030E04AE754E4AF966FAD0B
:109C2000AF97E3967FADE397E7968FADE797E8961A
:109C30009FADE8970F94EE460F94544D7F936F932A
:109C400087E897E012C0AF966FADAF97E3967FAD10
:109C5000E397E7968FADE797E8969FADE8970F9467
:109C6000544D7F936F9380E897E09F938F93CE013D
:109C700040969F938F930F9423460F900F900F90D1
:109C80000F900F900F9060E0C1010E942F7381E050
:109C90008093FD0C0F940C210F9426218091FC0CD5
:109CA0008093FD0CAF962FADAF97E3963FADE39752
:109CB000E7964FADE797E8965FADE897CB56DF4F55
:109CC0006881C559D040CA56DF4F7881C659D04007
:109CD000C956DF4F8881C759D040C856DF4F988199
:109CE000C859D0400F94494D18163CF4CC56DF4F5C
:109CF000F881C459D040FF316CF0C254DF4F288145
:109D0000CE5BD040CC56DF4F8881C459D040281755
:109D10000CF452C0C556DF4FE880CB59D040C45632
:109D2000DF4FF880CC59D040C356DF4F0881CD5962
:109D3000D040C256DF4F1881CE59D040AF962FADDC
:109D4000AF97E3963FADE397E7964FADE797E89679
:109D50005FADE897CC54DF4F688179818A819B8120
:109D6000C45BD0400F94894687FF26C0AF969FAD55
:109D7000AF97C556DF4F9883CB59D040E396AFAD30
:109D8000E397C456DF4FA883CC59D040E796BFADC8
:109D9000E797C356DF4FB883CD59D040E896EFAD73
:109DA000E897C256DF4FE883CE59D0400C94623B0F
:109DB00088E298E00E9404609FD14FC0C655DF4FF3
:109DC0001882CA5AD040C855DF4F1882C85AD040AE
:109DD00010E00C943339CD54DF4FE881C35BD040A1
:109DE000EE2391F0C756DF4FF881C959D040C855CE
:109DF000DF4FF883C85AD040C655DF4FF883CA5AA0
:109E0000D0401F2F0C943A39C756DF4F1881C959DB
:109E1000D040C855DF4F1882C85AD0400C942D3915
:109E2000C655DF4F1882CA5AD040C855DF4F188236
:109E3000C85AD04010E0F1E0C755DF4FF883C95A47
:109E4000D040C854DF4F1882C85BD040C955DF4F9F
:109E50001882C75AD0400C945839CD5FDE4F0FB6E8
:109E6000F894DEBF0FBECDBFDF91CF911F910F9150
:109E7000FF90EF90DF90CF90BF90AF909F908F902A
:109E80007F906F905F904F903F902F9008952F920A
:109E90003F924F925F926F927F928F929F92AF927A
:109EA000BF92CF92DF92EF92FF920F931F93CF93C7
:109EB000DF93CDB7DEB72D970FB6F894DEBF0FBE98
:109EC000CDBF9E012F5F3F4F19012CE0F101119290
:109ED0002A95E9F78B016C0186E9E82EF12C1D86A5
:109EE000B7010F2C000C880B990B0F948F462BEDAC
:109EF0003FE049E450E40F94EE4620E030E044E3D4
:109F000053E40F94B14B2B013C01FD85FF2349F035
:109F10008090AA149090AB14A090AC14B090AD14A3
:109F200003C0812C912C5401C301B2010F94AE4B9C
:109F30009B01AC01C501B4010F94EE4669837A839D
:109F40008B839C83C301B2010F94844D9B01AC01B0
:109F5000C501B4010F94EE466D837E838F8398878D
:109F6000F60181919191A191B1916F0189879A87B1
:109F7000AB87BC87C1010F940022EEE7F6E0D80161
:109F800041915191619171914D935D936D937D9349
:109F900026E0EA38F207A1F73D853F5F3D878CE375
:109FA000E80EF11C045F1F4F373009F099CF2D9652
:109FB0000FB6F894DEBF0FBECDBFDF91CF911F91DA
:109FC0000F91FF90EF90DF90CF90BF90AF909F9058
:109FD0008F907F906F905F904F903F902F9008955B
:109FE0000F931F93CF93DF938C01EB018FE69BE0E0
:109FF0000E940460C8010E9404608AE30E94F35F2B
:10A0000020E030E0A901688179818A819B810F94E9
:10A01000494D87FD03C08BE20E94F35F688179811F
:10A020008A819B8142E0DF91CF911F910F910C9427
:10A030003C61CF93DF93D82FC62F4091850E50916E
:10A04000860E6091870E7091880E88E99BE00E94D1
:10A05000AD61DD23A1F163EA7EE085E99BE0C0DF2D
:10A0600067EA7EE082E99BE0BBDF6BEA7EE08FE897
:10A070009BE0B6DFC1110DC040914D1050914E10C4
:10A0800060914F107091501082E79BE00E94AD618B
:10A090002EC040914D1050914E1060914F10709114
:10A0A000501085E89BE00E94AD618AE00E94F35F5A
:10A0B0008EE20E94F35F8DE00E94FA5F02C0CC2323
:10A0C000B1F061E570E182E89BE08ADF65E570E16F
:10A0D0008FE79BE085DF69E570E18CE79BE080DF3F
:10A0E000D11103C0C111C8CF02C0CC2329F28AE02C
:10A0F000DF91CF910C94F35FCF93DF9300D01F9249
:10A10000CDB7DEB719821A821B821C82BE016F5F37
:10A110007F4F8BE492E00E94CCD480E00E941FE24B
:10A1200080919F0E9091A00EA091A10EB091A20ED1
:10A130008093470290934802A0934902B0934A0249
:10A1400080919D0E90919E0E90931C0280931B0215
:10A150000F900F900F900F90DF91CF910895CF93B4
:10A16000C62F0E94B4EF882319F0CF910C9477EE9C
:10A170008C2FCF91089580E1EDE6F6E0ADE8BEE0EA
:10A1800001900D928A95E1F7089580914510909184
:10A190004610892B39F00E9477EE91E0811103C0BF
:10A1A00090E001C091E0892F08952F923F924F9245
:10A1B0005F926F927F928F929F92AF92BF92CF9257
:10A1C000DF92EF92FF920F931F93CF93DF93CDB760
:10A1D000DEB762970FB6F894DEBF0FBECDBF83E542
:10A1E0000E94BFEE882341F0D0DF182F811106C0F6
:10A1F00080E00E9487F402C010917D0680916D0678
:10A2000090916E06A0916F06B091700689839A8333
:10A21000AB83BC838091710690917206A091730606
:10A22000B09174068D839E83AF83B8878091750645
:10A2300090917606A0917706B091780689879A87E3
:10A24000AB87BC8786E50E94BFEE682E809198148C
:10A2500090919914892B09F4ABC083E40E94BFEE5E
:10A26000882309F4B0C00E9488EE1B012C01712CD8
:10A27000812C68EC962E72ECA72EB12CC12C28EC08
:10A280002F8732E4388B89E08D879D8591509D879B
:10A290009F3FD9F1E9E0EE8739E0399F9001112421
:10A2A0003A8B298B3E8531503E873F3F71F3E989D8
:10A2B000FA89E30FF11DEE0FFF1FEE0FFF1FE255AE
:10A2C000FB4ED080E180F28003812B2D3C2D4F8509
:10A2D00058896D2D7E2D8F2D902F0F94894687FFE5
:10A2E00004C0BD2CCE2CFF86088B2D2D3E2D4F2D6E
:10A2F000502F672D782D892D9A2D0F94894687FF31
:10A30000D1CF7D2C4701A02ECDCF272D382D492D23
:10A310005A2D6B2D7C2D8F8598890F94D54A20E07E
:10A3200030E040E05FE30F94EE46A20191010F940C
:10A33000D54A1B012C012DEB37E346E855EB0F9472
:10A34000494D87FD0AC02DEB37E346E855E3C201CE
:10A35000B1010F9489461816B4F580E00E9487F485
:10A3600039E0D32E49E0C42EDA949FEFD91659F183
:10A3700009E0CD9C500111240150B0F37501E00EAD
:10A38000F11CC701880F991F880F991FFC01E25526
:10A39000FB4E7F01A20191016081718182819381D5
:10A3A0000F94D44AF7016083718382839383E4CF4F
:10A3B000111102C0662089F00E9423608DED9AE0A1
:10A3C0000E9404600DC0662041F080919814909125
:10A3D0009914892B11F00E946BF2812F0E9487F44F
:10A3E000112351F080917D06811106C00E942360E7
:10A3F0008EEB9AE00E9404600E94486080EB9AE035
:10A400000E94046080917D06811103C089EA9AE070
:10A4100002C08DEA9AE00E9404608AE00E94F35F25
:10A420004CE050E06DE676E0CE0101960F94324E9E
:10A43000892BD1F062960FB6F894DEBF0FBECDBF68
:10A44000DF91CF911F910F91FF90EF90DF90CF9010
:10A45000BF90AF909F908F907F906F905F904F9044
:10A460003F902F900D94161F62960FB6F894DEBFA2
:10A470000FBECDBFDF91CF911F910F91FF90EF9055
:10A48000DF90CF90BF90AF909F908F907F906F9014
:10A490005F904F903F902F900895CF93DF93C82FF8
:10A4A000D62F0E94B4EF882319F0DF91CF916DCEA3
:10A4B0008C2F0E94BFEE811101C08D2FDF91CF91B3
:10A4C00008951F93CF93DF9300D01F92CDB7DEB7CF
:10A4D00060E08FE4E2DF882329F080917F0F8770AE
:10A4E000873049F10E94D1C810917D0680E00E941A
:10A4F00087F40E9420CF81E08093FD0C0F940C2103
:10A500000F9426218091FC0C8093FD0C19821A82F5
:10A510001B821C82BE016F5F7F4F8BE492E00E9422
:10A52000CCD4812F0E9487F40E940FD383E08093C4
:10A5300050020F94161F0F900F900F900F90DF9105
:10A54000CF911F9108950E9467EECB010895CF939C
:10A55000DF93EB010E94B4EF882319F0DF91CF91D4
:10A56000F2CFCE01DF91CF9108952F923F924F927B
:10A570005F926F927F928F929F92AF92BF92CF9293
:10A58000DF92EF92FF920F931F93CF93DF93CDB79C
:10A59000DEB7A9970FB6F894DEBF0FBECDBF1091FE
:10A5A0007D0687E50E94BFEE882309F4E9C080910B
:10A5B000981490919914892B29F40E9423608DE5B9
:10A5C0009BE034C08AE50E94B4EF882379F00E94B2
:10A5D00088EE2091EB0E3091EC0E4091ED0E5091F3
:10A5E000EE0E0F94D44A4B015C0108C080907506B2
:10A5F00090907606A0907706B090780620E030E044
:10A6000040E251ECC501B4010F94494D87FD0AC0E9
:10A6100020E030E040E251E4C501B4010F948946E6
:10A6200018163CF40E94236080E59BE00E940460C1
:10A6300088C440E050E060EC7FE788E50E9468DB7A
:10A640002091E30E3091E40E4091E50E5091E60E1C
:10A650000F94D44A6B017C0140E050E060EC7FE74E
:10A6600089E50E9468DB2091E70E3091E80E409169
:10A67000E90E5091EA0E0F94D44A2B013C016FEF82
:10A6800089E46DDD082F6FEF8AE469DD382EA701BC
:10A690009601C701B6010F94CF4D81114EC0A301A1
:10A6A0009201C301B2010F94CF4D811146C0609158
:10A6B000B1057091B205072E000C880B990B0F9411
:10A6C0008F469B01AC01C701B6010F94D44A20E02C
:10A6D00030E0A9010F94D54A20E030E0A9010F94A1
:10A6E000B14B0F94194C062F6091B3057091B405CE
:10A6F000072E000C880B990B0F948F469B01AC0121
:10A70000C301B2010F94D44A20E030E0A9010F94B4
:10A71000D54A20E030E0A9010F94B14B0F94194CB9
:10A72000E02F09300CF0E8E00E2FE7FD00E0693083
:10A730000CF068E0362E67FD312C093008F001C4BA
:10A7400029E0231508F4FDC380E00E9487F439E076
:10A750000302F0011124E30DF11D37FCFA95EE0F11
:10A76000FF1FEE0FFF1FE255FB4E80829182A282F7
:10A77000B382812F0E9487F4112309F4E2C3BCC085
:10A780008AE40E94BFEE882309F4B9C00E94CCF489
:10A79000D8C329853A85C21AD30AD7FE03C037E049
:10A7A000C30ED11C43E0D594C7944A95E1F7B60196
:10A7B0000D2C000C880B990B0F948F46698F7A8FA4
:10A7C0008B8F9C8FE618F708F7FE03C087E0E80E32
:10A7D000F11C33E0F594E7943A95E1F7B7010F2CBB
:10A7E000000C880B990B0F948F466D8F7E8F8F8F87
:10A7F00098A30E9420CF6091981470919914072E0D
:10A80000000C880B990B0F948F469B01AC01698D4E
:10A810007A8D8B8D9C8D0F948946811148C26091F1
:10A820009A1470919B14072E000C880B990B0F94AF
:10A830008F469B01AC016D8D7E8D8F8D98A10F94FD
:10A840008946811134C28091B1059091B205A985E4
:10A85000BA85A817B90709F02AC28091B30590916B
:10A86000B4056816790609F022C260E085E415DEB9
:10A87000882309F432C2F1E0F9A3212C312CC12C38
:10A88000D12C760131E03E8B81E0888F99E09F8B5F
:10A890001986FE8921E0F227FE8BC101032C000CF2
:10A8A000AA0BBB0B8EA39FA3A8A7B9A79F89A985B5
:10A8B0009A1316C2F8E02F16310449F0A701960149
:10A8C000C701B6010F94CF4D882309F410C380E06F
:10A8D0000E941FE2882309F4B3C2812F0E9487F4EB
:10A8E0000E940FD381E08093810F80917D068111BA
:10A8F0000F94141F0E94D7E10F94161F22C360E02B
:10A9000070E086E524DE9C878B87059718F088E247
:10A910009BE08CCE60E084E4C0DD8D8740E050E0B9
:10A92000BA018AE50E9468DB6AA37BA38CA39DA37E
:10A9300040E050E86BEB75E483E50E9468DB20E0C3
:10A9400030E040E752E40F94B14B609343027093C0
:10A950004402809345029093460288E40E94BFEE31
:10A96000882309F482C00E9488EE0F94194C4B0191
:10A970005C0177FF02C06F5F7F4F7595679571959A
:10A9800061957109072E000C880B990B0F948F4667
:10A99000762EE72EF82E092F20E030E04AEC52EC1C
:10A9A0000F94494D18162CF4572D4E2D3F2D202F66
:10A9B00004C050E040E03AEC22EC652F742F832F66
:10A9C000922F0F94194C7A876987680D791D072E8D
:10A9D000000C880B990B0F948F461B012C0120E073
:10A9E00030E04AEC52E40F94894687FD06C0212CE2
:10A9F000312CAAEC4A2EA2E45A2EC201B1010F94C6
:10AA0000194C6B0120E030E04AEC52EC672D7E2DB2
:10AA10008F2D902F0F94494D18162CF0712CE12C8E
:10AA2000FAECFF2E02EC672D7E2D8F2D902F0F94C8
:10AA3000194C3B01680D791D072E000C880B990BF2
:10AA40000F948F464B015C0120E030E04AEC52E469
:10AA50000F94894687FD06C0812C912CEAECAE2E1E
:10AA6000E2E4BE2EC501B4015CC08CE40E94B4EFE8
:10AA7000882389F00E9488EE2091E30E3091E40E45
:10AA80004091E50E5091E60E0F94D44A0F94194C64
:10AA90007A87698704C08BE99FEF9A87898782E567
:10AAA0000E94B4EF882381F00E9488EE2091E30E8B
:10AAB0003091E40E4091E50E5091E60E0F94D44A89
:10AAC0000F94194C6B0103C075E6C72ED12C86E498
:10AAD0000E94B4EF882381F00E9488EE2091E70E57
:10AAE0003091E80E4091E90E5091EA0E0F94D44A4D
:10AAF0000F94194C3B0104C06BE9662E77247A94BD
:10AB000082E40E94B4EF882381F00E9488EE2091B5
:10AB1000E70E3091E80E4091E90E5091EA0E0F9445
:10AB2000D44A0F94194C7B0103C055E6E52EF12C55
:10AB3000A985BA85BD01BB0F880B990B0F948F4671
:10AB40006E877F87888B998B9B01AC010F94EE46B3
:10AB500020E030E0A9010F94D54A4B015C0120E0D0
:10AB600030E442E556E40F948946181674F120E06B
:10AB700034E64FE156E4C501B4010F948946181636
:10AB800024F1B6010D2C000C880B990B0F948F4605
:10AB90009B01AC010F94EE4620E030E0A9010F9438
:10ABA000D54A4B015C0120E030E442E556E40F94C5
:10ABB0008946181654F020E034E64FE156E4C5010A
:10ABC000B4010F94894618161CF48CE09BE02ECD3E
:10ABD000B301072C000C880B990B0F948F466A8BDE
:10ABE0007B8B8C8B9D8B9B01AC010F94EE4620E000
:10ABF00030E0A9010F94D54A4B015C0120E030E41C
:10AC000042E556E40F9489461816FCF220E034E63B
:10AC10004FE156E4C501B4010F9489461816ACF211
:10AC2000B7010F2C000C880B990B0F948F469B01DA
:10AC3000AC010F94EE4620E030E0A9010F94D54A14
:10AC40004B015C0120E030E442E556E40F94894674
:10AC500018160CF4BACF20E034E64FE156E4C501F3
:10AC6000B4010F94894618160CF4AFCFEB85FC8520
:10AC7000EF2B71F086EF9AE00E940460FD85FF23C0
:10AC800021F08CEE9AE00E9404608AE00E94F35F5B
:10AC90000E94D1C880E00E9487F481E00E941FE2F8
:10ACA000882309F476CD812F0E9487F44AC10E943F
:10ACB000CCF4D0929914C0929814F0929B14E09224
:10ACC0009A14E985FA85F093B205E093B105709284
:10ACD000B4056092B30510E0C8CD22E029A3CDCD24
:10ACE0006A2FAA0F770B880B990B0F948F46298D2B
:10ACF0003A8D4B8D5C8D0F94EE462E853F854889AD
:10AD000059890F94D54A2B013C016EA17FA188A5DA
:10AD100099A50F948F462D8D3E8D4F8D58A10F9480
:10AD2000EE462A893B894C895D890F94D54A4B01AF
:10AD30005C0120E030E0A901C301B2010F94894613
:10AD400087FF04C020E030E0A90104C020E030E02B
:10AD500040E05FE3C301B2010F94D54A0F944A4C1F
:10AD60002B013C0169837A838B839C8320E030E054
:10AD7000A901C501B4010F94894687FF04C020E0F2
:10AD800030E0A90104C020E030E040E05FE3C5010D
:10AD9000B4010F94D54A0F944A4C4B015C016D836A
:10ADA0007E838F839887A3019201C301B2010F9420
:10ADB000EE462B013C01A5019401C501B4010F949D
:10ADC000EE469B01AC01C301B2010F94D54A4B0181
:10ADD0005C0120E030E442E556E40F948946181601
:10ADE00054F120E034E64FE156E4C501B4010F947C
:10ADF0008946181604F18EC029E039853203800196
:10AE00001124020D131D000F111F000F111F0255F9
:10AE10001B4EA70196016AA17BA18CA19DA10F9455
:10AE2000D54AD8016D937D938D939C93139780E0C1
:10AE30000E94746210E0B88DE985BE0FB98736CDE7
:10AE4000A7019601C701B6010F94CF4D811148CDDE
:10AE50002D85222309F10E946BF20E94FEF13D85AF
:10AE6000311142C08DE696E00E94E7EF9B01AC01F4
:10AE700060917506709176068091770690917806BC
:10AE80000F94D44A60937506709376068093770684
:10AE90009093780611E028C004E098E0E92E84E061
:10AEA000F82EDE2CD01ACE2CCF1821E041E06F2DE9
:10AEB000802F0E94F3F221E04FEF6F2D8D2D0E9425
:10AEC000F3F22FEF41E06C2D802F0E94F3F22FEF71
:10AED0004FEF6C2D8D2D0E94F3F2FA948FEFF81244
:10AEE000E2CF0150E0F6B7CF10937D06F9CC9E89F2
:10AEF000992349F0A1E0A88FB9E0BF8B1986EFEF45
:10AF00002E1A3E0AC6CCAFEFA88FBFEFBF8BE8E08A
:10AF1000E987F5CF01E02B8549A1BE016B5F7F4F2B
:10AF2000CE0101960E9406E36B017C019B01AC01FE
:10AF30000F94CF4D882309F45FCF812F0E9487F4AF
:10AF4000C6CCA9960FB6F894DEBF0FBECDBFDF9179
:10AF5000CF911F910F91FF90EF90DF90CF90BF9016
:10AF6000AF909F908F907F906F905F904F903F90A9
:10AF70002F900895E091810EF0E0EF51F34F808122
:10AF8000882339F08AE499E00E9404608AE00C94F6
:10AF9000F35F0895E7E0F4E0808181838DE499E038
:10AFA0000E9404608091890490918A04A0918B048E
:10AFB000B0918C04BC01CD016F5F7F4F8F4F9F4FCD
:10AFC0000E9417610E94BC61D5CF0F931F93CF934E
:10AFD0008C01C62F0E942360C8010E94046060910A
:10AFE000890470918A0480918B0490918C040E9452
:10AFF00017610E94BC61CEDFEC2FF0E0EE0FFF1F67
:10B00000EF50FB4F11821082CF911F910F91089545
:10B01000CF93DF93EC01CE010F942437811103C04D
:10B020000E947462F8CFDF91CF910895DF92EF9282
:10B03000FF920F931F93CF93DF93CDB7DEB7EC97BB
:10B040000FB6F894DEBF0FBECDBF6091F1057091D1
:10B05000F2056115710549F14BE350E0CE0101960F
:10B060007C010F94FA451CAEF7018F010E191F09E0
:10B07000D190DD2019F09AE0D912F7CFF701E00F57
:10B08000F11F1082C7010F942437882371F0DD204F
:10B09000A9F00F5F1F4F8091F1059091F205080F05
:10B0A000191F1093F2050093F10581E02091F1053D
:10B0B0003091F205232B29F480E003C000E010E07A
:10B0C000F0CFEC960FB6F894DEBF0FBECDBFDF9188
:10B0D000CF911F910F91FF90EF90DF9008954F92C5
:10B0E0005F926F927F929F92AF92BF92CF92DF92C8
:10B0F000EF92FF920F931F93CF93DF931F92CDB7E1
:10B10000DEB794DF811151C28091830E843008F044
:10B110002EC18091070490910804891B8F7709F450
:10B1200026C10E94CB619C0197FDEECF0091F104F6
:10B130001091F2048A3019F08D3009F0E9C01092B4
:10B14000F3040115110519F40F942633DDCFF8012E
:10B15000EF56FB4F10821092F2041092F10401E9B5
:10B1600014E0F8018191803211F48F01FACF8E340E
:10B1700009F07AC00115110509F476C06DE77AE08F
:10B18000C8010F9409467C01892B41F06EE470E000
:10B19000C80104960F94664E009709F4C8014AE06E
:10B1A00050E060E070E001960F948C4360938D0452
:10B1B00070938E0480938F04909390044090890440
:10B1C00050908A0460908B0470908C042FEF421A88
:10B1D000520A620A720A641575058605970531F0F0
:10B1E000EF2821F460E08AE49AE04CC06AE270E063
:10B1F000C8010F949E4E9C01009709F1982F901B57
:10B20000F12C992339F09150F801E90FF11D80815B
:10B21000F826F7CF4AE050E060E070E0C9010196FF
:10B220000F948C43CF2CD12CE12CF12C6C157D0587
:10B230008E059F0541F060E08BE29AE023C060E05C
:10B2400081E09AE01FC080918D0490918E04A091BE
:10B250008F04B09190048093890490938A04A09302
:10B260008B04B0938C0410C08091951480FF0CC0A7
:10B2700061E273E0C8010F94714E892B29F060E000
:10B2800087ED99E0A2DE73C080915F0281111BC03F
:10B2900067E470E0C8010F94664E0097A1F04AE0A1
:10B2A00050E060E070E001960F948C4364307105CB
:10B2B0008105910540F480E699E0A6D660E086E538
:10B2C00099E00E94F37265E273E0C8010F94714E39
:10B2D000892B21F4109219021092800F6AE273E018
:10B2E000C8010F94714E892B21F480E090E00E94F8
:10B2F00030626FE273E0C8010F94714E892B11F434
:10B300000E949F6561E081E994E00F940837FCCECC
:10B310000F3511050CF0F8CE8C35A1F40E94CB61ED
:10B3200097FDF2CE2091F3042111EECE98012F5F0C
:10B330003F4F3093F2042093F104F801EF56FB4F96
:10B340008083E2CE8B3321F481E08093F304DCCE62
:10B350008091F3048111D8CEC80101969093F20434
:10B360008093F104F801EF56FB4F2083CDCE8091FE
:10B37000951482FF1AC18091830E811102C0109230
:10B38000F504EE24E394409191145091921460914D
:10B3900093147091941480918D1490918E14A091B7
:10B3A0008F14B0919014481759076A077B0708F467
:10B3B000E12C00E010E0BB24B39480E6A82E92E8D4
:10B3C000C92E9AE0D92E29E6922E8091830E8430E0
:10B3D00008F0EBC0E110E9C08091F5048111E5C0EF
:10B3E0008091A1129091A212A091A312B091A412E7
:10B3F0008093911490939214A0939314B093941407
:10B4000041E050E0BE016F5F7F4F89E992E10E9409
:10B410006DAB019719F4898190E002C08FEF9FEF27
:10B42000F82E409091145090921460909314709064
:10B43000941440918D1450918E1460918F147091DA
:10B440009014EE24E394441655066606770608F435
:10B45000E12C4416550666067706B0F4019609F409
:10B460005FC08AE0F81609F46AC02DE0F21609F40C
:10B4700066C083E2F81619F02AE3F21278C08091D0
:10B48000F404811174C050C00E94D1C889E992E1CE
:10B490000E946DAD80918C14882339F18150809386
:10B4A0008C14989EC001112441E061E088509A4FAD
:10B4B0000E946DB6E0918C1484E0E89FF0011124A5
:10B4C000EC50FA4F40815181628173814093911415
:10B4D00050939214609393147093941489E992E1B9
:10B4E0000E94D1A90E9460B314C00E9450B30E9470
:10B4F0009CCA0E94FBE50E943C9B6D33710581054F
:10B50000910528F0D092F205C092F1058FDD0E94DE
:10B5100057738091951482FD0BC085E99AE003C0B2
:10B5200092D586E89AE070D523E2F21208C005C0F1
:10B5300023E2F21237C000E010E0B092F50410925E
:10B54000F4040115110519F40F9426330DC08091F0
:10B55000000DA89E000D111D1124F801EF5FF24FA0
:10B56000108280E00F94F33600E010E02ECF0F350C
:10B57000110508F02ACF8BE3F81203C0B092F4044F
:10B5800024CF8091F404811120CF8091000DF80127
:10B59000A89EE00DF11D1124EF5FF24FF0820F5FC6
:10B5A0001F4F13CF1092F404CFCF0F90DF91CF91A4
:10B5B0001F910F91FF90EF90DF90CF90BF90AF90D1
:10B5C0009F907F906F905F904F9008958F929F9281
:10B5D000AF92BF92CF92DF92EF92FF920F931F93A1
:10B5E000CF93F82E662351F01092200510921C057F
:10B5F00010921D0510921E0510921F050E9473B235
:10B6000080901C0590901D05A0901E05B0901F0510
:10B610009B01AC01281939094A095B0957FD41C052
:10B62000C0912005F7FC16C02F2D0F2C000C330BFA
:10B630002C5F3F4F4C2F0C2E000C550B2417350759
:10B6400084F1CF153CF034EFC32EDD24D394E12CEC
:10B65000F12C06C028EEC22E23E0D22EE12CF12CD4
:10B66000DC01CB018C0D9D1DAE1DBF1D80931C0503
:10B6700090931D05A0931E05B0931F050C2F01701C
:10B6800010E084E2809FB001819F700D701B112437
:10B6900060597C4F82E390E00E94EC9FCF5FC093A3
:10B6A0002005CF911F910F91FF90EF90DF90CF90E9
:10B6B000BF90AF909F908F9008958F929F92AF927E
:10B6C000BF92CF92DF92EF92FF92CF93FC01C080A6
:10B6D000D180E280F38020E030E0A901C701B6010B
:10B6E0000F94894687FF08C0C701B601905820E033
:10B6F00030E04AE754E406C020E030E04AE754E492
:10B70000C701B6010F94EE4620E030E040EA50E475
:10B710000F94D54A20E030E040E251E40F94B14B61
:10B720000F94194C6B017C01603AF6E87F07F1E059
:10B730008F07910584F020EA36E841E050E00F944D
:10B74000994ACA01B9012AE030E040E050E00F9484
:10B75000994A605D01C060E26093770F80E1C8168E
:10B7600087E2D806E104F10494F0C701B60120E1B4
:10B7700037E240E050E00F94994ACA01B9012AE04B
:10B7800030E040E050E00F94994A605D01C060E213
:10B790006093780FE8EECE16E3E0DE06E104F104F4
:10B7A00094F0C701B60128EE33E040E050E00F947A
:10B7B000994ACA01B9012AE030E040E050E00F9414
:10B7C000994A605D01C060E26093790FC701B601DC
:10B7D00024E630E040E050E00F94994A8AE0882E59
:10B7E000912CA12CB12CCA01B901A50194010F948F
:10B7F000994A605D60937A0F8EE280937B0FC70158
:10B80000B601A50194010F94994AC62FCA01B90146
:10B81000A50194010F94994A605D60937C0FC05D0F
:10B82000C0937D0F87E79FE0CF91FF90EF90DF906F
:10B83000CF90BF90AF909F908F9008958F929F92DE
:10B84000AF92BF92CF92DF92EF92FF92CF93FC0123
:10B85000C080D180E280F38020E030E04AE754E409
:10B86000C701B6010F94EE464B015C0120E030E0C9
:10B87000A901C701B6010F94894687FD05C060E0A4
:10B8800070E080EA90E404C060E070E080EA90EC50
:10B89000A50194010F94D54A20E030E040E251E444
:10B8A0000F94B14B0F94194C6B017C0197FF0AC0A8
:10B8B000F094E094D094C094C11CD11CE11CF11C04
:10B8C0008DE201C08BE28093770FC701B60120E1C2
:10B8D00037E240E050E00F94994A8AE0882E912C9C
:10B8E000A12CB12CCA01B901A50194010F94994A68
:10B8F000605D6093780FC701B60128EE33E040E049
:10B9000050E00F94994ACA01B901A50194010F941E
:10B91000994A605D6093790FC701B60124E630E073
:10B9200040E050E00F94994ACA01B901A501940181
:10B930000F94994A605D60937A0F8EE280937B0F3B
:10B94000C701B601A50194010F94994AC62FCA01F7
:10B95000B901A50194010F94994A605D60937C0F31
:10B96000C05DC0937D0F87E79FE0CF91FF90EF9080
:10B97000DF90CF90BF90AF909F908F9008958F925F
:10B980009F92AF92BF92CF92DF92EF92FF92FC0113
:10B99000C080D180E280F38020E030E0A901C701BF
:10B9A000B6010F94894687FF08C0C701B6019058B9
:10B9B00020E030E040E251E406C020E030E040E228
:10B9C00051E4C701B6010F94EE4620E030E040EAB2
:10B9D00050E40F94D54A20E030E040E251E40F9467
:10B9E000B14B0F94194C6B017C016031F7E27F077A
:10B9F0008105910584F020E137E240E050E00F94AA
:10BA0000994ACA01B9012AE030E040E050E00F94C1
:10BA1000994A605D01C060E26093790F88EEC816B4
:10BA200083E0D806E104F10494F0C701B60128EEE2
:10BA300033E040E050E00F94994ACA01B9012AE08E
:10BA400030E040E050E00F94994A605D01C060E250
:10BA500060937A0FE4E6CE16D104E104F10494F089
:10BA6000C701B60124E630E040E050E00F94994A67
:10BA7000CA01B9012AE030E040E050E00F94994A51
:10BA8000605D01C060E260937B0FFAE0CF16D104E5
:10BA9000E104F1049CF08AE0882E912CA12CB12CB9
:10BAA000C701B601A50194010F94994ACA01B901D1
:10BAB000A50194010F94994A605D01C060E2609312
:10BAC0007C0FC701B6012AE030E040E050E00F945F
:10BAD000994A605D60937D0F89E79FE0FF90EF904A
:10BAE000DF90CF90BF90AF909F908F9008958F92EE
:10BAF0009F92AF92BF92CF92DF92EF92FF92FC01A2
:10BB0000C080D180E280F38020E030E048EC52E455
:10BB1000C701B6010F94EE464B015C0120E030E016
:10BB2000A901C701B6010F94894687FD05C060E0F1
:10BB300070E080EA90E404C060E070E080EA90EC9D
:10BB4000A50194010F94D54A20E030E040E251E491
:10BB50000F94B14B0F94194C9B0177FF06C022271D
:10BB60003327261B370B8DE201C08BE28093780FC1
:10BB7000C90168EE73E00F940B4ECB01EAE0F0E0F0
:10BB8000BF010F940B4E805D8093790FC90164E66D
:10BB900070E00F940B4ECB01BF010F940B4E805DF4
:10BBA00080937A0FC901BF010F940B4E282FCB0150
:10BBB000BF010F940B4E805D80937B0F8EE28093CC
:10BBC0007C0F205D20937D0F88E79FE0FF90EF9032
:10BBD000DF90CF90BF90AF909F908F9008958F92FD
:10BBE0009F92AF92BF92CF92DF92EF92FF92CF934C
:10BBF000FC01C080D180E280F38020E030E04AE7A1
:10BC000054E4C701B6010F94EE464B015C0120E0FD
:10BC100030E0A901C701B6010F94894687FD05C030
:10BC200060E070E080EA90E404C060E070E080EAE8
:10BC300090ECA50194010F94D54A20E030E040E259
:10BC400051E40F94B14B0F94194C6B017C0197FD9B
:10BC500010C020E137E240E050E00F94994ACA0159
:10BC6000B9012AE030E040E050E00F94994A605D6D
:10BC700009C0F094E094D094C094C11CD11CE11C84
:10BC8000F11C6DE26093780FC701B60128EE33E036
:10BC900040E050E00F94994A8AE0882E912CA12C24
:10BCA000B12CCA01B901A50194010F94994A605DB4
:10BCB0006093790FC701B60124E630E040E050E020
:10BCC0000F94994ACA01B901A50194010F94994AA8
:10BCD000605D60937A0F8EE280937B0FC701B6019F
:10BCE000A50194010F94994AC62FCA01B901A50173
:10BCF00094010F94994A605D60937C0FC05DC0937E
:10BD00007D0F88E79FE0CF91FF90EF90DF90CF907D
:10BD1000BF90AF909F908F9008959C0197FF0AC0AD
:10BD2000EE27FF27E81BF90BE436F1050CF44CC0B5
:10BD30008DE230C0283E83E038073CF1C90168EE4F
:10BD400073E00F940B4ECB01EAE0F0E0BF010F94DB
:10BD50000B4E805D80937A0FC90164E670E00F940A
:10BD60000B4ECB01BF010F940B4E805D80937B0F78
:10BD7000C901BF010F940B4ECB01BF010F940B4EB5
:10BD8000805D80937C0FF9013EC0F90124363105B6
:10BD9000DCF080E280937A0FCF0164E670E00F94CC
:10BDA0000B4ECB012AE030E0B9010F940B4E805DC1
:10BDB00080937B0FCF01B9010F940B4ECB01B901DA
:10BDC0000F940B4E805D1DC080E280937A0F8093AC
:10BDD0007B0FEA30F10584F037FF02C08DE201C02D
:10BDE00080E280937B0FCF016AE070E00F940B4EEE
:10BDF000605D60937C0F07C037FF02C08DE201C019
:10BE000080E280937C0FCF016AE070E00F940B4ECC
:10BE1000805D80937D0F8AE79FE008959C01EAE0B2
:10BE2000F0E0BF010F940B4E805D80937D0F2A30B0
:10BE30003105CCF0CB01BF010F940B4E805D809398
:10BE40007C0F2436310594F0C90164E670E00F944C
:10BE50000B4ECB01BF010F940B4E805D80937B0F87
:10BE60008BE79FE008958DE79FE008958CE79FE0C2
:10BE700008959C0197FD0EC08436910584F064E618
:10BE800070E00F940B4ECB016AE070E00F940B4E04
:10BE9000805D06C03195219531098DE201C080E2B7
:10BEA00080937B0F2A30310564F0EAE0F0E0C901AD
:10BEB000BF010F940B4ECB01BF010F940B4E805D61
:10BEC00001C080E280937C0FC9016AE070E00F94AA
:10BED0000B4E805D80937D0F8BE79FE00895282FA8
:10BEE000843628F064E60F94EB4D805D01C080E25B
:10BEF00080937B0F2A3048F03AE0822F632F0F9413
:10BF0000EB4D0F94EB4D905D01C090E290937C0F50
:10BF1000822F6AE00F94EB4D905D90937D0F8BE73D
:10BF20009FE00895CF92DF92EF92FF926B017C0128
:10BF300083E3C816D104E104F10470F082E3C81A67
:10BF4000D108E108F10862E370E080E090E00E942F
:10BF50003BB20F942633ECCFC701B6010E943BB22F
:10BF6000FF90EF90DF90CF900D9426338F929F92A9
:10BF7000AF92BF92CF92DF92EF92FF920F93CF9347
:10BF8000DF931F92CDB7DEB75C016B017A014901E7
:10BF9000F501808191810F94524A8983002311F029
:10BFA000F6018083BE016F5F7F4FC4010F942A2486
:10BFB000F50180819181019691838083FFEFCF1AF3
:10BFC000DF0A81E0E81AF10819F780E00F90DF91AD
:10BFD000CF910F91FF90EF90DF90CF90BF90AF90F7
:10BFE0009F908F9008959091C00095FFFCCF809313
:10BFF000C6000895CF93C82FCC2321F080E2F3DF51
:10C00000C150FACFCF910895CF93DF93FC01849173
:10C01000EF012196882319F0E6DFFE01F8CFDF91CA
:10C02000CF9108950F931F93CF93DF938B01ECDF94
:10C03000E8018991882311F0D6DFFBCFDF91CF9102
:10C040001F910F91089580EC9CE0DECF90918B0CB6
:10C0500093FD0FC09091C40691110BC04091060F43
:10C060005091070F2091100230911102421753078F
:10C070004CF040E0682F8AE00F94D21A61E080E033
:10C080000C9439F9E0DF87EC9CE0BEDF80E0089596
:10C090008AEB9CE0B9CF7F928F929F92AF92BF9232
:10C0A000CF92DF92EF92FF920F931F93CF93DF9384
:10C0B0001F92CDB7DEB77C0159018B016B01C40E15
:10C0C000D51E0C151D0549F1F70180809180F801FE
:10C0D00071908F017982C4010F94524A781681F0D1
:10C0E000672DC4010F945A4AC4010F94524A998192
:10C0F000891731F0CDDF80EA9CE086DF81E00EC059
:10C10000BE016F5F7F4FC5010F942A24F701808124
:10C110009181019691838083D4CF80E00F90DF914D
:10C12000CF911F910F91FF90EF90DF90CF90BF9034
:10C13000AF909F908F907F9008958F929F92AF9233
:10C14000BF92EF92FF920F931F93CF93DF93CDB7E0
:10C15000DEB7A0970FB6F894DEBF0FBECDBF611556
:10C1600071058105910589F100E0842E912CA12CA7
:10C17000B12C102FEE24E394F12CEC0EFD1EE00EFA
:10C18000F11C07FDFA94A50194010F94774AF70179
:10C190006083B901CA010F5F6115710581059105C1
:10C1A00041F71F3F21F1E1E0F0E0EC0FFD1FE10F4F
:10C1B000F11D17FDFA9580818A3010F097E301C0D8
:10C1C00090E3890F10DF1150ECCF80E3A0960FB6FB
:10C1D000F894DEBF0FBECDBFDF91CF911F910F91BD
:10C1E000FF90EF90BF90AF909F908F90FCCEA09665
:10C1F0000FB6F894DEBF0FBECDBFDF91CF911F9178
:10C200000F91FF90EF90BF90AF909F908F90089507
:10C21000CF92DF92EF92FF926A017B01F5DE4AE056
:10C22000C701B601FF90EF90DF90CF9086CFCF92FD
:10C23000DF92EF92FF926B017C0197FF0AC08DE2C3
:10C24000D2DEF094E094D094C094C11CD11CE11CC7
:10C25000F11C4AE0C701B601FF90EF90DF90CF904C
:10C260006CCFCF93DF93EB01CFDEBE01DD0F880BE8
:10C27000990BDF91CF91DBCF8F929F92AF92BF92BC
:10C28000CF92DF92EF92FF92CF936B017C01B42E9D
:10C2900020E030E0A9010F94894687FF06C08DE2B7
:10C2A000A2DEF7FAF094F7F8F094C0E060E070E0F6
:10C2B00080E09FE3CB1541F02DEC3CEC4CEC5DE3D2
:10C2C0000F94EE46CF5FF6CF9B01AC01C701B601DC
:10C2D0000F94D54A6B017C010F941E4C4B015C01FD
:10C2E0004AE02BDFCC2379F1C501B4010F948D46D0
:10C2F0009B01AC01C701B6010F94D44A6B017C01CC
:10C300008EE271DE20E030E040E251E4C701B60188
:10C310000F94EE464B015C010F94194C6B01770FA3
:10C32000EE08FF08C701B60182DFC701B6010F940E
:10C330008F469B01AC01C501B4010F94D44A6B0137
:10C340007C01C150F9F6CF91FF90EF90DF90CF9034
:10C35000BF90AF909F908F900895CF92DF92EF9211
:10C36000FF926A017B0150DE42E0C701B601FF90F7
:10C37000EF90DF90CF9080CF8DE035DE8AE033CE36
:10C38000CF93DF93EC018991882311F02CDEFBCF52
:10C39000DF91CF91F1CF8091070490910804981715
:10C3A00059F0E92FF0E0E95FFB4F82819F5F9F77B3
:10C3B0009093080490E008958FEF9FEF08951F92E7
:10C3C0000F920FB60F9211240F900FBE0F901F9077
:10C3D00018951F920F920FB60F9211240BB60F9261
:10C3E0002F938F939F93EF93FF9320910804E091F5
:10C3F000070481E08E0F8F779091C600281729F0EF
:10C40000F0E0E95FFB4F9283E82FE0930704FF9190
:10C41000EF919F918F912F910F900BBE0F900FBEB8
:10C420000F901F9018958EBD0DB407FEFDCF089597
:10C430008FEF8EBD0DB407FEFDCF8EB508959091A0
:10C4400064009B7F90936400982F906A96959CBDA2
:10C4500080FD03C091E0863009F490E09DBD089511
:10C46000EC010E9462FEEFDD80E89CE0CDDD2097CC
:10C4700011F4C7E7DCE00E9428D561E0CE010E94FC
:10C48000F3720E94CF6F60E080E00E94DA7086E86D
:10C490009FE00E94D77062E080E00E94DA7088E638
:10C4A0009CE00E94CE7063E080E00E94DA708BE531
:10C4B0009CE00E94CE7089EE93E030E6019729F06F
:10C4C000232F2A950000E9F7F9CFF89489EE93E03D
:10C4D00038EE019729F0232F2A950000E9F7F9CFCC
:10C4E0000E9462FEA895FECF2F923F924F925F92DC
:10C4F0006F927F928F929F92AF92BF92CF92DF9274
:10C50000EF92FF920F931F93CF93DF93CDB7DEB7D8
:10C5100027970FB6F894DEBF0FBECDBF89830E9468
:10C52000CB730E9473B26B017C018091000288235F
:10C5300039F18091810F882319F1409106055091BE
:10C540000705609108057091090597018601041B94
:10C55000150B260B370B37FD26C0833069F034F4FA
:10C56000813074F095DD8FEE9BE009C0843041F49A
:10C570008FDD80EC9BE003C08BDD88ED9BE044DD2C
:10C580002091000230E0A8EEB3E00F94C54AC60E39
:10C59000D71EE81EF91EC0920605D0920705E0924C
:10C5A0000805F09209058091830E843010F40E94F2
:10C5B0006F580E9473B26B017C014091F903509156
:10C5C000FA036091FB037091FC034115510561056D
:10C5D0007105F9F08091231090912410A0912510FD
:10C5E000B0912610840F951FA61FB71FA7019601B3
:10C5F000281B390B4A0B5B0B57FD0BC024DD6091E8
:10C60000830F7091840F81E29CE00CDD8AE0EBDC0B
:10C610006BC040910102509102026091030270913F
:10C620000402411551056105710509F442C090915C
:10C63000101380911113981749F0C0922310D092D3
:10C640002410E0922510F092261033C08091F3055B
:10C6500081112FC0098101112CC08091231090916C
:10C660002410A0912510B0912610840F951FA61FAD
:10C67000B71FA7019601281B390B4A0B5B0B57FD0F
:10C6800018C05F9A8091FE0C8E7F8093FE0C8A9A70
:10C690008091FE0C8D7F8093FE0C80910801809527
:10C6A0008170809306018091FE0C8B7F8093FE0C3D
:10C6B000129A8091120590911305909902C00196EB
:10C6C00004C0181619062CF4019790931305809353
:10C6D000120580911205909113058E3E92403CF018
:10C6E000B2DC81E09CE090DC80E090E0B9DE8091FB
:10C6F0000E0590910F05A0911005B09111059701BD
:10C700008601081B190B2A0B3B0B37FD3DC190918D
:10C71000101380911113981306C06091B206109106
:10C72000B30619831BC0E09111138CE58E9FF001B5
:10C730001124E15EF84F6081E09111138E9FF001AA
:10C740001124E05EF84F00810983809111139091CC
:10C750001013981719F08F5F8F70F9CF70E089E090
:10C760000E9474B11981612F70E087E00E9474B15A
:10C7700080911510882309F4FAC020903B02309074
:10C780003C0200913D020F8310913E021E83609196
:10C79000060F7091070F6E5F7F4F072E000C880BFE
:10C7A000990B0F948F469101A8010F94894687FD3C
:10C7B000DEC00091111309831A821B821C821D8224
:10C7C000809110131981811709F460C0812F90E0C6
:10C7D0002CE5289FF001299FF00D1124E753F94F14
:10C7E000458956896789708D452B462B472B81F4E7
:10C7F000418D528D638D748D452B462B472B41F413
:10C80000458D568D678D70A1452B462B472BC9F161
:10C810003CE5389F8001399F100D11240753194FB3
:10C82000F80161817281838194810F948E4D4B0157
:10C830005C01F80161A172A183A194A10F948D46BE
:10C840002B013C01F80165A176A187A190A50F9469
:10C850008D469B01AC01C301B2010F94B14BA50100
:10C8600094010F94EE465B018C012A813B814C813F
:10C870005D810F94494D181624F4AA82BB820C8363
:10C880001D8389818F5F8F7089839ACF20913F02AA
:10C890003091400240914102509142026A817B8175
:10C8A0008C819D810F94EE4691014F815E810F94A2
:10C8B000D54A5B018C019B01AC01B1018F819E8146
:10C8C0000F94494D1816B4F020903702309038027A
:10C8D000F0913902FF8320913A022E8391014F2F6C
:10C8E0005E81B501C8010F94494D18161CF0150161
:10C8F0000F831E8380900A0590900B05A0900C0575
:10C90000B0900D0591014F815E81C501B4010F9476
:10C91000494D1816D4F420E037ED43EA5CE3B10149
:10C920008F819E810F94EE462B013C0128E431EE6D
:10C930004AE75FE3C501B4010F94EE46A3019201FB
:10C940000F94D54A1B018F839E83C101AF81BE81A5
:10C9500080930A0590930B05A0930C05B0930D05E9
:10C96000B101CD010F94194CCB010E9452FE34E667
:10C97000C30ED11CE11CF11CC0920E05D0920F0514
:10C98000E0921005F09211050F9426338091DE0E8F
:10C99000813009F06EC00E9473B26B017C018091FE
:10C9A000180590911905A0911A05B0911B059701E2
:10C9B0008601081B190B2A0B3B0B37FD3AC08090F0
:10C9C000DF0E9090E00EA090E10EB090E20E0E947B
:10C9D0003C9B6093DF0E7093E00E8093E10E90938A
:10C9E000E20E0091F00C1091F10C2091F20C3091BC
:10C9F000F30C081919092A093B09DC01CB01800F46
:10CA0000911FA21FB31F8093F00C9093F10CA09381
:10CA1000F20CB093F30CD701C601805F984DAF4F75
:10CA2000BF4F8093180590931905A0931A05B093F2
:10CA30001B058091140590911505A0911605B091E4
:10CA40001705A7019601281B390B4A0B5B0B57FDF5
:10CA500010C030E8C30E3EEED31EE11CF11CC092A4
:10CA60001405D0921505E0921605F09217050E9464
:10CA7000D9E50E94309C8091F403882309F446C0D4
:10CA80000E9473B20091F0031091F1032091F20320
:10CA90003091F303DC01CB01801B910BA20BB30B94
:10CAA000B7FD34C00E9473B26B017C012091F40386
:10CAB00030E0A8EEB3E00F94C54AC60ED71EE81EBC
:10CAC000F91EC092F003D092F103E092F203F092CB
:10CAD000F30380E00E94C8F88AE027960FB6F89426
:10CAE000DEBF0FBECDBFDF91CF911F910F91FF90A1
:10CAF000EF90DF90CF90BF90AF909F908F907F90FE
:10CB00006F905F904F903F902F906DCA27960FB611
:10CB1000F894DEBF0FBECDBFDF91CF911F910F9173
:10CB2000FF90EF90DF90CF90BF90AF909F908F904D
:10CB30007F906F905F904F903F902F900895CF938C
:10CB400080916F00C82FC27081FF05C080916F0077
:10CB50008D7F80936F0080911113809310138093C9
:10CB60000F1380930E1384E680930D130E94AACDB9
:10CB700088EE93E090938A0C8093890CCC2329F063
:10CB800080916F00826080936F0081E08093F41544
:10CB90000E94D1C88EEF0F947F1BCF910D94141F6C
:10CBA000E2EBF6E01082118208952CEA35EC47E2C0
:10CBB0005EE360912605709127058091280590918C
:10CBC00029050F94B14B6093251670932616809318
:10CBD00027169093281608952CEA35EC47E25EE379
:10CBE00060912A0570912B0580912C0590912D055F
:10CBF0000F94EE46609321167093221680932316AD
:10CC0000909324160895CF93DF93EC01CB01BA01E2
:10CC10000F948F4620E030E048EC52E40F94EE464B
:10CC20000F941E4C688379838A839B83DF91CF9115
:10CC300008950C942DE80C94E6E70F931F93CF937F
:10CC4000DF93CDB7DEB76E970FB6F894DEBF0FBE99
:10CC5000CDBF809106028F93809105028F931F9222
:10CC60001F9283E39DE09F938F938E010F5F1F4F71
:10CC70001F930F930F94234681E080934710C801C0
:10CC80000E940858109247100FB6F894DEBF0FBEEE
:10CC9000CDBF6E960FB6F894DEBF0FBECDBFDF914D
:10CCA000CF911F910F91089590917D0681E0892782
:10CCB0000C9487F40C94B4FD80E00C9403FE63E0C4
:10CCC00076E68BE696E60C94247162EB7DE68BE2C9
:10CCD0009EE60C9424710F948F4620E030E048ECDF
:10CCE00052E40F94EE460C94EA6F63E972E084E636
:10CCF00090E00E94EC9F6AEB72E084E690E00C9476
:10CD0000EC9F8111F2CF68EB71E084E190E00C942C
:10CD1000EC9F0F94A22EF5CF0E943C87F2CF382FC4
:10CD20001092760F8091110F9091120FA091130F16
:10CD3000B091140F81309048A105B10540F01092D8
:10CD4000110F1092120F1092130F1092140F2091C6
:10CD5000110F20930A0F1092090F8091080F1816D7
:10CD6000ECF4082E000C990B831B9109022E000C89
:10CD7000330B2817390794F097FF02C080E090E04A
:10CD800080930A0F092E000CAA0BBB0B8093110F86
:10CD90009093120FA093130FB093140F80910A0F6A
:10CDA0006623A9F090910B0F891714F480930B0F51
:10CDB00020910B0F022E000C330B2D5F3F4F482F9D
:10CDC000082E000C550B241735071CF48350809354
:10CDD0000B0F0895EF92FF920F931F93CF93DF9362
:10CDE00061E081E09CDFD0910B0FC0E0D1110BC05E
:10CDF00080910A0F81112AC08091050F1092050FB2
:10CE000081111EC023C0D13061F480910A0F81309E
:10CE100009F043C08091050F1092050F811128C0C1
:10CE20003CC0D23009F05EC080910A0F823009F018
:10CE30008AC08091050F1092050F81116FC083C0C9
:10CE40000E94D56F8091090F81116BC180915002B2
:10CE5000882309F43EC081E090910A0F911180E08F
:10CE600003E023E045E25EE06C2F0E94347231C0A3
:10CE70000E94DFEAE12C10ECF12E09E714E420E037
:10CE800030E040E85FE360EB7CE08EE19EE00E94F2
:10CE9000EBEA8091090F811144C1809150028823EF
:10CEA000C1F011E080910A0F813009F010E060912B
:10CEB000B00C7091B10C8091B20C9091B30C0E94A7
:10CEC000217000E09C0147E15EE06C2F812F0E9401
:10CED000E571CF5FDF5FC43009F088CF87E08093D2
:10CEE000080F1FC1D33061F480910A0F833009F01D
:10CEF00067C08091050F1092050F81114CC060C072
:10CF0000D430D9F580910A0F843009F097C0809110
:10CF1000050F1092050F81117CC090C00E94DFEABE
:10CF2000E12C10ECF12E09E714E420E030E040E8B9
:10CF30005FE364EB7CE080E19EE00E94EBEA80919D
:10CF4000090F8111EEC080915002882309F4C1CFEE
:10CF500011E080910A0F823009F010E06091B40C6A
:10CF60007091B50C8091B60C9091B70C0E94217015
:10CF700000E09C0149E05EE0A8CFD530D9F5809172
:10CF80000A0F853009F087C08091050F1092050FB8
:10CF900081116DC080C00E94DFEAE12C10ECF12EFF
:10CFA00009E714E420E030E040E85FE368EB7CE070
:10CFB00082E09EE00E94EBEA8091090F8111B1C0EE
:10CFC00080915002882309F484CF11E080910A0FE8
:10CFD000833009F010E06091B80C7091B90C809129
:10CFE000BA0C9091BB0C0E94217000E09C014BEFA9
:10CFF0005DE06BCFD63009F06CCF80910A0F8630A0
:10D0000009F076C08091050F1092050F81115CC068
:10D010006FC00E94DFEAE12C10ECF12E09E714E466
:10D0200020E030E040E85FE36CEB7CE084EF9DE0E3
:10D030000E94EBEA8091090F811173C08091500228
:10D04000882309F446CF11E080910A0F843009F05B
:10D0500010E06091BC0C7091BD0C8091BE0C909161
:10D06000BF0CEFD700E09C014DEE5DE02ECF0E949B
:10D07000DFEAE12C10ECF12E09E714E420E030E0C7
:10D08000A9016CEC7CE088EE9DE00E94EBEA8091C7
:10D09000090F811146C080915002882309F419CFED
:10D0A00011E080910A0F853009F010E06091CC0CFE
:10D0B0007091CD0C8091CE0C9091CF0CC2D700E036
:10D0C0009C0143EE5DE001CF0E94DFEAE12C10EC11
:10D0D000F12E09E714E420E030E0A90160ED7CE0E6
:10D0E00089ED9DE00E94EBEA8091090F811119C042
:10D0F00080915002882309F4ECCE11E080910A0F50
:10D10000863009F010E06091D00C7091D10C8091C4
:10D11000D20C9091D30C95D700E09C014FEC5DE0D0
:10D12000D4CEDF91CF911F910F91FF90EF90089592
:10D130002F923F924F925F926F927F928F929F9227
:10D14000AF92BF92CF92DF92EF92FF920F931F9315
:10D15000CF93DF9300D01F92CDB7DEB761E081E0BF
:10D16000DEDDA0900B0FB12C7FE3272E72E0372E6F
:10D17000E4E64E2E512C612C712CF1ED8F2EF1E74F
:10D180009F2EA1100BC080910A0F811129C08091A0
:10D19000050F1092050F81111EC022C081E0A81258
:10D1A0000BC090910A0F9130C1F58091050F10923C
:10D1B000050F811126C031C092E0A9129BC0809159
:10D1C0000A0F823009F0C8C08091050F1092050F38
:10D1D0008111B1C0C1C0E9D68091090F81117AC215
:10D1E00080915002882369F181E090910A0F91119A
:10D1F00080E003E023E04DEB5DE06B2D0E94347294
:10D2000020C0809115108A258093151083E08093AB
:10D2100050028091090F81115DC2809150028823D4
:10D2200081F080911510811174C02DEA3DE081E0FC
:10D23000913009F080E001E044EB5DE06B2D0E944D
:10D24000E5712CEA35EC47E25EE3609121167091BE
:10D25000221680912316909124160F94B14B60935F
:10D260002A0570932B0580932C0590932D052CEAAD
:10D2700035EC47E25EE360912516709126168091A9
:10D280002716909128160F94EE466093260570930A
:10D290002705809328059093290585E0A8120CC0E6
:10D2A00080910A0F853009F01AC18091050F109204
:10D2B000050F8111FFC013C196E0A9120CC0809127
:10D2C0000A0F863009F042C18091050F1092050FB8
:10D2D000811125C13BC187E0A8128EC180910A0F40
:10D2E000873009F0AFC18091050F1092050F8111B1
:10D2F00092C1A8C183E0A8120FC080910A0F8330A9
:10D3000009F054C08091050F1092050F81113DC0A6
:10D310004DC021EB3DE08BCF94E0A91292CF8091DC
:10D320000A0F843009F0A4C08091050F1092050FF8
:10D33000811158C09DC0E12CF12C02E813E420E0DB
:10D3400030E0A9016BE372E086EA9DE00E94EBEA1F
:10D350008091090F8111BEC180915002882309F488
:10D3600070CF11E080910A0F823009F010E06091D7
:10D370003B0270913C0280913D0290913E0261D649
:10D3800000E09C014FE95DE029C0E12CF12C02E8AE
:10D3900013E420E030E0A90167E372E088E99DE052
:10D3A0000E94EBEA8091090F811194C18091500293
:10D3B000882309F446CF11E080910A0F833009F0E9
:10D3C00010E060913702709138028091390290919B
:10D3D0003A0237D600E09C0141E95DE06B2D812FD8
:10D3E000F4D7DEC020E030E048EC52E460913F0228
:10D3F0007091400280914102909142020F94EE465A
:10D400000F94194C6B017C01AAD583E080935002E4
:10D4100089E89DE09093200F80931F0F30921E0F9C
:10D4200020921D0F1092190F10921A0F10921B0FBD
:10D4300010921C0F4092150F5092160F6092170F0A
:10D440007092180FC092110FD092120FE092130F2A
:10D45000F092140F90927B1380927A131092100F17
:10D4600010920F0F10920E0F8091090F811132C18F
:10D4700080915002882309F493C011E080910A0F33
:10D48000843009F010E080913F0290914002A09119
:10D490004102B091420289839A83AB83BC83CE015F
:10D4A00001960E94EF5D00E09C0141E85DE06B2D7C
:10D4B000812FC5CEC12CD12CE12C18E1F12E0CE12D
:10D4C00016E420E030E040E85FE36DE176E18BE7D1
:10D4D0009DE00F948B3F8091090F8111FBC08091DB
:10D4E0005002882309F453C011E080910A0F85305F
:10D4F00009F010E080911D1690911E16A0911F1644
:10D50000B091201689839A83AB83BC83CE010196A8
:10D510000E941E5C00E09C0145E75DE035C02CEEFA
:10D52000C22E25E6D22EE12C18E1F12E0CE116E4F4
:10D530002AE037ED43E25CE36AE275E08FE69DE0C6
:10D540000F948B3F8091090F8111C4C080915002CC
:10D550008823E9F011E080910A0F863009F010E08D
:10D5600080912A0590912B05A0912C05B0912D0555
:10D5700089839A83AB83BC83CE0101960E941E5C93
:10D5800000E09C0149E65DE06B2D812F1ED7B3942E
:10D59000A39494E0B912F5CD89E08093080F9AC066
:10D5A0002CEA35EC47E25EE3609121167091221679
:10D5B00080912316909124160F94B14B60932A0505
:10D5C00070932B0580932C0590932D052CEA35EC58
:10D5D00047E25EE36091251670912616809127162A
:10D5E000909128160F94EE466093260570932705B8
:10D5F000809328059093290598E0A912C8CF8091BF
:10D600000A0F883009F050C08091050F1092050F65
:10D61000811138C049C085EDC82E85E6D82EE12C91
:10D6200018E1F12E0CE116E420E030E040E85FE381
:10D6300066E275E083E69DE00F948B3F8091090FD1
:10D64000811148C080915002882309F4A0CF11E0D5
:10D6500080910A0F873009F010E0809126059091A3
:10D660002705A0912805B091290589839A83AB836A
:10D67000BC83CE0101960E941E5C00E09C014DE53A
:10D680005DE082CF0E94DFEA0DE116E624E031E0A2
:10D6900046E950E065E072E080E59DE00F94463E8B
:10D6A0008091090F811116C080915002882309F4DE
:10D6B0006ECF11E080910A0F883009F010E0809160
:10D6C0000502909106020E94395F00E09C0143E44C
:10D6D0005DE05ACF0F900F900F900F90DF91CF9198
:10D6E0001F910F91FF90EF90DF90CF90BF90AF9080
:10D6F0009F908F907F906F905F904F903F902F9072
:10D700000895AF92BF92CF92DF92EF92FF920F9364
:10D710001F93CF93DF9361E081E001DBC0910B0F9A
:10D72000B12C43E0A42EC1110BC080910A0F8111CE
:10D730001AC08091050F1092050F81110FC013C000
:10D74000C13001F580910A0F813009F0BAC0809193
:10D75000050F1092050F8111A7C0B3C026D4809188
:10D76000090F8111FCC080915002882359F081E09B
:10D7700090910A0F911180E003E023E041E25DE027
:10D780006B2D72D68091AF0E882371F0C23071F488
:10D7900080910A0F823009F0C6C08091050F109267
:10D7A000050F8111A8C0BFC0D2E001C0D3E0DC13D7
:10D7B00037C080910A0F8D131AC08091050F109207
:10D7C000050F8823A1F00E94DFEAE12C10E8F12E7A
:10D7D0000BE314E420E030E0A9016CE974E182EF8E
:10D7E0009CE00E94EBEA8091090F8111B8C0809102
:10D7F00050028823A9F011E080910A0F8C1310E0E9
:10D8000060919C1470919D1480919E1490919F142E
:10D8100018D400E09C0148EE5CE06B2D812FD5D53B
:10D8200081E08D0F8C1337C080910A0F8C131AC0C2
:10D830008091050F1092050F8823A1F00E94DFEA66
:10D84000E12C10E8F12E0BE314E420E030E0A90114
:10D8500060EA74E180EE9CE00E94EBEA8091090F9F
:10D8600081117DC0809150028823A9F011E0809140
:10D870000A0F8C1310E06091A0147091A114809194
:10D88000A2149091A314DDD300E09C0148ED5CE06C
:10D890006B2D812F9AD5B394CF5F84E0B81243CF1C
:10D8A000DE5FD093080F5BC08091AF0E8C27809312
:10D8B000AF0EA09250020E940DC88091090F8111F5
:10D8C0004EC080915002882309F45CCF8091AF0E46
:10D8D000811103C020E13DE002C024E13DE081E090
:10D8E00090910A0F913009F080E001E047E15DE09E
:10D8F0006B2D6BD547CF0E94DFEA2DE0C22E28ECBE
:10D90000D22EE12CF12C00E510E420E030E040ECD8
:10D910005FE364EB7EE086E09DE00F94053F80913D
:10D92000090F81111CC0809150028823B1F0D1E011
:10D9300080910A0F823009F0D0E06091B40E7091AE
:10D94000B50E8091B60E9091B70E5DD300E09C01AC
:10D950004CEF5CE06B2D8D2F38D5D3E061CFDF919C
:10D96000CF911F910F91FF90EF90DF90CF90BF90DC
:10D97000AF9008958091101390911113891B8F70AF
:10D9800031F48091951482FB882780F9089581E015
:10D990000895CF92DF92EF92FF920F931F93CF9350
:10D9A000DF93EC016A017B0180917A1390917B13E4
:10D9B0008C179D0709F479C023EACE34D207A1F46D
:10D9C000875D964D89F50E9473B2DC01CB018E51C3
:10D9D0009B4FAF4FBF4F8093220590932305A09399
:10D9E0002405B093250520C026EDC73DD20709F0D8
:10D9F0004FC08E54934A09F03CC00E9473B200910C
:10DA00002205109123052091240530912505DC0184
:10DA1000CB01801B910BA20BB30BB7FF2AC0AADF6F
:10DA2000882311F0CEE1D9E9D0937B13C0937A1308
:10DA3000C092110FD092120FE092130FF092140FB8
:10DA400086EDC73DD80731F41092C4051092210528
:10DA5000C7EDD6ED0F94A42481E0C75DD64D09F043
:10DA600080E024D382E08093500281E08093090F0C
:10DA70001CC087ED96ED90937B1380937A13C09230
:10DA8000110FD092120FE092130FF092140FDCCF0F
:10DA9000D0937B13C0937A134093110F5093120FBE
:10DAA0006093130F7093140FD5CFDF91CF911F9117
:10DAB0000F91FF90EF90DF90CF900895CF93DF9379
:10DAC000EC014DD240E050E0BA01CE01DF91CF91A0
:10DAD00060CF0F931F93CF93DF93809150028823E1
:10DAE00051F06091C2057091C30500E010E020E0A4
:10DAF00041E081E0ECD48091471081111AC081E0AF
:10DB000080934710C0917A13D0917B1340E050E08E
:10DB1000BA0189E69DE63DDF0E94D1C81092471008
:10DB200040E050E0BA01CE01DF91CF911F910F91FB
:10DB300030CFDF91CF911F910F910895CF93DF9355
:10DB4000EC01CB01BA010F948F462AE037ED43E296
:10DB50005CE30F94EE46688379838A839B83DF912D
:10DB6000CF910895CF93DF93EC01CB01BA010F94CD
:10DB70008F462AE037ED43E25CE30F94EE4668837C
:10DB800079838A839B83DF91CF910895CF93DF932D
:10DB9000EC01CB01BA010F948F462AE037ED43E246
:10DBA0005CE30F94EE46688379838A839B83DF91DD
:10DBB000CF910895CF93DF93EC01CB01BA010F947D
:10DBC0008F4620E030E048EC52E40F94EE46688344
:10DBD00079838A839B83DF91CF910895CF93DF93DD
:10DBE000EC01CB01BA010F948F462FE632E143E8F6
:10DBF0005AE30F94EE46688379838A839B83DF918F
:10DC0000CF910895CF93DF93EC01CB01BA010F942C
:10DC10008F46688379838A839B83DF91CF910895B0
:10DC2000CF93DF93EC01CB01BA010F948F460F9491
:10DC30001E4C6883DF91CF910895CF93DF93EC0161
:10DC4000CB01BA010F948F460F94194C79836883E6
:10DC5000DF91CF910895CF93DF9300D01F92CDB77E
:10DC6000DEB70F948F462AE037ED43E25CE30F9472
:10DC7000EE4669837A838B839C83CE0101960E9452
:10DC80005D5B0F900F900F900F90DF91CF910895F3
:10DC9000CF93DF9300D01F92CDB7DEB70F948F469E
:10DCA0002AE037ED43E25CE30F94EE4669837A8322
:10DCB0008B839C83CE0101960E941E5C0F900F9077
:10DCC0000F900F90DF91CF910895CF93DF9300D005
:10DCD0001F92CDB7DEB70F948F4620E030E048ECBE
:10DCE00052E40F94EE4669837A838B839C83CE0142
:10DCF00001960E94BF5C0F900F900F900F90DF91E4
:10DD0000CF910895CF93DF9300D01F92CDB7DEB7A8
:10DD10000F948F462AE037ED43E25CE30F94EE4622
:10DD200069837A838B839C83CE0101960E94EF5D89
:10DD30000F900F900F900F90DF91CF9108950F9457
:10DD40008F460F941E4C862F0C946F5F0F948F4656
:10DD50000F94194CCB010C94395FEF92FF920F9303
:10DD60001F93CF93DF93CDB7DEB728970FB6F89404
:10DD7000DEBF0FBECDBF8E010F5F1F4FD80120E069
:10DD800030E0FB01E20FF31FE491ED932F5F3F4F73
:10DD900028303105B1F7877028E0829FC001112437
:10DDA00080640F949E247E0189E0E80EF11CF80146
:10DDB00061918F0182E693E10E9441B3E016F10682
:10DDC000B1F728960FB6F894DEBF0FBECDBFDF9136
:10DDD000CF911F910F91FF90EF900895CF92DF9216
:10DDE000EF92FF920F931F93CF93DF9300D000D059
:10DDF000CDB7DEB78A0146E0469F9001479F300DC0
:10DE00001124BC01620F731F46E050E0CE01019661
:10DE10000F94C945C980DA80EB80FC80F80140810D
:10DE2000518162817381C416D506E606F70648F073
:10DE300081E090E04C155D056E057F0520F080E0E7
:10DE400002C08FEF9FEF26960FB6F894DEBF0FBE8D
:10DE5000CDBFDF91CF911F910F91FF90EF90DF9099
:10DE6000CF9008950F931F93CF93DF93CDB7DEB775
:10DE70002E970FB6F894DEBF0FBECDBF1E861D864F
:10DE80006F83788789879A872FEF2B8741155105F4
:10DE9000C1F18A016038710581059105B0F19E01DB
:10DEA000235F3F4FAE01495F5F4F69EB70E08EEF3C
:10DEB00093E10F94422497FD0BC08D859E8526E04B
:10DEC000289FB001299F700D112462507C4E22C002
:10DED0009E01235F3F4FAE01495F5F4F6AEE70E0E6
:10DEE00082E89EE00F94422497FD0EC08D859E85AA
:10DEF00026E0289FB001299F700D11246E57714FA5
:10DF000009C080E090E020C06FE382E693E10E94C8
:10DF100041B318C046E050E0CE0101960F94C945C8
:10DF20006D8182E693E10E9441B30230110550F009
:10DF30006E81662339F082E693E10E9441B382E06C
:10DF400090E002C081E090E02E960FB6F894DEBF1C
:10DF50000FBECDBFDF91CF911F910F91089580919A
:10DF600021058630D8F496E0899FF0011124EF5BFB
:10DF7000FA4F20917A1330917B13318320834091A3
:10DF8000110F5091120F6091130F7091140F428373
:10DF90005383648375838F5F80932105089540E0E8
:10DFA00050E0BA0187ED96EDF4CCE0912105EE2327
:10DFB00081F0E150E093210586E0E89FF001112413
:10DFC000EF5BFA4F42815381648175818081918139
:10DFD000E0CCE5CFCF93DF9300D01F92CDB7DEB773
:10DFE0000F941E4C0F948D4669837A838B839C8398
:10DFF000CE0101960E94BF5C0F900F900F900F9082
:10E00000DF91CF910895CF93DF9300D01F92CDB7CA
:10E01000DEB769837A838B839C83CE0101960E944D
:10E020004AEA0F900F900F900F90DF91CF910895D3
:10E030000F948F462FE632E143E85AE30F94EE4601
:10E04000E2CFCF92DF92EF92FF926B017C0120E052
:10E0500030E0A9010F94894687FD05C020E030E03B
:10E0600040E05FE304C020E030E040E05FEBC70148
:10E07000B6010F94D54A0F94194CCB01FF90EF9045
:10E08000DF90CF900C94395F0F948F46DACFCF9307
:10E09000C4E0C15048F088E0C89FB0011124655524
:10E0A000774E8C2F5ADEF5CFCF910895823009F448
:10E0B000EECF6CE878E180E050DE64E878E181E062
:10E0C0004CDE6CE778E182E048DE64E778E186E0E8
:10E0D00044DE6CE678E187E040DE64E678E183E0E8
:10E0E0003CDE6CE578E184E038DE64E578E185E0EB
:10E0F00034CE64E084E10F94AB2481E020917A1364
:10E1000030917B13275D364D09F080E0CFDF0D9411
:10E11000A4244FEF5FEFA6CEAF92BF92CF92DF92D3
:10E12000EF92FF920F931F93CF93DF9300D01F9234
:10E13000CDB7DEB76C015B017A0100E010E00E158F
:10E140001F05E0F419821A821B821C82AE014F5F08
:10E150005F4FB501C6010E9443D56C0169817A8188
:10E160008B819C81611571058105910539F0A701AD
:10E17000401B510B77DE080F191FE1CFC8010F902C
:10E180000F900F900F90DF91CF911F910F91FF9003
:10E19000EF90DF90CF90BF90AF9008954FEF5FEF7B
:10E1A0006AEE74EDB9CFAB016DEE74EDB5CF6FEFE4
:10E1B0007FEFF9CF643008F063E090917513691731
:10E1C00010F06FEF690FE62FF0E0EE59FC4E9489E6
:10E1D000890F80680D949E24EF92FF921F93CF9336
:10E1E000DF937C01EB0161E081E0E4DFC701D6DF72
:10E1F000209721F16AE370E080E090E08ADFCE01B1
:10E200000E94B6D6182FC7010E9495D690E00196BD
:10E21000810F911D429714F461E001C062E082E138
:10E22000811BC8DF60E270E080E090E072DFCE0129
:10E23000DF91CF911F91FF90EF90B9CFDF91CF91F8
:10E240001F91FF90EF9008950F931F93CF93DF934B
:10E25000FC01EB018091110F9091120FA091130F0F
:10E26000B091140FB7FF08C01092110F1092120F47
:10E270001092130F1092140F8091150F9091160F9A
:10E28000A091170FB091180F4091110F5091120FDC
:10E290006091130F7091140F84179507A607B707A5
:10E2A00044F48093110F9093120FA093130FB09327
:10E2B000140F809150028823F9F04091110F509172
:10E2C000120F6091130F7091140F8091190F90919C
:10E2D0001A0FA0911B0FB0911C0F8A019B01080F10
:10E2E000191F2A1F3B1FC901B8011995BC01809154
:10E2F0001F0F9091200F70DF8091050F811108C0D2
:10E3000080910E0F8823C9F1809150028823A9F1D2
:10E3100080911D0F90911E0F0097B1F00091110F89
:10E320001091120F2091130F3091140F4091190F7B
:10E3300050911A0F60911B0F70911C0F400F511FCD
:10E34000621F731FFE011995E0910F0FF091100FDE
:10E35000309741F080910E0F811103C08091050F1D
:10E36000811119958091050F1092050F882329F0CE
:10E37000DF91CF911F910F9118CEDF91CF911F9117
:10E380000F91089566EC7DE688E49EE65DCF6AED28
:10E390007DE685E69EE658CF6EEE7DE688E190E765
:10E3A00053CF6EE97DE682E89EE64ECF62E07EE6E0
:10E3B00084E490E749CF60E17EE68FE99EE644CFB2
:10E3C0006DE17EE686EA9EE63FCFCF92DF92EF9246
:10E3D000FF920F931F93CF93DF93D82F162F6A01CD
:10E3E0007901C901002319F00E9495D602C00E944C
:10E3F000B6D6C2E1C81B612F80E0DCDED11105C0BA
:10E4000060E270E080E090E004C06EE370E080E0E5
:10E4100090E07FDE4C2F50E06AEE74EDC6017CDEAA
:10E42000C81B6AE370E080E090E073DECC2339F033
:10E4300060E270E080E090E06CDEC150F7CFC70191
:10E44000002349F0DF91CF911F910F91FF90EF9042
:10E45000DF90CF90A3CEDF91CF911F910F91FF90CE
:10E46000EF90DF90CF90A3CEEF92FF920F93CF93D8
:10E47000DF93D82F7A01C22F80E09CDEDD2331F0BC
:10E480006C2FCC0F770B880B990B04C060E270E007
:10E4900080E090E03EDE42E150E06AEE74EDC701BC
:10E4A0003BDEC2E1C81BCC2339F060E270E080E0C3
:10E4B00090E02FDEC150F7CF602F000F770B880B55
:10E4C000990BDF91CF910F91FF90EF9022CEEF92B9
:10E4D000FF920F931F93CF93DF937B01C42F682F7D
:10E4E00080E068DECC23F1F001151105D9F4C701F5
:10E4F0000E9495D624E130E0A901481B5109CA01C8
:10E5000057FD019695958795C4E1DBEED80F8D2FC9
:10E510008C0F87FD08C060E270E080E090E0F9DDDC
:10E52000C150F5CFC4E14C2F0C2E000C550B6AEEF8
:10E5300074EDC701F1DDC81B0115110539F06C2F11
:10E540000C2E000C770BC8012EDEC81B1C163CF4E9
:10E5500060E270E080E090E0DCDDC150F7CFDF9159
:10E56000CF911F910F91FF90EF9008950F931F93FC
:10E57000CF93DF938C010E9495D62CE030E0A90167
:10E58000481B5109CA0157FD0196EC01D595C79565
:10E5900060E08C2F0FDE60E070E0CB01BADD84EA32
:10E5A00098E1FCDD61E070E080E090E0B2DD61E0E8
:10E5B0008C2F00DE8BE998E1F1DDC801EFDD62E030
:10E5C0008C2FF8DD62E070E080E090E0A2DD84E96D
:10E5D00098E1E4DD63E070E080E090E0DF91CF91CE
:10E5E0001F910F9196CD0F931F93CF93DF938C01C3
:10E5F00067FF03C01092C90F60E08091C90F90E0DF
:10E60000262F062E000C330B281739071CF16093B8
:10E61000C90FC8010F94D945800F911FEC01C01B91
:10E62000D10BC334D1053CF00197FC012491207C2F
:10E630002038D1F3F3CFDD27AE01B80186E89FE0A3
:10E640000F94FA45CA57D04F18821092850F83E075
:10E6500080935002DF91CF911F910F910895CF9336
:10E66000DF932091C90F21111FC0FC0101900020F0
:10E67000E9F73197EF01C81BD90BC334D1052CF052
:10E680002291207C2038E1F3F5CFBC01DD27AE01DB
:10E6900086E89FE00F948F4ECA57D04F1882109291
:10E6A000850F83E080935002DF91CF910895809190
:10E6B000951482FD05C08091DE0E823061F410C099
:10E6C0008091300F882319F080E39FE002C083E23D
:10E6D0009FE061E0C4CF813031F489E69EE005C05F
:10E6E00085E79EE002C082E59EE06FEF7CCF0F934E
:10E6F0001F930E9473B200913D0510913E05209139
:10E700003F0530914005DC01CB01801B910BA20B32
:10E71000B30BB7FD0CC086B186FB992790F981E059
:10E720008927349B8260329B846080933C05809172
:10E730003C05817090913C0591FD826090913B0574
:10E74000891731F18130A9F028F0823041F083300F
:10E7500059F01CC0913089F0923099F017C099237C
:10E7600061F0933071F012C0913059F0923071F431
:10E7700004C0992331F0933049F490912F059150C2
:10E7800003C090912F059F5F90932F0580933B05C9
:10E790001F910F9108954F925F926F927F928F9287
:10E7A0009F92AF92BF92CF92DF92EF92FF920F9320
:10E7B0001F93CF93DF938091EA0581111EC0809152
:10E7C0000B028F3FD1F00E9473B20091E2051091CD
:10E7D000E3052091E4053091E505DC01CB01801BC8
:10E7E000910BA20BB30BB7FD08C080911013909151
:10E7F00011138F5F8F708913C3C179DF80913C053E
:10E8000082FF39C080913A05811137C091E0909321
:10E810003A052091800F211103C08091471089276C
:10E820008093050F1092800F83E080935002109226
:10E830003C050E9473B2DC01CB018C509E4FAF4F60
:10E84000BF4F80933D0590933E05A0933F05B09345
:10E85000400568E873E182E090E00E94EC9FC6E02A
:10E86000C15059F00E94309C62E070E080E090E07E
:10E870000E943BB2F5CF10923A0580910901817058
:10E8800091E09827C0912E05C917B9F090932E05F5
:10E890008111D4C164EF71E080E090E00E94925F4A
:10E8A0000E94C4B3C23009F0C4C110927C130E940C
:10E8B00046B383E0809350021CDC0E9473B26B016C
:10E8C0007C018091360590913705A0913805B09173
:10E8D0003905A7019601281B390B4A0B5B0B57FD25
:10E8E00030C2D701C6018C599F4FAF4FBF4F8093A5
:10E8F000360590933705A0933805B093390560919C
:10E900002F05062E000C770B77FF03C071956195DC
:10E910007109062E000C770B880B990B0F948F460C
:10E920002B013C0120E030E040E450E40F94494DDD
:10E9300087FF06C08091050F882309F494C082C028
:10E940008091760F882309F456C08090720F9090C2
:10E95000730FA090740FB090750F81149104A104EF
:10E96000B104E1F120E030E040E450E4C301B20141
:10E970000F94B14B2B013C01C701B601681979090D
:10E980008A099B090F948D469B01AC01C301B2011A
:10E990000F94B14B20E030E04AE754E40F94EE4688
:10E9A0004B015C0120E030E040EA52E40F94494D15
:10E9B00087FF0FC020E030E040EF51E4C501B40113
:10E9C0000F94494D87FD0AC02AE030E040E050E056
:10E9D00009C024E630E040E050E004C021E030E02F
:10E9E00040E050E0C092720FD092730FE092740F2B
:10E9F000F092750F04C021E030E040E050E0A091BB
:10EA00002F050A2E000CBB0B0F94BF4A23E030E009
:10EA100040E050E00F94994A8091110F9091120FAD
:10EA2000A091130FB091140F820F931FA41FB51F55
:10EA30008093110F9093120FA093130FB093140FA4
:10EA400010922F05D701C6018856954CAF4FBF4F86
:10EA50008093320590933305A0933405B093350528
:10EA600081E08093500220917A1330917B1346ED20
:10EA7000273D340741F480914F02882309F4F6C002
:10EA8000815080934F022451334971F48091210FBA
:10EA90009091220F891740F490914F02992309F425
:10EAA000F5C0915090934F0280916F00282F2270F3
:10EAB00081FF05C080916F008D7F80936F008091F2
:10EAC000AE069091AF06A091B006B091B106222398
:10EAD00029F020916F00226020936F002091500256
:10EAE000222309F440C04AE0B695A79597958795EB
:10EAF0004A95D1F7009731E0A307B10520F08FEFD9
:10EB00009FEFA0E0B0E096958795009709F4D6C0F6
:10EB100040913005509131054817590708F4CEC08F
:10EB200022C0243011F410925002E0917A13F09137
:10EB30007B1319951092050F0E9473B2DC01CB0173
:10EB40008C199D09AE09BF0900913005109131055E
:10EB500020E030E0081719072A073B0720F49093BC
:10EB600031058093300580917A1390917B13875DF6
:10EB7000964D09F4ADC08091C4058111A9C0D1C0E2
:10EB8000C0904702D0904802E0904902F0904A02BB
:10EB9000E0910B0254E0E502F0011124E859FD4F29
:10EBA00020E030E040E752E460817181828193810E
:10EBB0000F94B14B609347027093480280934902CF
:10EBC00090934A020E94BB50C0910B0284E0C8029D
:10EBD000E0011124C357D14F2091E6053091E7059C
:10EBE0004091E8055091E905688179818A819B818E
:10EBF0000F94D54A688379838A839B831092E605B4
:10EC00001092E7051092E8051092E9058FEF8093C6
:10EC10000B0281E08093EA050E943FCF1092EA0543
:10EC2000C0924702D0924802E0924902F0924A0212
:10EC3000E4CD60E084E49EE0D6DC3BCE0E9450B39D
:10EC400080919514877F80939514C23009F431CE5A
:10EC500060E087E39EE0C7DC80917A1390917B139C
:10EC6000875D964D09F425CE9AD923CE89E080930D
:10EC70004F028091300590913105019790933105B5
:10EC80008093300581E080935002FDCE96E0909312
:10EC90004F0291E0909350028F5F8093210FD70134
:10ECA000C6018856954CAF4FBF4F80933205909365
:10ECB0003305A0933405B0933505F6CE223008F421
:10ECC00034CF243008F02DCF81E0809350022DCF37
:10ECD00028E9C20E2AE3D21EE11CF11CC0923205C3
:10ECE000D0923305E0923405F092350580915002C0
:10ECF0008130A1F0833029F5DF91CF911F910F91E1
:10ED0000FF90EF90DF90CF90BF90AF909F908F904B
:10ED10007F906F905F904F900D94A42410925002BA
:10ED200010C08091320590913305A0913405B091C7
:10ED30003505C81AD90AEA0AFB0AF7FCD7CF2FD93A
:10ED4000D5CFDF91CF911F910F91FF90EF90DF9082
:10ED5000CF90BF90AF909F908F907F906F905F907B
:10ED60004F9008952F923F924F925F926F927F92B1
:10ED70008F929F92AF92BF92CF92DF92EF92FF92CB
:10ED80000F931F93CF93DF93CDB7DEB72F970FB6B7
:10ED9000F894DEBF0FBECDBF8FEF9FEF9093890039
:10EDA00080938800BAE0DB2E1F861E8678948091BF
:10EDB000AD059091AE05A091AF05B091B005892B3E
:10EDC0008A2B8B2B09F0D5C18091F4158823D1F0C3
:10EDD0001092F4158091F2159091F315892B91F012
:10EDE00010926E051092F3151092F2159091101377
:10EDF00080911113981731F0809111138F5F8F70EC
:10EE0000809311138091F2159091F315892B09F4D9
:10EE1000B0C10091A9051091AA052091AB053091D0
:10EE2000AC058091A5059091A605A091A705B0918C
:10EE3000A80540919C0550E060E070E0801B910BBC
:10EE4000A20BB30B481759076A077B0710F4DB01C5
:10EE5000CA01482F800F911FA21FB31F8093A905DD
:10EE60009093AA05A093AB05B093AC058091840064
:10EE70009091850080968090830590908405A09065
:10EE80008505B09086050091730510917405209159
:10EE9000750530917605080D191D2A1D3B1D00933F
:10EEA000830510938405209385053093860537FDEF
:10EEB0001CC0889A00910116109102162091031629
:10EEC0003091041680906505082C000C9908AA085A
:10EED000BB08080D191D2A1D3B1D00930116109338
:10EEE00002162093031630930416809087059090A5
:10EEF0008805A0908905B0908A050091770510914A
:10EF000078052091790530917A05080D191D2A1D83
:10EF10003B1D009387051093880520938905309346
:10EF20008A0537FD1CC08E9A0091051610910616B1
:10EF3000209107163091081680906605082C000C69
:10EF40009908AA08BB08080D191D2A1D3B1D00932E
:10EF50000516109306162093071630930816809016
:10EF60008B0590908C05A0908D05B0908E0500913A
:10EF70007B0510917C0520917D0530917E05080D63
:10EF8000191D2A1D3B1D00938B0510938C052093A2
:10EF90008D0530938E0537FD21C020910B01209502
:10EFA0002870209309010091091610910A162091EA
:10EFB0000B1630910C1680906705082C000C9908F0
:10EFC000AA08BB08080D191D2A1D3B1D0093091630
:10EFD00010930A1620930B1630930C1680908F0511
:10EFE00090909005A0909105B090920500917F05BA
:10EFF000109180052091810530918205080D191D21
:10F000002A1D3B1D00938F051093900520939105B9
:10F010003093920537FD1CC0149A00910D16109183
:10F020000E1620910F163091101680906805082C4E
:10F03000000C9908AA08BB08080D191D2A1D3B1DC4
:10F0400000930D1610930E1620930F163093101682
:10F05000209184003091850028173907C8F300916A
:10F06000830510918405209185053091860537FD33
:10F0700015C080906F0590907005A0907105B090BC
:10F080007205081919092A093B0900938305109391
:10F09000840520938505309386058898009187051F
:10F0A000109188052091890530918A0537FD15C09A
:10F0B00080906F0590907005A0907105B0907205DA
:10F0C000081919092A093B09009387051093880537
:10F0D0002093890530938A058E9800918B051091B5
:10F0E0008C0520918D0530918E0537FD19C08090DB
:10F0F0006F0590907005A0907105B0907205081989
:10F1000019092A093B0900938B0510938C0520935C
:10F110008D0530938E0520910B01287020930901F5
:10F1200000918F05109190052091910530919205E5
:10F1300037FD15C080906F0590907005A090710507
:10F14000B0907205081919092A093B0900938F0527
:10F150001093900520939105309392051498415097
:10F1600041F0209184003091850028173907C8F3B9
:10F1700081CE8091AD059091AE05A091AF05B09183
:10F18000B005892B8A2B8B2B09F0C1C5E091F215B4
:10F19000F091F315309709F440C78091A90590913B
:10F1A000AA05A091AB05B091AC054091A505509181
:10F1B000A6056091A7057091A80584179507A60775
:10F1C000B707D0F010926E051092F3151092F21559
:10F1D0009091101380911113981709F41EC7809114
:10F1E00011138F5F8F7080931113A0ED4A2EA7E04B
:10F1F0005A2E612C712CE5C34091A1055091A205B6
:10F200006091A3057091A405481759076A077B0709
:10F2100008F4A4C180909D0590909E05A0909F0544
:10F22000B090A00585A996A9A7A9B0AD88169906A2
:10F23000AA06BB0608F076C181149104A104B104AA
:10F2400049F480916A0590916B05A0916C05B0918D
:10F250006D0564C1B0E0AC2D882D392D2A2DF981C2
:10F26000EA817B816C815D814E819F815091F30E9B
:10F27000589F712D66274091F40E489F700D611DB7
:10F280001090F50E189E600D539F700D611D439FE9
:10F29000600D529F600DF72FE62FF79F512D4427E9
:10F2A0009927F69F500D411D9B1FE79F500D411D53
:10F2B0009B1FE69F400D911DF42FE92FF79FA12D75
:10F2C00044279927F69FA00D411D9B1FE79FA00D86
:10F2D000411D9B1FE69F400D911DF42FE92F5527DF
:10F2E00080916A0530916B0520916C0500900205B4
:10F2F0000B2A09F483C04091FE044F9F51198B0BD8
:10F300003B0B2B0B9091FF049F9F501981093B0BE6
:10F310002B0BA0910005AF9F801931092B0B4E9F3D
:10F32000501981093B0B2B0B9E9F801931092B0B28
:10F33000AE9F30192109F79FA12D44279927F69FE9
:10F34000A00D411D9B1FE79FA00D411D9B1FE69F28
:10F35000400D911DF42FE92F4091FA044F9F510D5C
:10F360008B1F3B1F2B1F9091FB049F9F500D811DF6
:10F370003B1F2B1FA091FC04AF9F800D311D2B1F45
:10F380004E9F500D811D3B1F2B1F9E9F800D311DD9
:10F390002B1FAE9F300D211DF79FA12D44279927CC
:10F3A000F69FA00D411D9B1FE79FA00D411D9B1FB8
:10F3B000E69F400D911DF42FE92F4091F6044F9FD9
:10F3C00051198B0B3B0B2B0B9091F7049F9F5019FE
:10F3D00081093B0B2B0BA091F804AF9F80193109D9
:10F3E0002B0B4E9F501981093B0B2B0B9E9F8019B5
:10F3F00031092B0BAE9F3019210982C04091FE04C8
:10F400004F9F510D8B1F3B1F2B1F9091FF049F9F00
:10F41000500D811D3B1F2B1FA0910005AF9F800D3C
:10F42000311D2B1F4E9F500D811D3B1F2B1F9E9F7B
:10F43000800D311D2B1FAE9F300D211DF79FA12D7B
:10F4400044279927F69FA00D411D9B1FE79FA00D04
:10F45000411D9B1FE69F400D911DF42FE92F409108
:10F46000FA044F9F51198B0B3B0B2B0B9091FB0414
:10F470009F9F501981093B0B2B0BA091FC04AF9F60
:10F48000801931092B0B4E9F501981093B0B2B0B17
:10F490009E9F801931092B0BAE9F30192109F79FD0
:10F4A000A12D44279927F69FA00D411D9B1FE79F83
:10F4B000A00D411D9B1FE69F400D911DF42FE92FCC
:10F4C0004091F6044F9F510D8B1F3B1F2B1F9091B6
:10F4D000F7049F9F500D811D3B1F2B1FA091F80427
:10F4E000AF9F800D311D2B1F4E9F500D811D3B1F67
:10F4F0002B1F9E9F800D311D2B1FAE9F300D211D98
:10F500001124CA2EF983EA837B836C835D834E8347
:10F510009F8390E0932BA0E0B0E0A22B2BEC30E295
:10F5200011E011C081A992A9A3A9B4A9F7CFB695FA
:10F53000A79597958795110F2C5F3F4F40E2273E87
:10F54000340709F439C4F9014591559165917491D5
:10F55000481759076A077B0750F32EC44091980556
:10F560005091990560919A0570919B05481759072C
:10F570006A077B0708F0B8C18091970581111FC009
:10F58000DF01AF5BBF4FED90FD900D911C91139784
:10F590001D962D913D914D915C9161A972A983A910
:10F5A00094A90E94F7E051E050939705E091F2157D
:10F5B000F091F31581A892A8A3A8B4A886C1809160
:10F5C000930590919405A0919505B091960541AD54
:10F5D00052AD63AD74AD84179507A607B70708F061
:10F5E0006EC10097A105B10549F480906A0590901D
:10F5F0006B05A0906C05B0906D0567C130E0488543
:10F60000882E292F8A2FE9857A856B855C859D85D3
:10F610009091F30E989D612D55272090F40E289C13
:10F62000600D511D1090F50E189C500D929F600DAD
:10F63000511D229E500D989F500DE62F752FE69F6D
:10F64000912D22243324E59F900D211C331E769F9B
:10F65000900D211C331E759F200C311CE22D732D43
:10F66000E69F412D22243324E59F400D211C331EAB
:10F67000769F400D211C331E759F200C311CE22DFE
:10F68000732D992780906A0520916B0580916C05F8
:10F6900000900205032A09F483C02090FE042E9EE8
:10F6A0009119830A230B830B3090FF043E9E90191F
:10F6B0008108230B830B409100054E9F8018210980
:10F6C000830B279E90198108230B830B379E80188C
:10F6D0002109830B479F20198109E69F412D222490
:10F6E0003324E59F400D211C331E769F400D211CC5
:10F6F000331E759F200C311CE22D732D2090FA04CF
:10F700002E9E910D831E231F831F3090FB043E9E6F
:10F71000900D811C231F831F4091FC044E9F800C81
:10F72000211D831F279E900D811C231F831F379E41
:10F73000800C211D831F479F200D811DE69F412DB9
:10F7400022243324E59F400D211C331E769F400D5B
:10F75000211C331E759F200C311CE22D732D20902F
:10F76000F6042E9E9119830A230B830B3090F70425
:10F770003E9E90198108230B830B4091F8044E9F05
:10F7800080182109830B279E90198108230B830B76
:10F79000379E80182109830B479F2019810982C059
:10F7A0002090FE042E9E910D831E231F831F3090F8
:10F7B000FF043E9E900D811C231F831F4091000576
:10F7C0004E9F800C211D831F279E900D811C231F9F
:10F7D000831F379E800C211D831F479F200D811D95
:10F7E000E69F412D22243324E59F400D211C331E2A
:10F7F000769F400D211C331E759F200C311CE22D7D
:10F80000732D2090FA042E9E9119830A230B830BEB
:10F810003090FB043E9E90198108230B830B40918E
:10F82000FC044E9F80182109830B279E90198108A4
:10F83000230B830B379E80182109830B479F2019C8
:10F840008109E69F412D22243324E59F400D211C90
:10F85000331E769F400D211C331E759F200C311CDA
:10F86000E22D732D2090F6042E9E910D831E231FF2
:10F87000831F3090F7043E9E900D811C231F831F31
:10F880004091F8044E9F800C211D831F279E900DF0
:10F89000811C231F831F379E800C211D831F479FC0
:10F8A000200D811D11244887E9877A876B875C8743
:10F8B0009D87912C922AA12CB12CA82A06C0E25B2C
:10F8C000FF4F80809180A280B3808BEC90E221E09A
:10F8D000FC014591559165917491481559056A054A
:10F8E0007B0508F4CCC2D6C2809107029091080231
:10F8F000A0910902B0910A02B7FF5BC0EA5BFF4F1B
:10F9000080809180A280B3808BEC90E221E0FC01AA
:10F910004591559165917491481559056A057B0586
:10F9200050F4B694A79497948794220F0496A0E27B
:10F93000873E9A0761F720939C0580E28816910420
:10F94000A104B10408F43AC320E2821A9108A10884
:10F95000B108811438E09306A104B10408F40AC385
:10F9600044E0949EC00111248553934EFC013296CD
:10F9700025913491782D6627739FA001729F410DC8
:10F98000561F0694461F561F112460E070E0FC01CC
:10F9900025913491C901A0E0B0E0841B950BA60B22
:10F9A000B70B8093070290930802A0930902B093CB
:10F9B0000A0240900702509008026090090270907D
:10F9C0000A028091F2159091F315892B09F097C1E5
:10F9D0000E947FE19093F3158093F215892B09F42F
:10F9E0008EC1E091F215F091F315808183FF3EC046
:10F9F00085899689A789B08D809301169093021608
:10FA0000A0930316B0930416818D928DA38DB48DAF
:10FA10008093051690930616A0930716B0930816C8
:10FA2000858D968DA78DB0A18093091690930A16A7
:10FA3000A0930B16B0930C1681A192A1A3A1B4A11F
:10FA400080930D1690930E16A0930F16B093101678
:10FA50009091101380911113981709F4B9CF8091E8
:10FA600011138F5F8F7080931113B2CF05891689A0
:10FA70002789308D81E0011511052105310509F433
:10FA800080E0818C928CA38CB48C81149104A104AD
:10FA9000B10409F08260458D568D678D70A14115C6
:10FAA00051056105710509F0846080936E0510921F
:10FAB0009305109294051092950510929605109258
:10FAC0009D0510929E0510929F051092A00585A19C
:10FAD00096A1A7A1B0A58093A5059093A605A09394
:10FAE000A705B093A805442455243201481A590AA1
:10FAF0006A0A7B0A40928F055092900560929105A8
:10FB00007092920540928B0550928C0560928D0503
:10FB100070928E0540928705509288056092890503
:10FB200070928A0540928305509284056092850503
:10FB300070928605000F111F221F331F009373055B
:10FB4000109374052093750530937605880C991CE5
:10FB5000AA1CBB1C8092770590927805A09279052B
:10FB6000B0927A05440F551F661F771F40937B059F
:10FB700050937C0560937D0570937E0541A152A151
:10FB800063A174A1440F551F661F771F40937F0523
:10FB9000509380056093810570938205880F991FAB
:10FBA000AA1FBB1F80936F0590937005A0937105EA
:10FBB000B09372051092A9051092AA051092AB0598
:10FBC0001092AC0581A592A5A3A5B4A58093A1052B
:10FBD0009093A205A093A305B093A40585A596A52F
:10FBE000A7A5B0A98093980590939905A0939A052D
:10FBF000B0939B05EB5BFF4F80819091690589175E
:10FC000021F0809369050E9449E10F9476208FEFDF
:10FC10009FEFDC018093070290930802A0930902F2
:10FC2000B0930A02E091F215F091F315DF01DD9631
:10FC3000ED90FD900D911C9121A932A943A954A9E1
:10FC4000E65BFF4F60817181828193810E94F7E0C2
:10FC500010929705E091F215F091F315E65BFF4FD6
:10FC600080809180A280B3808BEC90E221E0FC0147
:10FC70004591559165917491481559056A057B0523
:10FC800058F4B694A79497948794220F049647EE5D
:10FC900050E24817590759F720939C05B0E28B169C
:10FCA0009104A104B10408F4B2C190E2891A910848
:10FCB000A108B1088114A8E09A06A104B10408F4CF
:10FCC00083C1B4E09B9EC00111248553934EFC0177
:10FCD000329625913491782D6627739FA001729FEB
:10FCE000410D561F0694461F561F1124FC014590D6
:10FCF0005490612C712C441A550A61087108409285
:10FD0000AD055092AE056092AF057092B00580913E
:10FD1000AD059091AE05A091AF05B091B005AC01D5
:10FD2000BD01009721E0A207B10520F04FEF5FEF82
:10FD300060E070E0841B950BA60BB70B8093AD05BC
:10FD40009093AE05A093AF05B093B005F894809161
:10FD50008400909185004096DA94DD2059F0AE85BC
:10FD6000BF85A40FB51FBF87AE87A817B90708F4D2
:10FD70001DC802C09F878E872E853F8530938900DE
:10FD80002093880078942F960FB6F894DEBF0FBEAC
:10FD9000CDBFDF91CF911F910F91FF90EF90DF903A
:10FDA000CF90BF90AF909F908F907F906F905F901B
:10FDB0004F903F902F90089510939C0580329105AD
:10FDC000A105B10508F456C08097A109B1098115B4
:10FDD00028E09207A105B105F0F044E0949F90015E
:10FDE00011242553334EF901329645915491EE2753
:10FDF000859FB001849F610D7E1F06946E1F7E1F3C
:10FE00001124F90145905490612C712C461A570A1F
:10FE10006108710822C0AC01BD01769567955795C0
:10FE20004795FA01EC7FAF014553574EFA012591F2
:10FE30003491FA013296659174918770869FA00182
:10FE4000879F500D1124F3E056954795FA95E1F7F9
:10FE50002901441A550A612C712C840C951CA61C8E
:10FE6000B71C80929D0590929E05A0929F05B0922E
:10FE7000A005A7CD80E290E0A0E0B0E0A5CFB694C9
:10FE8000A79497948794220F049650E2873E950793
:10FE900009F01ECD20939C0570E287169104A10401
:10FEA000B10408F461C070E2871A9108A108B10892
:10FEB000811488E09806A104B104F8F0A4E09A9EA9
:10FEC000C00111248553934EFC0132962591349143
:10FED000B82D6627B39FA001B29F410D561F06940F
:10FEE000461F561F1124FC0145905490612C712C23
:10FEF000441A550A6108710822C0D501C401B6959B
:10FF0000A79597958795FC01EC7FCF018553974E78
:10FF1000FC0145905490FC01329625913491482D76
:10FF20004770429FC001439F900D112463E0969556
:10FF300087956A95E1F7481A590A612C712C8091CE
:10FF4000930590919405A0919505B0919605840D27
:10FF5000951DA61DB71D8093930590939405A093BE
:10FF60009505B09396052DCD70E2872E912CA12C8E
:10FF7000B12C99CFD501C401B695A79597958795D2
:10FF8000FC01EC7FCF018553974EFC012591349104
:10FF9000FC01329645915491682D6770649FC001B1
:10FFA000659F900D112443E0969587954A95E1F75A
:10FFB000281B390BC901A0E0B0E0F3CC60E2862E2B
:10FFC000912CA12CB12CC0CCD501C401B695A7951C
:10FFD00097958795FC01EC7FCF018553974EFC01E7
:10FFE00045905490FC01329625913491482D4770EC
:10FFF000429FC001439F900D112403E09695879581
:020000021000EC
:100000000A95E1F7481A590A612C712C78CE40E222
:10001000842E912CA12CB12C48CE80ED482E87E067
:10002000582E612C712CD4CCEF92FF920F93CF936A
:10003000DF9361E081E00E948F66D0910B0FC0E0FA
:1000400083E5E82E82E2F82ED1110BC080910A0FD1
:10005000811129C08091050F1092050F81111DC0DB
:1000600022C0D13059F480910A0F8130A1F58091DE
:10007000050F1092050F811124C02DC0D23009F058
:1000800074C080910A0F823009F091C08091050FF1
:100090001092050F811185C08AC00E94D56F809192
:1000A000090F811158C180915002882329F181E004
:1000B00090910A0F911180E003E023E047E552E2BE
:1000C00018C0F092F205E092F1050E941658809156
:1000D000090F811140C180915002882369F081E0AD
:1000E00090910A0F913009F080E000E22EE342E4A3
:1000F00052E26C2F0E94347280917F0F877087309C
:1001000059F5D63061F480910A0F863009F0BCC0F1
:100110008091050F1092050F8111AEC0B5C0D73088
:1001200061F480910A0F873009F0C6C08091050FF5
:100130001092050F8111B8C0BFC0D83009F0CEC0F1
:1001400080910A0F883009F0DEC08091050F10926F
:10015000050F8111D0C0D7C086E0CF5FDF5FC4300C
:1001600009F072CF8093080FF6C0D33061F480910C
:100170000A0F833009F040C08091050F1092050FDF
:10018000811134C039C0D43011F580910A0F843008
:1001900009F04AC08091050F1092050F81113CC0F3
:1001A00043C00E948C668091090F8111D4C0809158
:1001B0005002882309F4A0CF81E090910A0F923079
:1001C00009F080E000E22EE343E352E292CFD53023
:1001D00009F092CF80910A0F853009F03DC08091DF
:1001E000050F1092050F81112FC036C00E9489663D
:1001F0008091090F8111AFC080915002882309F4CA
:100200007BCF81E090910A0F933009F080E000E20B
:100210002EE344E152E26DCF84EC91E80E945E6DE2
:100220008091090F811197C080915002882309F4B1
:1002300063CF81E090910A0F943009F080E00EE3E3
:100240002EE345E052E255CF81EB91E80E945E6DCE
:100250008091090F81117FC080915002882309F499
:100260004BCF81E090910A0F953009F080E00EE3CA
:100270002EE34BEF51E23DCF84E195E80E945E6DA5
:100280008091090F811167C080915002882309F481
:100290003EC081E090910A0F963009F080E00EE3B5
:1002A0002EE34FEE51E216C085E595E80E945E6DA3
:1002B0008091090F81114FC080915002882339F13C
:1002C00081E090910A0F973009F080E00EE32EE371
:1002D00043EE51E26C2F0E94347219C0D930B9F448
:1002E00080910A0F893041F58091050F1092050F1A
:1002F00081111AC021C086E995E80E945E6D809147
:10030000090F811128C080915002811102C08AE03A
:1003100024CF81E090910A0F983009F080E00EE33D
:100320002EE347ED51E2D6CF85EC95E80E945E6D55
:100330008091090F81110FC080915002882339F3F9
:1003400081E090910A0F993009F080E00EE32EE3EE
:1003500042E252E2BFCFDF91CF910F91FF90EF9039
:1003600008958FE691E29093F2058093F1050E9443
:10037000165840E050E0BA018BEA94E80C94C96C3E
:100380000E94CCF40D9437234F925F926F927F922C
:10039000AF92BF92CF92DF92EF92FF920F931F9393
:1003A000CF93DF9300D01F92CDB7DEB761E081E03D
:1003B0000E948F66A0900B0FB12CA1100BC08091F2
:1003C0000A0F81112BC08091050F1092050F81112A
:1003D0001FC024C081E0A8120CC080910A0F813098
:1003E00009F05AC08091050F1092050F811128C0A5
:1003F00053C082E0A8127BC080910A0F823009F0BE
:10040000AAC08091050F1092050F81118EC0A3C064
:100410000E94D56F8091090F81118AC2809150028C
:10042000882309F45BC081E090910A0F911180E06C
:1004300003E023E045EC51E26B2D0E9434724EC084
:10044000C090850ED090860EE090870EF090880EBA
:1004500020E030E040E251E4C701B6010F94D54AF4
:100460002B013C0120E030E040E251E4C701B6013D
:100470000F94D44A9B01AC0190ECC92E91E8D92E7F
:100480008301720165E87EE08EEB91E20F948B3F71
:100490008091090F81114CC2809150028823F1F0A4
:1004A00011E080910A0F813009F010E08091850EF3
:1004B0009091860EA091870EB091880E89839A83C1
:1004C000AB83BC83CE0101960E941E5C00E09C01C0
:1004D00047EB51E26B2D812F0E94E571B394A394F9
:1004E00084E0B8126ACF8AE08093080F21C283E0CB
:1004F000A8120CC080910A0F833009F06BC0809164
:10050000050F1092050F81114FC064C084E0A8123E
:100510003CC080910A0F843009F09BC08091050F88
:100520001092050F81117FC094C010ECC12E11E80C
:10053000D12EE12CF12C00EA10E420E030E040EA7A
:1005400050EC63EA7EE084EB91E20F94053F8091EA
:10055000090F8111EDC180915002882309F4BECFAB
:1005600011E080910A0F823009F010E06091A30E33
:100570007091A40E8091A50E9091A60E0E9403701A
:1005800000E09C0141EB51E2A5CF85E0A8123CC000
:1005900080910A0F853009F0B1C08091050F10924B
:1005A000050F81117FC0AAC0A0ECCA2EA1E8DA2EE7
:1005B000E12CF12C00EA10E420E030E040EA50ECBD
:1005C00067EA7EE08EEA91E20F94053F8091090F81
:1005D0008111AEC180915002882309F47FCF11E0D0
:1005E00080910A0F833009F010E06091A70E70919E
:1005F000A80E8091A90E9091AA0E0E94037000E0AF
:100600009C014BEA51E266CF86E0A8123CC0809183
:100610000A0F863009F0B7C08091050F1092050FC0
:1006200081119BC0B0C0E0ECCE2EE1E8DE2EE12CC3
:10063000F12C00EA10E420E030E040EA50EC6BEAF4
:100640007EE088EA91E20F94053F8091090F8111C5
:100650006FC180915002882309F440CF11E080914E
:100660000A0F843009F010E06091AB0E7091AC0E6F
:100670008091AD0E9091AE0E0E94037000E09C013F
:1006800045EA51E227CF87E0A81258C080910A0FAF
:10069000873009F0B7C08091050F1092050F8111C6
:1006A0009BC0B0C0C0904D10D0904E10E0904F1045
:1006B000F090501020E030E040EA50E4C701B6016D
:1006C0000F94D54A2B013C0120E030E040EA50E491
:1006D000C701B6010F94D44A9B01AC0170ECC72E40
:1006E00071E8D72E830172016DE470E18EE991E229
:1006F0000F948B3F8091090F81111AC18091500294
:10070000882309F4EBCE11E080910A0F853009F0BF
:1007100010E080914D1090914E10A0914F10B0912B
:10072000501089839A83AB83BC83CE0101960E94CB
:100730001E5C00E09C0147E951E2CCCE88E0A812A3
:100740003CC080910A0F883009F08CC08091050F61
:100750001092050F811170C085C050ECC52E51E874
:10076000D52EE12CF12C00EA10E420E030E040EA44
:1007700050EC61E570E184E991E20F94053F8091CE
:10078000090F8111D5C080915002882309F4A6CEAB
:1007900011E080910A0F863009F010E0609151104D
:1007A0007091521080915310909154100E940370D8
:1007B00000E09C0141E951E28DCE89E0A8128ECE85
:1007C00080910A0F893009F093C08091050F109233
:1007D000050F811161C08CC030ECC32E31E8D32EDF
:1007E000E12CF12C00EA10E420E030E040EA50EC8B
:1007F00065E570E18EE891E20F94053F8091090F65
:10080000811196C080915002882309F467CE11E0CF
:1008100080910A0F873009F010E0609155107091B7
:10082000561080915710909158100E94037000E06C
:100830009C014BE851E24ECE90ECC92E91E8D92EA6
:10084000E12CF12C00EA10E420E030E040EA50EC2A
:1008500069E570E188E891E20F94053F8091090F06
:10086000811166C080915002882309F437CE11E0CF
:1008700080910A0F883009F010E060915910709152
:100880005A1080915B1090915C100E94037000E000
:100890009C0145E851E21ECEC0904910D0904A100C
:1008A000E0904B10F0904C1020E030E040EA50E433
:1008B000C701B6010F94D54A2B013C0120E030E07E
:1008C00040EA50E4C701B6010F94D44A9B01AC0141
:1008D00080ECC82E81E8D82E8301720169E470E1B2
:1008E0008CE791E20F948B3F8091090F811120C01A
:1008F00080915002882309F4F1CD11E080910A0F14
:10090000893009F010E08091491090914A10A0912F
:100910004B10B0914C1089839A83AB83BC83CE017A
:1009200001960E941E5C00E09C0143E751E2D2CD9B
:100930000F900F900F900F90DF91CF911F910F911B
:10094000FF90EF90DF90CF90BF90AF907F906F902F
:100950005F904F9008950F931F93809150028823CA
:1009600049F000E010E020E041E064E671E281E05F
:100970000E94677284E08093500280917F0F87709D
:10098000873021F41F910F910C94D56F1F910F9117
:100990000895CF92DF92EF92FF920F931F93CF9320
:1009A000DF9300D01F92CDB7DEB719821A821B8267
:1009B0001C82FB012081318142815381FC016081D5
:1009C000718182819381FE0131966F01E12CF12CBE
:1009D00000EA10E40E9428D388E393E29093C305D1
:1009E0008093C2050E94696D8AE999E9A9E9BDE38E
:1009F0008093EB059093EC05A093ED05B093EE0585
:100A000040E050E0BA0184E792EA0E94C96C0F907E
:100A10000F900F900F90DF91CF911F910F91FF904A
:100A2000EF90DF90CF900895CF92DF92EF92FF92F8
:100A3000CF93DF93CDB7DEB728970FB6F894DEBF1C
:100A40000FBECDBFC090AA14D090AB14E090AC14F0
:100A5000F090AD1423E030E040E05FEBC701B60159
:100A60000F94EE466D837E838F83988725ED33EB5D
:100A70004DE55FEBC701B6010F94EE4669837A83BB
:100A80008B839C83BE016B5F7F4FCE01019681DF1C
:100A900028960FB6F894DEBF0FBECDBFDF91CF9181
:100AA000FF90EF90DF90CF900895CF92DF92EF927A
:100AB000FF92CF93DF93CDB7DEB728970FB6F894A8
:100AC000DEBF0FBECDBFC090AA14D090AB14E09093
:100AD000AC14F090AD1428EF3FEF4FEF5EEBC70181
:100AE000B6010F94EE466D837E838F8398872AED3F
:100AF00033EB4DE55FE3C701B6010F94EE46698322
:100B00007A838B839C83BE016B5F7F4FCE010196FE
:100B100040DF28960FB6F894DEBF0FBECDBFDF9141
:100B2000CF91FF90EF90DF90CF900895CF93DF9318
:100B3000CDB7DEB728970FB6F894DEBF0FBECDBF96
:100B40006091AA147091AB148091AC149091AD1483
:100B50006D837E838F8398872EE23DEB4BE353EBCF
:100B60000F94EE4669837A838B839C83BE016B5F0F
:100B70007F4FCE0101960DDF28960FB6F894DEBFA9
:100B80000FBECDBFDF91CF910895CF93DF93CDB747
:100B9000DEB728970FB6F894DEBF0FBECDBF1D821B
:100BA0001E821F82188619821A821B821C82BE0135
:100BB0006B5F7F4FCE010196ECDE28960FB6F8945E
:100BC000DEBF0FBECDBFDF91CF91089580E00D94C1
:100BD000340481E00D943404FF920F931F93CF935C
:100BE000DF9361E081E00E948F66C0910B0FD0E03F
:100BF000C1110BC080910A0F81111BC08091050F9C
:100C00001092050F81110FC014C0C13011F58091F1
:100C10000A0F813009F0FFC08091050F1092050F77
:100C20008111F1C0F8C00E94D56F8091090F811128
:100C30001DC180915002882361F081E090910A0FDC
:100C4000911180E003E023E04FE551E26D2F0E9417
:100C500034720E94BA6CF82E81110EC0C23071F449
:100C600080910A0F823009F0EEC08091050F10923A
:100C7000050F8111E0C0E7C012E001C013E01C13B2
:100C800022C080910A0F81130EC08091050F10922F
:100C9000050F882341F086EE95E80E945E6D8091F5
:100CA000090F8111E3C080915002882361F081E037
:100CB00090910A0F9C1380E00EE32EE34AE251E28A
:100CC0006D2F0E94347281E0810F8C1322C08091BD
:100CD0000A0F8C130EC08091050F1092050F882308
:100CE00041F089EE95E80E945E6D8091090F8111B7
:100CF000BDC080915002882361F081E090910A0F7D
:100D00009C1380E00EE32EE349E151E26D2F0E9437
:100D1000347282E0810F8C1320C080910A0F8C13F3
:100D20000CC08091050F1092050F882331F00E94AE
:100D30008C668091090F811199C08091500288239F
:100D400061F081E090910A0F9C1380E000E22EE3B5
:100D50004AE051E26D2F0E94347283E0810FF1105E
:100D60004AC08C1320C080910A0F8C130CC0809154
:100D7000050F1092050F882331F00E94896680913B
:100D8000090F811173C080915002882361F081E0C6
:100D900090910A0F9C1380E000E22EE34BEE50E2AC
:100DA0006D2F0E94347204E0010F0C1322C0809159
:100DB0000A0FC8130EC08091050F1092050F8823EB
:100DC00041F00F94F82C0E9475668091090F8111F3
:100DD0004DC080915002882361F081E090910A0F0C
:100DE000901380E000E22EE349EF50E26D2F0E9465
:100DF000347285E0810FDF5FCF5FD43009F0F8CE29
:100E00008093080F33C087ED90E00E945E6D809163
:100E1000090F81112BC080915002882309F419CF4A
:100E200081E090910A0F913009F080E00EE32EE30B
:100E30004DE451E20BCF84E190E80E945E6D809119
:100E4000090F811113C080915002882369F081E05D
:100E500090910A0F923009F080E00EE32EE34BE30D
:100E600051E26D2F0E94347213E02DCFDF91CF91AC
:100E70001F910F91FF900895EF92FF920F931F9390
:100E8000CF93DF93CDB7DEB7CB57D1090FB6F89428
:100E9000DEBF0FBECDBFE1961CAE1DAE1EAE1FAEB7
:100EA000E1978091340390913503A0913603B0917E
:100EB0003703E5968CAF9DAFAEAFBFAFE597E99630
:100EC0001FAE1EAEE99784E690E0EB969FAF8EAF23
:100ED000EB971092C1059E0129583F4F44E050E026
:100EE000BE016F587F4FCE0187589F4F0E944B60C5
:100EF000EB968EAD9FADEB970296EB969FAF8EAFC4
:100F0000EB97E9961FAE1EAEE99781E0EC968FAFA6
:100F1000EC979E0129583F4F41E050E0BE016558D3
:100F20007F4FCE0187589F4F0E944B609E012958EA
:100F30003F4F48E450E06CE87CE0CE0187589F4F7B
:100F40000E944B609E0129583F4F40E150E06AE803
:100F500076E0CE0187589F4F0E944B608AE097ED64
:100F6000A3EABCE3E1968CAF9DAFAEAFBFAFE19714
:100F70009E0129583F4F44E050E0BE0163597F4F26
:100F8000CE0187589F4F0E944B608E010F5F1F4F0D
:100F90008CE0F80111928A95E9F79E0129583F4F9C
:100FA0004CE050E0B801CE0187589F4F0E944B6043
:100FB00080E090E0A0E2B1E489839A83AB83BC83B4
:100FC0009E0129583F4F44E050E0B801CE018758B8
:100FD0009F4F0E944B60E1961CAE1DAE1EAE1FAE31
:100FE000E19783E0E6968FAFE69789839E012958C3
:100FF0003F4F44E050E0BE0163597F4FCE01875818
:101000009F4F0E944B609E0129583F4F41E050E0A6
:10101000BE016B587F4FCE0187589F4F0E944B6097
:101020009E0129583F4F41E050E0B801CE0187585A
:101030009F4F0E944B602AE0F22EFA949E0129589D
:101040003F4F44E050E0FF2049F0BE0163597F4F1D
:10105000CE0187589F4F0E944B60EFCF6FEE7EE02E
:10106000CE0187589F4F0E944B60E1961CAE1DAE8B
:101070001EAE1FAEE1979AE0F92EFA94FF2071F0B0
:101080009E0129583F4F44E050E0BE0163597F4F15
:10109000CE0187589F4F0E944B60EFCF89E0E696C4
:1010A0008FAFE69789839E0129583F4F41E050E07A
:1010B000BE016B587F4FCE0187589F4F0E944B60F7
:1010C0009E0129583F4F41E050E0B801CE018758BA
:1010D0009F4F0E944B609E0129583F4F44E050E0D3
:1010E00068E974E1CE0187589F4F0E944B609E01D2
:1010F00029583F4F44E050E061EB75E0CE0187583E
:101100009F4F0E944B609E0129583F4F44E451E09D
:101110006EEA74E1CE0187589F4F0E944B60E696BD
:101120001FAEE6978FEF89839E0129583F4F41E01C
:1011300050E0BE016B587F4FCE0187589F4F0E94F1
:101140004B609E0129583F4F41E050E0B801CE016D
:1011500087589F4F0E944B6080E1F82EF8018F2D39
:1011600011928A95E9F79E0129583F4F40E150E0DE
:10117000B801CE0187589F4F0E944B609E012958AD
:101180003F4F44E050E065E87EE0CE0187589F4F36
:101190000E944B609E0129583F4F4CE050E063EAAB
:1011A0007EE0CE0187589F4F0E944B609E012958D8
:1011B0003F4F44E050E06DE470E1CE0187589F4F0F
:1011C0000E944B609E0129583F4F44E050E069E483
:1011D00070E1CE0187589F4F0E944B609E012958B5
:1011E0003F4F44E050E069E87EE0CE0187589F4FD2
:1011F0000E944B609E0129583F4F44E050E06AEA4C
:1012000074E1CE0187589F4F0E944B609E01295880
:101210003F4F4CE050E061E570E1CE0187589F4FB1
:101220000E944B609E0129583F4F44E050E061E02E
:101230007FE0CE0187589F4F0E944B609E01295846
:101240003F4F44E050E066EA74E1CE0187589F4F7B
:101250000E944B609E0129583F4F42E050E064EAF3
:1012600074E1CE0187589F4F0E944B60F8011192A4
:10127000FA94E9F780E090E0A0E8BFE38D879E87CD
:10128000AF87B88B80911D1690911E16A0911F16E6
:10129000B091201689839A83AB83BC8380912116F9
:1012A00090912216A0912316B09124168D839E83CF
:1012B000AF83B8878091251690912616A0912716A6
:1012C000B091281689879A87AB87BC879E012958D9
:1012D0003F4F40E150E0B801CE0187589F4F0E9438
:1012E0004B6084E190E09A8389839E0129583F4FA7
:1012F00042E050E0B801CE0187589F4F0E944B60FA
:101300009E0129583F4F4CE050E061E176E1CE016B
:1013100087589F4F0E944B6080E290E09A838983B8
:101320009E0129583F4F42E050E0B801CE01875856
:101330009F4F0E944B6081E089839E0129583F4F57
:1013400041E050E0B801CE0187589F4F0E944B60AA
:1013500080E2E8E7F2E0D80101900D928A95E1F78A
:101360009E0129583F4F40E250E0B801CE01875816
:101370009F4F0E944B60E6961FAEE6979E0129584C
:101380003F4F41E050E0BE016B587F4FCE01875880
:101390009F4F0E944B609E0129583F4F41E050E013
:1013A0006FEA7EE0CE0187589F4F0E944B609E01FE
:1013B00029583F4F44E050E064EB7EE0CE0187586F
:1013C0009F4F0E944B608AE1F80111928A95E9F7DC
:1013D0009E0129583F4F4AE150E0B801CE0187589D
:1013E0009F4F0E944B6084E3E8E9F2E0D80101904E
:1013F0000D928A95E1F79E0129583F4F44E350E052
:10140000B801CE0187589F4F0E944B601A82198203
:101410001C821B821E821D829E0129583F4F46E07E
:1014200050E0B801CE0187589F4F0E944B608DE07D
:10143000F80111928A95E9F79E0129583F4F4DE036
:1014400050E0B801CE0187589F4F0E944B60E19653
:101450001CAE1DAE1EAE1FAEE1979E0129583F4F38
:1014600044E050E0BE0163597F4FCE0187589F4F43
:101470000E944B608CE0F80111928A95E9F79E0179
:1014800029583F4F4CE050E0B801CE0187589F4F9C
:101490000E944B608CE6F80111928A95E9F79E0153
:1014A00029583F4F4CE650E0B801CE0187589F4F76
:1014B0000E944B609E0129583F4F4CE050E065EB85
:1014C00075E0CE0187589F4F0E944B609E012958BE
:1014D0003F4F48E050E06CE974E1CE0187589F4FE0
:1014E0000E944B601091C105111159C0EB96EEACF2
:1014F000FFACEB97F4E6EF1AF108E9968EAD9FADDD
:10150000E997E7969FAF8EAFE79784E690E0EB967A
:101510009FAF8EAFEB979E0129583F4F44E050E0BC
:101520006CEF72E0CE0187589F4F0E944B609E0186
:1015300029583F4F42E050E0BE016B587F4FCE012B
:1015400087589F4F0E944B600E9448608CE692E251
:101550000E940460B70180E090E04AE00E949D6034
:10156000E7964EAD5FADE79760E070E08FE592E201
:101570000E9408618CE592E20E94046083E9E8160B
:1015800083E0F80639F00E9423608EE792E20E9421
:10159000046011E08091C105182B1093C105909152
:1015A000C10581E08927C558DF4F0FB6F894DEBF2B
:1015B0000FBECDBFDF91CF911F910F91FF90EF90A4
:1015C0000895CF93DF93CDB7DEB760970FB6F89449
:1015D000DEBF0FBECDBF80916D0690916E06A091CB
:1015E0006F06B091700689839A83AB83BC83809128
:1015F000710690917206A0917306B09174068D8366
:101600009E83AF83B8878091750690917606A091EE
:101610007706B091780689879A87AB87BC878091D7
:10162000790690917A06A0917B06B0917C068D8711
:101630009E87AF87B88B0E94E6E70F9437230E94FE
:101640000DC880E00E94EAD181E00E94EAD182E0E8
:101650000E94EAD10E94FEF10E942DE840E150E094
:101660006DE676E0CE0101960F94324E892B51F053
:1016700060960FB6F894DEBF0FBECDBFDF91CF915D
:101680000D94161F60960FB6F894DEBF0FBECDBF47
:10169000DF91CF9108952F923F924F925F926F9278
:1016A0007F928F929F92AF92BF92CF92DF92EF92F2
:1016B000FF920F931F93CF93DF93CDB7DEB7CC5933
:1016C000D1090FB6F894DEBF0FBECDBF2DB63EB622
:1016D000CB56DF4F19821882C559D04084E690E07E
:1016E000C956DF4F99838883C759D04001E09E01D6
:1016F0002B563F4F44E050E0BE016F567F4FCE0166
:1017000089569F4F0E94B65F9E012B563F4F42E085
:1017100050E0BE0167567F4FCE0189569F4F0E9411
:10172000B65F43E050E0BE016F567F4F8CEF92E012
:101730000F94814E892B39F1CC56DF4F8881C459E3
:10174000D040882359F08FE3CF56DF4F8883C159AB
:10175000D040CE56DF4F1882C259D0400E94486018
:101760008FE193E20E940460BE016F567F4F86E1D5
:1017700093E20E94126088E093E20E94046081E09C
:101780008093C105A6C5C357DF4F188219821A82FC
:101790001B82CD58D040CB56DF4F19821882C559D5
:1017A000D04001E09E012B563F4F41E050E0BE018A
:1017B00064567F4FCE0189569F4F0E94B65F4DB64B
:1017C0005EB680E1ECECF2E0DE01A358BF4F019081
:1017D0000D928A95E1F780E1ECEDF2E0DE01A3598C
:1017E000BF4F01900D928A95E1F780E1ECEEF2E0B7
:1017F0009E012F5F3F4F3901D90101900D928A95CB
:10180000E1F7C456DF4F4881CC59D04050E04D5FDE
:101810005F4F440F551F440F551F6DB77EB7641BB4
:10182000750B0FB6F8947EBF0FBE6DBF8DB79EB718
:1018300001966C010091971411E001272C563F4F3F
:10184000BC01CE0189569F4F0E94B65F009197144C
:1018500001279E012B563F4F44E050E06CE97CE0AD
:10186000CE0189569F4F0E94B65FC456DF4FE88075
:10187000CC59D040F12C93E0E90EF11CEE0CFF1C8A
:10188000EE0CFF1CADB7BEB7AE19BF090FB6F8948A
:10189000BEBF0FBEADBFEDB7FEB731965F012DB72E
:1018A0003EB72E193F090FB6F8943EBF0FBE2DBFAD
:1018B0006DB77EB76F5F7F4F4B0100919714012783
:1018C0009E012B563F4FA701BF01CE0189569F4F66
:1018D0000E94B65F0091971401279E012B563F4F3F
:1018E000A701B401CE0189569F4F0E94B65F0091B7
:1018F0009714002309F4C3C011E001279E012B5661
:101900003F4F44E050E060EC7CE0CE0189569F4FB1
:101910000E94B65F0091971401279E012B563F4FFE
:1019200044E050E064EC7CE0CE0189569F4F0E9479
:10193000B65F0091971401279E012B563F4F44E05C
:1019400050E068EC7CE0CE0189569F4F0E94B65F64
:101950000091971401279E012B563F4F44E050E021
:101960006CEC7CE0CE0189569F4F0E94B65F0091DF
:10197000971401279E012B563F4F44E050E060ED45
:101980007CE0CE0189569F4F0E94B65F009197146C
:1019900001279E012B563F4F40E150E06AE876E078
:1019A000CE0189569F4F0E94B65F00919714012780
:1019B0009E012B563F4F44E050E0BE0163577F4FDE
:1019C000CE0189569F4F0E94B65F0FB6F8945EBE57
:1019D0000FBE4DBE0091971401279E012B563F4F1D
:1019E0004CE050E0BE016F5F7F4FCE0189569F4FA4
:1019F0000E94B65F0091971401279E012B563F4F1E
:101A000044E050E0BE0163577F4FCE0189569F4F9F
:101A10000E94B65F0091971401279E012B563F4FFD
:101A200044E050E0BE0163577F4FCE0189569F4F7F
:101A30000E94B65F01E09E012B563F4F41E050E00F
:101A4000BE0163597F4FCE0189569F4F0E94B65FFA
:101A50009E012B563F4F41E050E0BE016F5F7F4F2C
:101A6000CE0189569F4F0E94B65FAE968FADAE975E
:101A7000C9808C9D60011124E12CF12C71C0C456E9
:101A8000DF4F2881CC59D04030E02E5F3F4FECE84B
:101A9000FCE080E090E02817390714F0D60111C06F
:101AA000AC018430910510F043E050E0440F551F25
:101AB000440F551F6DE770E06C0F7D1F460F571FD9
:101AC000DA014D915D916D917C91419351936193B8
:101AD00071932817390714F0D50111C0AC01843077
:101AE000910510F043E050E0440F551F440F551F7F
:101AF0006DE670E06C0F7D1F460F571FDA014D91A8
:101B00005D916D917C91408B518B628B738B28170B
:101B1000390714F0D4010DC0AC018430910510F0E8
:101B200043E050E0440F551F440F551F460D571D0D
:101B3000DA014D915D916D917C9140A351A362A317
:101B400073A30196B4E08B0E911C44E0A40EB11C6B
:101B500064E0C60ED11C8430910509F09CCFCCCE38
:101B600000919714EC14FD0491F001279E012B566F
:101B70003F4F44E050E0BE0163577F4FCE0189568E
:101B80009F4F0E94B65F7FEFE71AF70AE9CF81E027
:101B900008279E012B563F4F44E050E06FEE7EE059
:101BA000CE0189569F4F0E94B65F1AE0FF24F3943E
:101BB000115089F0009197140F259E012B563F4F2D
:101BC00044E050E0BE0163577F4FCE0189569F4FDE
:101BD0000E94B65FEDCF01E09E012B563F4F41E0E2
:101BE00050E0BE0165567F4FCE0189569F4F0E943F
:101BF000B65F9E012B563F4F41E050E0BE01635857
:101C00007F4FCE0189569F4F0E94B65FC556DF4F6A
